:100000000C94DF0D0C94100E0C94100E0C94100E2A
:100010000C94100E0C94100E0C94100E0C94100EE8
:100020000C94100E0C94100E0C94100E0C94100ED8
:100030000C94100E0C94100E0C94100E0C94100EC8
:100040000C94100E0C94100E0C94100E0C94100EB8
:100050000C94100E0C94100E0C94100E0C94089B23
:100060000C94100E0C94577D0C942D7D0C94100E56
:100070000C94100E0C94100E0C94100E0C94100E88
:100080000C94100E0C94100E0C94100E0C94100E78
:100090000C94037D0C94D97C0C94100E0C9427299D
:1000A0000C94100E0C94100E0C94100E0C94100E58
:1000B0000C94100E0C94100E0C94100E0C94100E48
:1000C0000C94100E0C94100E0C94100E0C94AF7C2B
:1000D0000C94857C0C94100E0C945B7C0C94317CFD
:1000E0000C94100E07634236B79BD8A71A3968568E
:1000F00018AEBAAB558C1D3CB7CC5763BD6DEDFD4A
:10010000753EF6177231BF000000803F0800000006
:10011000BE922449123EABAAAA2ABECDCCCC4C3EFC
:1001200000000080BEABAAAAAA3E00000000BF00EB
:100130000000803F0000000000084178D3BB4387E7
:10014000D1133D190E3CC3BD4282AD2B3E68EC82FB
:1001500076BED98FE1A93E4C80EFFFBE01C4FF7F80
:100160003F00000000000C94BD710C9447AF0C944C
:10017000BFA00C9414140C94511A0C940C570C94AA
:10018000EB170C9473150C94681B0C94B51A0C9413
:10019000FF930C94FB5A0C9474120C94B9280C9491
:1001A000BD110C94015B0C9459190C94800F0C94A4
:1001B000201C0C94861E0C94EF930C94E66E0C9409
:1001C000706F0C9428590C9498110C944D0E0C944B
:1001D000555A0C94B00F0C94E91C0C94E5930C94B4
:1001E000DF380C94B40F0C94890F0C94FD120C940E
:1001F00056200C9404710C9430180C940E1C0C9422
:10020000F11E0C947B120C94F01A0C9432160C9480
:10021000FAA90C94B9440C94F4800C941A610C94CF
:1002200093330C947B410C943B570C947D0F0C94AE
:100230003B6D0C94A35A0C94DD1E0C94CC930C943F
:10024000FB920C94A70F0C94120E0C948E130C942A
:10025000F2580C94BF120C9410110C94A5560C94E7
:10026000AB710C946B330C9431130C9454A90C9413
:10027000EB700C945A340C94BF340C94F5440C94E9
:1002800028330C94EF560C94011F0C94F7930C94A4
:100290000F9D0C94051C0C94A01B0C9419450C94F8
:1002A000BE0F0C9430340C94C30F0C94E7170C94CD
:1002B000B11D0C9409930C940D930C945E280C942E
:1002C00072210C94A5110C94F96E0C94F7220C94E5
:1002D000667F0C9481710C9456710C94D9120C9415
:1002E000A00F0C948A1B0C945E410C94C4930C9444
:1002F000860F0C941E930C9489100C94EE1B0C9496
:1003000062A90C94AE100C945B340C9427280C94C6
:10031000ED170C941F930C9478110C94DFA90C9496
:100320006B700C94EE7E0C9440940C946B120C94B5
:10033000CB0F0C9404340C948F210C94FF920C94EA
:10034000F1130C94E8380C94092E0C940B140C94B3
:1003500071120C94F8680C9489200C9400570C943A
:1003600051700C940A150C94A8130C94951B0C94C2
:1003700072710C943C1B0C942C0E0C94B7730C945F
:1003800099250C9472700C9454940C9471110C94E3
:10039000DB930C94D8590C948E280C9465320C94F1
:1003A000E5170C940B1B0C94E5720C946E0F0C94D7
:1003B0009A320C94AD120C9436940C943E330C94F7
:1003C000E30F0C9429370C941D140C94CB250C943A
:1003D0008E0F0C94F1920C94FF7E0C94B3320C941B
:1003E0003F6F0C944CA90C9490A20C944D160C9455
:1003F000ED920C9456210C94626F0C94011C0C9499
:1004000051150C94BC1D0C94C5170C94823B0C9494
:100410003E340C940E560C94BE680C94C7130C9486
:100420001E340C94E3920C9413930C94221F0C949E
:10043000C56F0C94BB120C94F7920C9493190C9406
:10044000FA330C9443640C9437720C94E3560C9476
:1004500080320C94B17F0C94FD560C9485340C942E
:10046000C2120C94A22A0C946E120C946F720C940B
:1004700077590C94F51B0C9491100C94F86E0C9415
:1004800024310C94FE5A0C94AEA70C9499410C9410
:10049000420E0C944B560C94AB590C946E5A0C941F
:1004A0007F2F0C9451110C940C700C94DC440C9420
:1004B00029160C947F1B0C945A110C94F6270C945B
:1004C000B8A30C944A340C9472130C94EF200C943F
:1004D0003E270C94280E0C94BC270C949F0F0C9470
:1004E000AC0F0C941F7F0C943E200C94F1590C948B
:1004F000F2560C94DDA80C941D9F0C941A200C94B9
:100500004A200C9467330C9445340C9414160C94C4
:10051000D9330C948B520C94B8250C94C4710C9460
:10052000087F0C9439370C949A160C949F110C94F4
:10053000B9560C9425150C9488340C94C00F0C9467
:1005400013940C944E6F0C9429AF0C94CB690C94BB
:1005500006210C94AE110C9474380C94B8700C9461
:100560008D120C94FC440C94EC140C94E7920C94B3
:1005700079140C94DD220C94DF920C9469110C9484
:10058000BB720C94DF600C94910F0C94CC560C94BD
:10059000225B0C9409940C944A940C947B700C94F8
:1005A0007F130C94B11B0C9426780C942C940C940F
:1005B00082A90C9405930C941B930C94CF0F0C946C
:1005C0001D940C945E940C94850F0C949D320C94A5
:1005D000335A0C945B1B0C94A3330C945E590C940B
:1005E000BD410C94D30F0C94BA100C944E640C942F
:1005F0007C0F0C94C3330C94E2410C94DF340C94C4
:1006000075700C94787F0C9432110C94201E0C940D
:10061000A0650C941D1C0C94E9170C94DE1A0C9424
:100620004A440C94D1930C94111F0C948C440C9458
:1006300017930C9467180C945B330C941D330C9433
:10064000E2380C94D9920C9457726364696E6F709F
:10065000737578585B00556E6B6E6F776E2073758F
:10066000666669782000556E6B6E6F776E20636DDD
:10067000642000636C724374723A20005365656BAA
:100680003A002F00496E3A20003D00494E3A003DA5
:10069000004C454741435920494E3A000000200094
:1006A0002300260029002C002F003200000100004A
:1006B0000301060109012D3E00200023002D3E000C
:1006C000200050656E6465643A20230072617700F3
:1006D00076616C0074656D70007361740068756597
:1006E0000066616E0052474200485356006D6F64C9
:1006F0006500536574436D643A0053746F726564AA
:10070000204558543A00737566666978436F64658E
:100710003A004452590046414E5F4F4E4C590058E2
:100720004F4E0048414C54002074696D653A0043B7
:1007300074726C205265733A002054533A0020546E
:100740003A003D0050696E3A004F4E3A416C726576
:10075000616479204163746976650A0048414C54AC
:100760003A416C726561647920496E61637469769F
:10077000650A00584F4E3A416C72656164792041B8
:1007800063746976650A00584F464620736B69703A
:100790007065642E205072657620636D643A005453
:1007A00075726E6564206F66662066726F6D3A00C2
:1007B000526573746F7265642066726F6D3A00499A
:1007C000676E6F7265642C206368616E6E656C2065
:1007D000636D643D0020457865633A004163746948
:1007E00076653A0048414C543A416C7265616479CF
:1007F00020496E6163746976650A00584F4E3A412C
:100800006C7265616479204163746976650A005889
:100810004F464620736B69707065642E2050726578
:100820007620636D643A005475726E6564206F665D
:10083000662066726F6D3A00526573746F726564FC
:100840002066726F6D3A002044697361726D656451
:1008500000206D73203A0041726D656420666F72EE
:1008600020004F75744F664D656D6F7279210A00D7
:1008700020436D643A00205375623D002049746541
:100880006D3D0052414D3D00282D292000282B2987
:1008900020002076616C7565206973200020756EDC
:1008A0006B6E6F776E0A005D3D005B0020696E76AF
:1008B000616C6964002000206F6B003A0020666163
:1008C000696C6564003A005265747279696E6720DC
:1008D0006D6F6462757320434D440A002073656335
:1008E0002072656D61696E696E670053746174751D
:1008F000732064656666657265640A002D3E00506B
:1009000075623A2000636D6400434F4F4C004845C8
:100910004154004155544F002D3E005075623A201D
:10092000007365740064656C002D3E005075623A7A
:1009300020002D3E005075623A2000556E6B6E6FA0
:10094000776E20636D64200A004F4646004F4E00CC
:1009500020002D3E00436F6E76657274696E6720CD
:10096000002D3E0057726F6E672041737369676E8A
:100970006D656E742000524742783A200020764C14
:100980006576656C3A0020436F6E76563A002043D8
:100990006F6E76533A0020486F743A00436F6C6470
:1009A0003A0020436F6E76657274656420563A0093
:1009B000436F6E76657274656420533A002D3E0075
:1009C00057726F6E672041737369676E6D656E74E1
:1009D00020002D3E0057726F6E6720417373696768
:1009E0006E6D656E74200053617665643A00000098
:1009F000000000000000004F4E000000000000005A
:100A00004F464600000000000052455354000000CD
:100A10000000544F47474C4500000048414C5400EB
:100A200000000000584F4E000000000000584F46E4
:100A3000460000000000494E4352454153450044E2
:100A4000454352454153450048454154000000008C
:100A500000434F4F4C00000000004155544F000030
:100A600000000046414E5F4F4E4C59004452590021
:100A7000000000000053544F50000000000048499F
:100A8000474800000000004D454449554D00000016
:100A90004C4F570000000000005452554500000024
:100AA000000046414C534500000000454E41424C79
:100AB0004544000044495341424C4544005247429A
:100AC0000000000000004853560000000000002015
:100AD000537566663A002041543A00436D643A20EB
:100AE00000504F5354202F636F6D6D616E642F0063
:100AF000474554202F6974656D2F00504F53542083
:100B00002F6974656D2F004C6F636174696F6E3A65
:100B100020687474703A2F2F6C617A79686F6D65F4
:100B20002E72752F7077613F6D61633D00474554AC
:100B3000202F00536B697070696E672E2E004F7501
:100B4000744F664D656D6F727921005D20003A5BD0
:100B5000000A003A004D41433A0055445020537971
:100B6000736C6F6720696E697469616C697A65641A
:100B70002E0A005379736C6F6720706172616D7318
:100B80003A0043757272656E74204C414E20636F5B
:100B90006E6669672869702C646E732C67772C7396
:100BA00075626E6574293A000A557365207468652C
:100BB000736520636F6D6D616E64733A202768659D
:100BC0006C7027202D207468697320746578740A0E
:100BD000276D61632064653A61643A62653A6566CF
:100BE0003A66653A3030272073657420616E642060
:100BF00073746F7265204D41432D61646472657337
:100C00007320696E20454550524F4D0A2769702068
:100C10005B69705B2C646E735B2C67775B2C737500
:100C2000626E65745D5D5D5D27202D2073657420A7
:100C30007374617469632049500A2773617665276C
:100C4000202D20736176652063757272656E742045
:100C5000636F6E66696720696E204E5652414D3B48
:100C6000204F4E7C4F4646202D20656E61626C659C
:100C70002F64697361626C65206175746F7361764E
:100C8000650A2767657427205B636F6E6669672056
:100C9000616464725D27202D2067657420636F6E28
:100CA0006669672066726F6D207072652D636F6E66
:100CB000666967757265642055524C20616E6420C8
:100CC00073746F726520616464722C204F4E7C4F88
:100CD0004646202D20656E61626C652F64697361E4
:100CE000626C6520646F776E6C6F6164206F6E203C
:100CF000737461727475700A276C6F616427202D9C
:100D0000206C6F616420636F6E6669672066726F26
:100D10006D204E5652414D0A2770776427202D20B2
:100D2000646566696E6520616E642073746F7265B8
:100D3000204D5154542070617373776F72640A2789
:100D40006F746170776427202D20646566696E6515
:100D500020616E642073746F726520485454502073
:100D60004150492070617373776F72640A276C6F0A
:100D700067205B73657269616C5F6C6F676C657629
:100D8000656C5D205B7564705F6C6F676C65766524
:100D90006C5D27202D20646566696E65206C6F6729
:100DA000206C6576656C2028302E2E37290A276B3B
:100DB000696C6C27202D20746573742077617463CF
:100DC00068646F670A27636C65617227202D206352
:100DD0006C65617220454550524F4D0A277265621D
:100DE0006F6F7427202D207265626F6F7420636FA0
:100DF0006E74726F6C6C657200536F6674207265EE
:100E0000626F6F74696E672E2E2E0052414D3D0049
:100E10000A6D71747420000A696E70757473200015
:100E20000A6974656D7320000A436F6E66696775A1
:100E30007265643A003B003D0050696E3A003B0029
:100E40003D4C4F5700546865726D6F3A004C6F61AE
:100E5000646564006C6F6164206661696C65640040
:100E60004E6F2073746F72656420636F6E6669677E
:100E7000004C6F6164696E6720436F6E666967201E
:100E800066726F6D20454550524F4D00436F6E6640
:100E90006967206175746F736176653A000A5379EA
:100EA000736C6F67206465627567206C6576656C2E
:100EB0003A0053657269616C206465627567206CE5
:100EC0006576656C3A0053617665640A0053657413
:100ED0002064796E616D69632049500A0045455070
:100EE000524F4D20636C65617265640A004D515428
:100EF000542050617373776F7264207570646174ED
:100F000065640A004F54412050617373776F7264B7
:100F100020757064617465640A00636F756C642089
:100F20006E6F742070617273653A20005570646151
:100F30007465640A004C6F6164696E67204854549C
:100F40005020636F6E666967206F6E2073746172E4
:100F50007475703A004F4646004F4E002B002D002E
:100F6000485454502F312E312025690020485454C4
:100F7000502F312E310D0A486F73743A2025730DAE
:100F80000A4163636570743A202A2F2A0D0A436F61
:100F90006E6E656374696F6E3A20636C6F73650D76
:100FA0000A0025730020000D0A00474554006661C1
:100FB000696C656420746F20636F6E6E6563740A7C
:100FC000004552524F523A20536572766572207234
:100FD000657475726E65642000446F6E652E0A003C
:100FE0004170706C79696E672E0A00436F6E666996
:100FF000672070617273696E67206661696C6564F1
:101000000A00676F7420436F6E6669670A00726535
:1010100074636F6465200068636C69656E74006654
:101020007265652000436F6E666967205552493AC4
:1010300020687474703A2F2F002044656661756CC7
:101040007420636F6E6669672073657276657220BF
:10105000757365643A20006C617A79686F6D652EEE
:10106000727500205361766564000A282D294D446D
:101070004E53000A282D29554152544252494447A3
:1010800045000A282B295359534C4F47000A282D55
:1010900029504944000A282D294D4350323330311C
:1010A00037000A282D294152544E4554000A282B56
:1010B000294F5441000A282D29535049204C4544BA
:1010C000000A282D294D4F544F5220435452000AF4
:1010D000282B294143204841494552000A282D29FF
:1010E000434353383131202620484443313038308F
:1010F000000A282B29524553544152545F4C414E0B
:101100005F4F4E5F4D5154545F4552524F52530002
:101110000A282D294841524452455345542C2075E4
:1011200073696E6720736F6674000A282D29434F18
:10113000554E544552000A282D29444854000A2887
:101140002D294F57495245000A282D294D4F444219
:101150005553000A282D29444D58000A282B295799
:10116000697A6E657435783030000A282B2944532B
:10117000323438322D313030000A282B294672653E
:101180006552616D207072696E74696E6700646586
:101190003A30313A32333A30303A30303A30310046
:1011A0000A4669726D77617265204D414320416442
:1011B000647265737320006C617A79686F6D652E57
:1011C0007275000A436F6E66696720736572766593
:1011D000723A000A282B295741544348444F47008C
:1011E0003230313130334C0020432B2B2076657266
:1011F00073696F6E3A00303334333139655F3230A2
:1012000032312D31302D3038000A4C617A79686FD7
:101210006D652E7275204C6967687448756220632D
:101220006F6E74726F6C6C65722000204F464600C2
:10123000204F4E00757074696D6500667265656853
:10124000656170002054696D65723A00204C6F63CF
:101250006B733A002000204C6F636B733A000A52A4
:10126000414D3D0020457870697265640A00202D6B
:10127000746172676574207A6F6E652D0020416C11
:1012800061726D20457870697265640A0020636D33
:10129000643A00204375723A00205365743A005353
:1012A0006176656420746F20454550524F4D005360
:1012B0006176696E6720636F6E66696720746F2060
:1012C000454550524F4D2E2E002069732000446535
:1012D0006C6574696E6720636F6E662E2052414D97
:1012E000207761733A0053746F70706564005374B3
:1012F0006F7070696E67206368616E6E656C7320D5
:101300002E2E2E004E6F7420756E6C6F636B6564AD
:1013100020696E20313073202D20636F6E74696EEA
:101320007565202E2E2E00556E6C6F636B696E678F
:1013300020636F6E666967202E2E2E004552520084
:101340004C4F57004D454449554D004849474800CA
:1013500046414E5F4F4E4C5900445259004845415A
:101360005400434F4F4C004155544F007261770079
:101370007175656974007377696E67006C6F636B74
:101380000044656661756C742073657269616C20D8
:101390006D6F6465204E3831207573656400384583
:1013A00031002600384E31000600384532002E004C
:1013B000384E32000E00384F31003600384F3200C0
:1013C0003E00374531002400374532002C00374FAE
:1013D00031003400374F32003C00374E31000400FA
:1013E000374E32000C00203D3E002C002C002C001B
:1013F0002C00456C657661746F723A20636F6E667F
:101400006967206661696C65643A00456C65766160
:10141000746F7220636F6E666967206572726F7297
:1014200000456C657661746F7220636F6E666967E4
:10143000206C6F616465642000456C657661746F33
:10144000723A204F7574206F66206D656D6F7279EA
:10145000003C003E00556E6B6E6F776E20737566B4
:101460006669782000556E6B6E6F776E20636D64D1
:101470002000536574206E6F7420696D706C656D0B
:10148000656E74656400466F726365642065786597
:10149000637574696F6E004D756C746956656E7412
:1014A00020636F6E666967206661696C6564004DD4
:1014B000756C746956656E7420696E6974004D753B
:1014C0006C746976656E742044652D496E6974008C
:1014D000204F75743A00206D33002066726F6D20C6
:1014E00000204D617820726571756573743A002033
:1014F00066616E253A002061637469766520563A0C
:1015000000546F74616C20563A0050574D2D4F7542
:101510007420496E69740050574D2D4F75742073B7
:10152000746F70005247422050574D002050574D65
:1015300000524742572050574D003D0050696E3AC7
:10154000005B305D3A2000202D202D202D20EFBBA8
:10155000BF003E003E31202D200020002E00696E8D
:1015600000735F6F7574006D79686F6D6500202D75
:101570003E2000456D69743A2000202D3E20004930
:1015800074656D436D643A2000202D3E200049743F
:10159000656D3A20003E3E2000496E76616C6964BC
:1015A00020636F6D6D616E64003E3E3E004E6F20A5
:1015B0004D414320636F6E666967757265643A20BA
:1015C000736574206669726D776172652773204D4B
:1015D00041430A004E6F2076616C69642045455096
:1015E000524F4D206461746100476F742049502050
:1015F000616464726573733A00276970205B697077
:101600005B2C646E735B2C67775B2C7375626E6505
:10161000745D5D5D5D27202D20736574207374619A
:101620007469632049500A004661696C65642074DE
:101630006F20636F6E6669677572652045746865B3
:10164000726E6574207573696E6720444843502E2E
:1016500020596F752063616E207365742069702056
:101660006D616E75616C6C7921000A75736573200C
:10167000444843500A00204D41534B3A00204757FD
:101680003A0020444E533A004C6F61646564206612
:10169000726F6D20666C6173682049503A00537414
:1016A000617274696E67206C616E0041424344450B
:1016B000464748494A4B4C4D4E4F50515253545552
:1016C000565758595A6162636465666768696A6B00
:1016D0006C6D6E6F707172737475767778797A301D
:1016E0003132333435363738392B2F3D004F5441A2
:1016F00020696E697469616C697A65640A004445A1
:101700004641554C542070617373776F7264206644
:101710006F72204F5441204150492E20557365204F
:101720006F746170776420636F6D6D616E64207497
:101730006F2073657400757074696D652C667265D1
:1017400065686561700024737461747300303334AC
:10175000333139655F323032312D31302D30380040
:101760004C696768744875622000246E616D65007D
:10177000726561647900546F6F206D616E79204DE0
:1017800051545420636F6E6E656374696F6E20658B
:1017900072726F72732E2052657374617274204C72
:1017A000414E002074727920616761696E20696E14
:1017B0002035207365636F6E6473006661696C65C4
:1017C000642C2072633D004177616974696E672003
:1017D000666F722072657461696E656420746F70E3
:1017E00069637300636F6E6E656374656420617313
:1017F0002000202E2E2E0020757365723A003A00CC
:101800000A417474656D7074696E67204D5154544B
:1018100020636F6E6E656374696F6E20746F200055
:1018200024737461746500646973636F6E6E6563BD
:10183000746564005573696E67204D51545420706F
:10184000617373776F72642066726F6D20636F6E61
:1018500066696700446576696365204E616D653A27
:1018600000526562696E6420737563636573732EDD
:1018700020495020616464726573733A0045727246
:101880006F723A20726562696E64206661696C00ED
:1018900052656E6577656420737563636573732E37
:1018A00020495020616464726573733A0045727216
:1018B0006F723A2072656E65776564206661696C47
:1018C000000A4E6F206C696E6B0041636365707433
:1018D000696E6720636F6D6D616E64732E2E2E0AC4
:1018E000004E6F204D51545420636F6E66696775CA
:1018F0007265640044454C455445005055540047BA
:10190000455400504F535400617574686F72697A82
:101910006174696F6E3A2000417574686F72697AFC
:101920006174696F6E3A2000436F6E74656E742D3A
:101930004C656E6774683A2000000021002400277F
:10194000002A002D003000330001010000040107CF
:10195000010A0100002200250028002B002E003182
:1019600000340002010000050108010B0105050516
:1019700005070508080808020202020A0A08080406
:101980000404040101010101010101030303030334
:10199000030303040707070C0C0C0C0C0C0C0C02C3
:1019A00002020206060606060606060B0B0B0B0BCA
:1019B0000B0B0B050505080807070404040A0A0AAF
:1019C0000A0A0A01021020200808102040102040B6
:1019D00080020102010804020101020408102040F3
:1019E0008080402010080402018004020180402011
:1019F000100804020108040201010204081020403A
:101A000080010204081020408004408004800810F7
:101A100010204004081020408000000B0C030A0D29
:101A20000E0F09080405020000000000000000007D
:101A300000000000000000000000000000000000A6
:101A40000000000000131211000000000000000060
:101A50000000000000000000000000000000000086
:101A60000000000000000000000000000000006F07
:101A7000637465742F73747265616D00696D61675D
:101A8000652F6A70656700696D6167652F676966B4
:101A900000746578742F68746D6C00746578742FA9
:101AA0006A736F6E00746578742F706C61696E0074
:101AB000436F6E74656E742D547970653A200043DF
:101AC0006F6E6E656374696F6E3A20636C6F7365D9
:101AD00000556E6B6E6F776E004F4B004D6F7665E5
:101AE00064207065726D616E656E746C7900496E0C
:101AF0007465726E616C20536572766572204572F2
:101B0000726F72005061796C6F616420546F6F2046
:101B10004C61726765004E6F7420666F756E64006D
:101B20005757572D41757468656E746963617465A4
:101B30003A204261736963207265616C6D3D224198
:101B4000636365737320726573747269637465642B
:101B50002200556E617574686F72697A6564005011
:101B600061796C6F61642073697A652077726F6E3A
:101B700067004261642072657175657374002000AE
:101B8000485454502F312E312000202D3E204154F6
:101B90003A004368616E20747970653A004E6F2098
:101BA00073746F7265642076616C756573202D2087
:101BB00064656661756C743A200047AF29AF1124E3
:101BC0001FBECFEFD1E2DEBFCDBF00E00CBF17E0FC
:101BD000A0E0B2E0EAE9F8E801E00BBF02C007903C
:101BE0000D92AC34B107D9F72EE0ACE4B7E001C0F8
:101BF0001D92A03DB207E1F71DE0CEEDDDE000E073
:101C000006C021970109802FFE010E940BBFCD3D28
:101C1000D10780E00807A9F70E946F9B0C943BC492
:101C20000C940000CF93DF931F92CDB7DEB769838A
:101C3000DC01ED91FC910280F381E02D41E050E068
:101C4000BE016F5F7F4F19950F90DF91CF9108957F
:101C5000FC01818D928D0895CF93DF931F92CDB7B4
:101C6000DEB76983DC01ED91FC910280F381E02D08
:101C700041E050E0BE016F5F7F4F19950F90DF91FB
:101C8000CF910895FC019485FB018485981303C0CE
:101C900081E0983008F080E00895CF93DF931F92A1
:101CA000CDB7DEB76983DC01ED91FC910280F38151
:101CB000E02D41E050E0BE016F5F7F4F19950F901E
:101CC000DF91CF91089585ED8093BC008091BC0099
:101CD00084FDFCCF1092E00808952091BC08260FE7
:101CE0003327331F21323105ECF42091E008FC0149
:101CF00090E080E0243069F082E00895A091BC0873
:101D00002191AC014456574FA40FB52FB11D2C9310
:101D10000196861798F38091BC08680F6093BC0801
:101D200080E0089581E008958FEF9FEF08958FEF91
:101D30009FEF089580919B0890E09195819591097E
:101D40000895CF93DF93CB01EA01642F0E946D0EBB
:101D5000CE01DF91CF910895CF93DF931F92CDB73E
:101D6000DEB7698361E0CE0101960E946D0E81E0CD
:101D700090E00F90DF91CF9108958F929F92AF9254
:101D8000BF92CF92DF92EF92FF920F931F93CF9368
:101D9000DF9300D000D000D01F921F92CDB7DEB7E6
:101DA0007C018E010F5F1F4F68018AE0882E912C05
:101DB000A12CB12CC601801B910B41155105610569
:101DC000710581F0CB01BA01A50194010E9480BE8A
:101DD000942F852F605DF60161936F01A901692F32
:101DE000782FE8CFF801E80FF91FD701015011094A
:101DF00022912D93E017F107D9F7E80EF91EF701AC
:101E000010822B960FB6F894DEBF0FBECDBFDF91C8
:101E1000CF911F910F91FF90EF90DF90CF90BF90E7
:101E2000AF909F908F900895FC01DC018D918111FE
:101E3000FDCF30E020E050E040E08AE0919199232E
:101E400001F1443051055CF59E3271F42F3F3105AC
:101E500009F02CF5DB01A40FB51F12962C934F5FF0
:101E60005F4F30E020E0EACF829FD001839FB00D2A
:101E70001124292F990F330B205331092A0F3B1FAF
:101E8000DDCF2F3F310509F054F4443051053CF4C7
:101E9000640F751FFB01228381E090E0089590E0BC
:101EA00080E00895CF93DF931F921F92CDB7DEB7E6
:101EB0008091C40E9091C50E009711F480ED9EE0C4
:101EC000BE016F5F7F4F681B790B072E000C880BDC
:101ED000990B0F900F90DF91CF910895DC0115962B
:101EE0008D919C91009739F0DC01ED91FC91068079
:101EF000F781E02D19940895089590E080E0089509
:101F000080914308909144080895089583E090E0FB
:101F100008958091410890914208089584E090E0EE
:101F20000895DC011496ED91FC91309729F08081A1
:101F3000082E000C990B089590E080E00895089514
:101F400080918A0790918B078170992708958091DD
:101F5000790790917A070895FC018481958108950D
:101F6000FC01768765870895DC01ED91FC91068C74
:101F7000F78DE02D199591E089270895862F089512
:101F800081E08627089521E0FC018485883008F0EF
:101F900020E0822F0895FC01848595850895FC0139
:101FA00084899589089520E034E0FC013183208301
:101FB000FB014089518962897389FC014283538303
:101FC000648375830895DC01ED91FC91048CF58D9B
:101FD000E02D1994CF93DF9300D000D01F921F9271
:101FE000CDB7DEB7FC01862F8F706281607F682BD2
:101FF000628388E0DE01119601900D928A95E1F7E7
:1020000029813A814B815C816D817E818F819885A8
:1020100028960FB6F894DEBF0FBECDBFDF91CF91EB
:102020000895CF93DF9300D000D01F921F92CDB7B9
:10203000DEB7FC01608398E0DE01119601900D92FD
:102040009A95E1F729813A814B815C816D817E818E
:102050008F81988528960FB6F894DEBF0FBECDBF4E
:10206000DF91CF910895CF93DF9300D000D01F92DE
:102070001F92CDB7DEB7FC016F3F710519F014F068
:102080006FEF70E077FD60E09281892F82958F700D
:1020900081508230C8F4648388E0DE01119601909B
:1020A0000D928A95E1F729813A814B815C816D819E
:1020B0007E818F81988528960FB6F894DEBF0FBE7B
:1020C000CDBFDF91CF9108959F7090619283E3CF50
:1020D0000F931F93CF93DF93DC01C62F1296EC91E1
:1020E0001297E295EF70EC3008F0BCC0F0E0882762
:1020F000E358FF4E8F4F0C940BBF8910AE10AE10FB
:102100003211321132111011BA10321132119110F4
:10211000911070E060E0CB01DF91CF911F910F91A2
:10212000089514968D919D910D90BC91A02D8F3F97
:102130009105A105B10529F024F08FEF90E0A0E012
:10214000B0E0B7FF03C080E090E0DC016FEF70E02B
:10215000681B790BC111DFCFBC01DDCF14966C91E8
:1021600070E0CC23C1F28FEF90E09C01261B370B6F
:10217000B901D1CF862F14960C91149715961C9106
:1021800015971696DC9116971796CC9120E030E0C3
:10219000A901B801882331F18D2F9C2F0E9436BDF3
:1021A00087FD1BC020E030E04FE753E4B8018D2FDE
:1021B0009C2F0E943EC0181624F400E010E0DFE7D8
:1021C000C3E498014D2F5C2F60E070E08FE793E44B
:1021D0000E9429BF0E9408C09ECF00E010E0D0E01E
:1021E000C0E0EFCF8D2F9C2F0E9436BD87FD13C01E
:1021F00020E030E04FE753E4B8018D2F9C2F0E9480
:102200003EC0181624F400E010E0DFE7C3E4B80194
:102210008D2F9C2FDFCF00E010E0D0E0C0E0F7CFA3
:1022200014966D917D918D919C9117972AE030E0E5
:1022300040E050E00E94A2BE2F3F3105410551050C
:1022400029F024F02FEF30E040E050E057FF03C0CA
:1022500020E030E0A9016FEF70E0621B730BC11149
:102260005ACF86CF6FEF7FEF56CFDC011296EC91FD
:102270001297E295EF70E150EB3008F039C0F0E0D2
:102280008827EA5BFE4E8F4F0C940BBF69116911D2
:102290007811511151115A1171117111711151119E
:1022A000511114966D917D918D919C9117970E947B
:1022B0003DBD089514966D917D918D919C911797D8
:1022C0002AE030E040E050E00E94A2BECA01B9011D
:1022D000EECF14966C9170E090E080E00E943BBDE0
:1022E000089514966D917D918D919C911797089505
:1022F00060E070E0CB010895DC011296EC9112973A
:10230000E295EF70E150EB3008F037C0F0E088273D
:10231000E357FE4E8F4F0C940BBF9F119F11BD11C1
:1023200098119811AE11A511A511A5119811981128
:1023300014966D917D918D919C91179708951496A7
:102340006C9170E090E080E0089514966D917D911D
:102350008D919C9117970E9408C0089514966D91D5
:102360007D918D919C9117972AE030E040E050E0FC
:102370000E94A2BECA01B901089560E070E0CB01DD
:102380000895FC01A7812A2F2E7FD1F082818295AA
:102390008F7081508330A0F4A695A150BB0B2BE524
:1023A00031E00E9422BF24E630E040E050E00E948D
:1023B000A2BEDA01C90187569F4FAF4FBF4F0895A4
:1023C0008FEF9FEF0895CF93DF93EC018A81982FD1
:1023D00092959F7041F180E0943010F59B01770F4A
:1023E000440B550B2959310941095109A4E6B0E0C4
:1023F0000E94C1BE2BE531E040E050E00E94A2BE49
:1024000037FF02C030E020E02536310514F024E625
:1024100030E02F5F220F8F818170282B2F8381E086
:10242000DF91CF9108958F7080628A83D7CFFC01AE
:102430009281892F82958F7021F0823029F080E07F
:1024400008959F70906292839B0177FF02C030E0F5
:1024500020E02E3681E0380714F02DE631E02683A7
:10246000878130FB80F9878381E00895DC01ED915D
:10247000FC91309729F090859F7081E0953009F0AC
:1024800080E00895DC011496ED91FC91159730974A
:1024900099F090859F708EEF890F823010F0911126
:1024A0000BC041875287638774871496ED91FC9126
:1024B0008085807F826080870895DC0119968D91E8
:1024C0009C91009739F0DC01ED91FC910280F38141
:1024D000E02D199408958AE090E0089581E090E05D
:1024E000089588E090E00895DC01ED91FC9106806C
:1024F000F781E02D1994CF93DF93EC01E881F98106
:102500000484F585E02D199529893A892F5F3F4F7D
:102510003A8B298BDF91CF910895CF93DF93EC0114
:102520008E8581110DC081E090E049895A892C8502
:102530003D854217530708F080E0DF91CF91089561
:10254000E881F9810484F585E02DCE0119958F3F4E
:10255000910549F780E090E0F0CFDC011E962C91C8
:102560001E97222339F0ED91FC910190F081E02D2E
:102570006FEF19940895FC0187859089089590E084
:1025800080E00895FC0122813381232B49F086816C
:1025900097818130910539F01CF00397029730F054
:1025A00090E080E0089581E090E0089582E090E07E
:1025B0000895CF93DF93CDB7DEB760970FB6F89449
:1025C000DEBF0FBECDBF19821A821B821C821D8204
:1025D0001E821F8218868B818F708B836FEF70E055
:1025E000CE0101960E94331060960FB6F894DEBFBC
:1025F0000FBECDBFDF91CF910895CF92DF92EF92C2
:10260000FF920F931F93CF93DF93CDB7DEB7609701
:102610000FB6F894DEBF0FBECDBF7C016B01BA01CF
:10262000A901CE0101960E94BD0ED701ED91FC914A
:102630000288F389E02D9801AE014F5F5F4FB6012C
:10264000C701199560960FB6F894DEBF0FBECDBFD7
:10265000DF91CF911F910F91FF90EF90DF90CF907E
:102660000895CF92DF92EF92FF920F931F93CF9333
:10267000DF9300D000D0CDB7DEB78C016B017A01BB
:10268000FC01808D883010F40E94808680E094E008
:102690009A838983F60182819381A481B5818B839A
:1026A0009C83AD83BE83B701CE0101960E94D79172
:1026B000F801808F8830A0F4F586E486128E118EA2
:1026C00081E026960FB6F894DEBF0FBECDBFDF9136
:1026D000CF911F910F91FF90EF90DF90CF900895D1
:1026E00080E0EFCFCF93DF93EC01888D883020F42A
:1026F0000E94808688E0888FDF91CF910895FC0149
:10270000808D883040F4218D328D232B21F00E9462
:10271000528590E008958FEF9FEF0895CF93DF9358
:10272000FC012485283028F08FEF9FEFDF91CF91B7
:102730000895EC010190F081E02D0084F185E02DF9
:102740001995892B89F38C850E94528590E0EECFF4
:10275000CF93DF93FC01218D328D2115310529F4B2
:102760008FEF9FEFDF91CF910895EC01808D42179D
:10277000530708F0A9010E94A1851816190684F7CD
:10278000298D3A8D281B390B3A8F298FEBCF0F9368
:102790001F93CF93DF931F92CDB7DEB7FC01218D3E
:1027A000328D232B41F48FEF9FEF0F90DF91CF916C
:1027B0001F910F9108958C0141E050E0BE016F5FC1
:1027C0007F4FFC01808D0E94A185181619065CF7C9
:1027D000F801818D928D0197928F818F898190E090
:1027E000E4CFCF93DF931F92CDB7DEB741E050E047
:1027F000BE016F5F7F4FFC0184850E94A185181682
:10280000190634F4898190E00F90DF91CF910895FB
:102810008FEF9FEFF9CFFC018485883010F40C9482
:10282000A18590E080E00895FC018485883010F453
:102830000C947A8590E080E008950F931F93CF93D6
:10284000DF9300D000D01F921F92CDB7DEB78C016E
:10285000D80159964D915C915A974115510551F007
:10286000ED91FC91048CF58DE02D70E060E0C801E5
:102870001995EECFF801808D0E947A85892BB1F1F0
:1028800048E050E0BE016F5F7F4FD80158968C91B1
:102890000E94A18518161906F4F4D801509684E018
:1028A000FE01319601900D928A95E1F78D8190E0BD
:1028B000982F88272E81820F911DF801958B848B8C
:1028C0008F81282F30E0322F22278885820F932F87
:1028D000911D928F818F28960FB6F894DEBF0FBEA0
:1028E000CDBFDF91CF911F910F91089590E080E0CF
:1028F000F2CFCF92DF92EF92FF920F931F93CF937D
:10290000DF93CDB7DEB7AF970FB6F894DEBF0FBE3B
:10291000CDBF7C016A0100E014E01A8309831C86A4
:102920001B8688EE93E0A0E0B0E08D879E87AF879E
:10293000B88B86ED93E09A878987188F0F8B198E55
:102940001A8E1B8E1C8E88E089A31BA70AA71CA6C3
:102950001DA61EA61FA68091600C9091610CA091EF
:10296000620CB091630C8EA39FA3A8A7B9A78B8319
:102970009C83AD83BE8318861F82AE01465D5F4F88
:10298000CE0101960E94A39881309105B1F4D70140
:10299000ED91FC910488F589E02D1DA30CA38CA575
:1029A0009DA5AEA5BFA58EA39FA3A8A7B9A7A60165
:1029B000BE016C5D7F4FC7011995AF960FB6F894B5
:1029C000DEBF0FBECDBFDF91CF911F910F91FF9062
:1029D000EF90DF90CF9008950F931F93CF93DF93E5
:1029E000EC018B01888D883010F40E948086B8013C
:1029F00082E00E94C986888F883050F41D870C873A
:102A00001A8E198E81E0DF91CF911F910F91089559
:102A100080E0F9CF0F931F93CF93DF938C01EA01EE
:102A2000FC018485883048F40E94F084892B39F4B5
:102A300081E090E0F80193838283D0E0C0E0CE0192
:102A4000DF91CF911F910F910895EF92FF920F9315
:102A50001F93CF93DF937C0180914F0AD4E083339F
:102A600009F0D8E00FE31AE0C0E0F80121913191BC
:102A70008F01F701848195812817390729F0CF5FED
:102A8000DC13F3CF80E006C08C2F0E948E86843149
:102A9000B1F781E0DF91CF911F910F91FF90EF90FF
:102AA0000895CF93DF93EC018C858830D0F40E9499
:102AB0008E86843189F0882379F0883169F021E0AD
:102AC0008C3159F4E881F9810084F185E02DCE0143
:102AD000199521E0892B09F420E0822FDF91CF9115
:102AE000089580E0FBCFCF92DF92EF92FF920F9399
:102AF0001F93CF93DF93CDB7DEB7AF970FB6F894A0
:102B0000DEBF0FBECDBF8C016B017A0180E094E087
:102B10009A8389831B821C821D821E821C861B86CF
:102B200048EE53E060E070E04D875E876F87788BFA
:102B300026ED33E03A872987988F8F8B198E1A8E6E
:102B40001B8E1C8E28E029A39BA78AA71CA61DA666
:102B50001EA61FA6D8011C968C91883060F40E9496
:102B60008E86882321F0F80184850E94728688E091
:102B7000D8011C968C938091600C9091610CA0916F
:102B8000620CB091630C8EA39FA3A8A7B9A78B83F7
:102B90009C83AD83BE8318861F82AE01465D5F4F66
:102BA000B601CE0101960E94A3980097C1F0D8010A
:102BB000ED91FC910684F785E02D80E094E09DA3E3
:102BC0008CA38CA59DA5AEA5BFA58EA39FA3A8A7EA
:102BD000B9A7A701BE016C5D7F4FC8011995AF96DB
:102BE0000FB6F894DEBF0FBECDBFDF91CF911F911E
:102BF0000F91FF90EF90DF90CF900895CF93C82F63
:102C00000E94B09504C09695879577956795CA956B
:102C1000D2F7611571058105910521F461E070E03D
:102C200080E090E0CF910895CF93DF93EC018C8505
:102C3000883060F40E948E86873111F08C3131F437
:102C40008C850E94D3848115984088F3DF91CF91C1
:102C50000895FC018485883010F40C94D38490E0AE
:102C600080E008956EEB74E185E99DE00E94CA78EA
:102C700085E99DE00E94C1771092420810924108B8
:102C800081E090E008956CE57FE0811102C06EE57F
:102C90007FE084EE9CE00C94CA7869EF7DE084EEDE
:102CA0009CE00E94CA78F0E0E0E019946DE878E0DA
:102CB000811102C068E878E085E99DE00C94CA784B
:102CC000EF92FF920F931F93CF93DF93EC01A881B4
:102CD000B981109761F18C91882349F1088119819C
:102CE000F8018081882351F08D3241F080538A3081
:102CF00028F00F5F1F4F19830883F0CFC8010E948F
:102D000075B57C016CE270E0C8010E9459C3009760
:102D100051F419821882C701DF91CF911F910F9151
:102D2000FF90EF900895019699838883F4CFF12C5A
:102D3000E12CF1CF4F925F926F927F92BF92CF9230
:102D4000DF92EF92FF920F931F93CF93DF9300D008
:102D500000D0CDB7DEB77C01B62E809197088823CE
:102D600009F4BBC0D70114969C9180912A0289175F
:102D700008F4B3C08091950890919608BAE06B135F
:102D8000EDC08B5B974FFC011082D70117960D9118
:102D90001C910115110509F49CC0F801618572852B
:102DA0006115710591F4458056806780708480912B
:102DB0005A0C90915B0CA0915C0CB0915D0C481684
:102DC00059066A067B0609F484C0D8011B964D910A
:102DD0005C911C974115510509F47BC0F7012481D2
:102DE00053968C91539790E0322F377002C095958F
:102DF00087953A95E2F780FF6CC0C22ED12CC601B0
:102E0000887F9370892B39F451968D919C91887F9E
:102E10009370C82AD92AD8018D919C91DC01ED913B
:102E2000FC916115710509F483C00688F789E02DCE
:102E30001995019709F04DC06CE3F80180819181EB
:102E40000E94D777B601D8018D919C910E94F78D91
:102E5000F80122818081918164E575E1222311F0DE
:102E600062E575E10E94CA78D8011D966D917C914A
:102E70001E978D919C910E94647860E2F801808198
:102E800091810E94D777D8011F966D917C915097C0
:102E90008D919C910E946478F801228180819181BA
:102EA00067E475E1222311F061E475E10E94CA78BC
:102EB00065E478E0D8018D919C910E946478F801D6
:102EC00080819181DC01ED91FC91008CF18DE02DF0
:102ED00019951092960810929508D70115968D9124
:102EE0009C911697009709F44DC014963C9120913F
:102EF0002B02231708F446C0DC01ED91FC910190F0
:102F0000F081E02D6B2D199526960FB6F894DEBF53
:102F10000FBECDBFDF91CF911F910F91FF90EF902A
:102F2000DF90CF90BF907F906F905F904F9008950B
:102F30000488F589E02D20E034E03A832983D80124
:102F400015964D905D906D907C9018974B825C82A9
:102F50006D827E82BE016F5F7F4F6ACF8F34910595
:102F60000CF0BBCFBDE06B1709F4B7CF9C012F5F0E
:102F70003F4F30939608209395088B5B974FFC0149
:102F80006083ABCF81E090E0BFCFCF93DF93EC01C4
:102F90008C859D856817790708F4CB019A8B898BFE
:102FA0006CE776E085E99DE00E94CA7869897A89B4
:102FB00085E99DE00E94F78D85E99DE00E94C1773B
:102FC00089899A89DF91CF9108950C9445B30C9427
:102FD00045B30C9445B30C9445B3CF93DF93DC0118
:102FE0001296ED91FC913097C1F1EC018E819F8199
:102FF00083309105B1F0049719F1608585E99DE072
:103000000E94118B6CE275E185E99DE00E94CA780F
:1030100085E99DE00E94C177EA81FB81808590E08F
:103020000CC064E275E185E99DE00E94CA7885E9FB
:103030009DE00E94C17782E090E0DF91CF910895FA
:1030400061E375E185E99DE00E94CA7885E99DE02C
:103050000E94C17781E090E0F0CF90E080E0EDCF7A
:103060000F931F93CF93DF938C01EB0102977CF0BA
:103070008A819B810E9475B580932B0202301105D5
:1030800031F08C819D810E9475B580932A0262EB9C
:103090007EE084EE9CE00E94CA7860912B0284EE70
:1030A0009CE00E94118B6DE97EE084EE9CE00E9422
:1030B000CA7860912A0284EE9CE00E94118B84EE13
:1030C0009CE0DF91CF911F910F910C94C177CF932A
:1030D000C1E068EE73E080E090E00E94A8946C2F5D
:1030E00084EE9CE00E94118BCF5FC43191F7CF91A9
:1030F0000895CF93DF93EC01FB012481358140815A
:103100005181628173810E94DE77CE01DF91CF9180
:103110000895EF92FF920F931F93CF93DF93EC01EB
:103120008B011D821C821A821B82E880F980E114C7
:10313000F10409F459C08091740790917507892BA7
:1031400009F452C0672B09F48701F80180858F705C
:103150008630A9F46EE074E0C8010E949C8A009752
:1031600019F0FC0181858A836FE277E0C8010E9433
:103170009C8A009709F43FC0FC0181858B8360E144
:1031800074E0C7010E949C8A009759F564E876E0D4
:1031900085E99DE00E94CA786B8185E99DE00E94E7
:1031A000118B62E876E085E99DE00E94CA786A8129
:1031B00085E99DE00E94118B85E99DE00E94C17721
:1031C00020E030E0A90160E174E0888199810E94EB
:1031D000198E60E174E0888199810E949C8A009731
:1031E00019F009969D838C83DF91CF911F910F91E8
:1031F000FF90EF900895F801808191810E9475B54C
:10320000BDCF0F931F93CF93DF93EC018B0163E14D
:1032100074E0C8010E94DE758823B1F0EA81FB8169
:103220000190F081E02D60817181E881F98102884F
:10323000F389E02D2EE234E04EE056E0CE01DF913E
:10324000CF911F910F91199465E374E0C8010E941A
:10325000DE75882389F0EA81FB810190F081E02D01
:1032600060817181E881F9810288F389E02D2EE285
:1032700034E041E056E0E2CF60E574E0C8010E942E
:10328000DE75882389F0EA81FB810190F081E02DD1
:1032900060817181E881F9810288F389E02D2EE255
:1032A00034E041ED56E0CACFDF91CF911F910F91ED
:1032B00008950F931F93CF93DF93EC018B016BE67F
:1032C00074E0C8010E94DE758823B9F01A8A198A51
:1032D00080E090E19D878C8784E690E09C8B8B8BCF
:1032E00081E08E8780E090E2988B8F8781E090E08C
:1032F000DF91CF911F910F91089568E774E0C801A5
:103300000E94DE75882361F01A8A198A1C8A1B8A3A
:1033100084E690E09D878C871E8680E090E3E4CF72
:1033200090E080E0E5CF64E874E085E99DE00E94EC
:10333000C57710927A071092790781E090E008959E
:10334000CF93DF93009709F484C0FC0120812223EE
:1033500009F47FC0EC0161E279E00E94D6B5892BC7
:1033600009F456C065E079E0CE010E94D6B5892BFC
:1033700009F451C06DEE76E0CE010E94D6B5892BDE
:1033800009F44CC069EE76E0CE010E94D6B5892BD7
:1033900009F447C065EE76E0CE010E94D6B5892BD0
:1033A00009F442C061EE76E0CE010E94D6B5892BC9
:1033B000F1F16DED76E0CE010E94D6B5892BD1F109
:1033C00069ED76E0CE010E94D6B5892BB1F164EDAE
:1033D00076E0CE010E94D6B5892B91F160ED76E0C2
:1033E000CE010E94D6B5892B71F165E279E0CE015C
:1033F0000E94D6B5892B51F16CEC76E0CE010E948B
:10340000D6B5892B31F58EE090E0DF91CF9108950C
:1034100082E090E0FACF81E090E0F7CF88E090E0A2
:10342000F4CF85E090E0F1CF86E090E0EECF87E04A
:1034300090E0EBCF89E090E0E8CF8AE090E0E5CF44
:103440008BE090E0E2CF8CE090E0DFCF8DE090E089
:10345000DCCF90E080E0D9CF0F931F93CF93DF9321
:103460008C01EB012197AE01BC0182E69AE00E943B
:10347000F96EF801329660E0CF01801B910B8C173A
:103480009D0718F48191680FF7CF82E69AE00E94B9
:10349000C56F82E69AE0DF91CF911F910F910C9456
:1034A0000C70CF92DF92EF92FF920F931F93CF9306
:1034B000DF93CDB7DEB762970FB6F894DEBF0FBECD
:1034C000CDBF6C010B871C872D873E874F87588B9C
:1034D000698B7A8B6CE773E1C7010E94D6B5EFE088
:1034E000F0E0892BF9F066E773E1C7010E94D6B5D9
:1034F000E1E1F0E0892BB1F060E773E1C7010E94E0
:10350000D6B5E0E1F0E0892B69F01D851F706CE60F
:1035100073E1C7010E94D6B5E12FF0E0892B11F4C9
:10352000EEE0F0E09B85992309F48CC1309709F413
:1035300057C03197E131F10508F040C08827EC55BC
:10354000F54E8F4F0C940BBFF01AB51ADE1ADE1A27
:10355000DE1ADE1AB11BEE1BDE1ADE1ADE1ADE1AC6
:10356000DE1ADE1AF51B0E1C011CCE010B960E9402
:103570007C117093B2076093B1079B012A50310907
:1035800025313105D8F420EF260F2093AF079B019A
:10359000770F440B550BD6011296ED91FC911397C2
:1035A0000190F081E02D60817181ED91FC910684A4
:1035B000F785E02D0FE814E0C601199510929D07DC
:1035C00081E0809395078DE4809396078FE5809343
:1035D000970765E270E08CE897E00E942C1A3BC0E8
:1035E000198291509E3008F073C0E92FF0E08827CF
:1035F000E350F54E8F4F0C940BBF0B1B3C1B681B0D
:10360000681B3C1B0B1B681B681B681B8A1B7F1BF2
:103610005B1BA01B951B80918A0781608093A90783
:103620006DE070E08CE192E00E942C1AD6011296B7
:10363000ED91FC9113970190F081E02D60817181F3
:10364000ED91FC910288F389E02D24E934E049E909
:1036500054E0C601199581E090E062960FB6F894A7
:10366000DEBF0FBECDBFDF91CF911F910F91FF90B5
:10367000EF90DF90CF90089580918A078E7F80939E
:10368000A9076DE070E08FE092E00E942C1AD6014D
:103690001296ED91FC9113970190F081E02D6081DD
:1036A0007181ED91FC910288F389E02D24E934E0E9
:1036B0004CE954E0CECF1092A30780918A07816035
:1036C0008093A90767E673E1CE0101960E94DFB5FA
:1036D000D6011296ED91FC9113970190F081E02DA7
:1036E00060817181ED91FC910288F389E02D24E9DC
:1036F00034E0AE014F5F5F4FC60119955FCF81E0A7
:103700008093A30780918A0781608093A90762E66E
:1037100073E1DACF82E08093A30780918A0781600A
:103720008093A9076DE573E1CFCF84E08093A30771
:1037300080918A0781608093A90769E573E1C4CF0E
:1037400083E08093A30760EA74E085E99DE00E942E
:10375000647880918A0781608093A90760E573E1AE
:10376000B3CF1982903179F148F49C3089F0CE01C1
:103770000B960E947C116093A50713C0913141F113
:103780009231A9F782E08093A50760E473E105C058
:1037900083E08093A50767E673E1CE0101960E945E
:1037A000DFB5D6011296ED91FC9113970190F0814F
:1037B000E02D60817181ED91FC910288F389E02D0B
:1037C00025EA34E096CF1092A5076BE473E1E5CFCC
:1037D00081E08093A50764E473E1DFCFCE010B960F
:1037E0000E947C116093A307E9CE913031F09230B2
:1037F00009F0E4CE1092A807E1CE80E58093A807F7
:10380000DDCE913049F09230A9F3CE010B960E94A3
:103810007C116093A707D2CE83E0F0CF913039F0CE
:10382000923009F0CBCE8091A907877F03C08091A9
:10383000A90788608093A907C1CE8FEF9FEF0DCFB6
:10384000198246CFE231F10508F0B8CE8827E45D51
:10385000F34E8F4F0C940BBF1D1C201CB51ADE1AA3
:10386000DE1ADE1ADE1AB11BEE1BDE1ADE1ADE1AB3
:10387000DE1ADE1ADE1ADE1ADE1A051CCF93DF937B
:1038800000D000D01F921F92CDB7DEB7EFECFCE066
:10389000128A118A80E090E19587848784E690E01F
:1038A000948B838B81E0868780E090E2908B878782
:1038B0001C821B8280E093E09A838983FE83ED83E0
:1038C0008FEF9FEF98878F836FEA72E184EE9CE021
:1038D0000E94CA786091740770917507CE010196B5
:1038E0000E94C07E8FEC9CE00E94AD128FEC9CE0A9
:1038F0000E9474126FE972E184EE9CE00E94CA7823
:1039000084EE9CE00E94C17728960FB6F894DEBF43
:103910000FBECDBFDF91CF910895FC0186819781C5
:10392000009799F0FC0120852F70223029F46185E1
:103930007285838594850895253039F460E00E946E
:10394000188B009711F0FC01F2CF60E070E0CB0122
:1039500008950F931F93CF93DF93FC01C281D3810E
:103960002097F9F088858F70823049F4672BC9F46D
:1039700089859A85DF91CF911F910F9108958530A8
:1039800081F48B01CE010E942D8B8017110649F026
:1039900044F0602FCE010E94188BFC018185928536
:1039A000E9CF90E080E0E6CFFC016115710519F4E4
:1039B00084819581089586819781681779072CF015
:1039C00084819581860F971F0895828193810C943D
:1039D000A91CCF93DF93EC0167E175E185E99DE0D8
:1039E0000E94CA7885E99DE00E94C177E881F9814B
:1039F000028CF38DE02DCE0119958130910529F0CF
:103A0000029759F060E08C811AC063E070E0CE014B
:103A10000E94D41C60E00E94509360E08C810E9460
:103A2000509361E070E0CE010E94D41C60E00E94DF
:103A3000509362E070E0CE010E94D41C60E00E94CE
:103A40005093109244081092430881E090E0DF9177
:103A5000CF9108950F931F93CF93DF93EB0163E012
:103A6000FC01808191810E94188B009799F0C0958C
:103A7000D095CF6FAE0170E060E0FC01018512854A
:103A80002385348540235123622373234187528742
:103A900063877487DF91CF911F910F9108950F93E2
:103AA0001F93CF93DF93EB0163E0FC018081918151
:103AB0000E94188B009789F0CC27AE0170E060E07F
:103AC000FC010185128523853485402B512B622B07
:103AD000732B4187528763877487DF91CF911F9142
:103AE0000F910895CF93DF93EB0163E0FC01808198
:103AF00091810E94188B009741F0FC01818592858D
:103B00008C239D23DF91CF91089590E080E0FACF40
:103B1000CF93C62F63E0FC01808191810E94188BB6
:103B20000097E9F0FC01418552856385748544273F
:103B3000662777274C2B418752876387748762EF0C
:103B400076E085E99DE00E94CA786C2F85E99DE0CA
:103B50000E94118B85E99DE0CF910C94C177CF91A4
:103B60000895FC0182819381009719F062E00E9420
:103B7000881D81E090E00895CF93DF93EC010E94CF
:103B8000B11D6AE075E185E99DE00E94CA7885E98A
:103B90009DE00E94C1778A819B81892B09F44DC0E9
:103BA0008C819D81892B09F048C0E881F981028CC4
:103BB000F38DE02DCE0119958130910529F0029702
:103BC00059F061E08C811AC063E070E0CE010E9480
:103BD000D41C61E00E94509361E08C810E9450935C
:103BE00061E070E0CE010E94D41C61E00E9450931D
:103BF00062E070E0CE010E94D41C61E00E9450930C
:103C00008091A100887F8093A10080919100887F9E
:103C1000809391008091A10082608093A1008091A7
:103C2000910082608093910081E090E0909344083D
:103C300080934308DF91CF91089590E080E0FACF20
:103C4000CF93DF93EC010E94B11DEC81FD81309791
:103C500009F44FC0C681D7812097C1F1E881F9816D
:103C6000309781F18081882369F160E974E0CE01A9
:103C70000E949C8A892B41F42FEF3FEFA90160E954
:103C800074E0CE010E94198E65E974E0CE010E94B5
:103C90009C8A892B41F42FEF3FEFA90165E974E07D
:103CA000CE010E94198E6AEA74E0CE010E949C8ABD
:103CB000892B41F42FEF3FEFA9016AEA74E0CE01AE
:103CC0000E94198E0A80DB81C02DC6CF6FEA74E195
:103CD00085E99DE00E94CA7885E99DE00E94C17750
:103CE00081E090E09093420880934108DF91CF916A
:103CF000089567E974E185E99DE00E94CA7885E945
:103D00009DE00E94C17790E080E0F0CF0E94B11D5D
:103D10006EEA74E085E99DE00E94C57726E040E800
:103D200055E260E070E082E69AE00E94817D81E0E9
:103D300090E090937A0780937907089563E0FC01FF
:103D4000808191810E94188B009719F0FC01818578
:103D500008958FEF08950F931F93CF93DF93C92F8B
:103D6000D62F082F192F17FF03C0119501951109A0
:103D700061E0802F0E9450936C2FDD23A9F06095A5
:103D8000661F6627661F802F0E94229360E372E100
:103D900085E99DE00E94CA7885E99DE0DF91CF9199
:103DA0001F910F910C94C177661F6627661F802FA5
:103DB0000E9422936BE272E1EBCF029784F06CE8F1
:103DC0007EE084EE9CE00E94CA7870E060E084EEC1
:103DD0009CE00E94258B84EE9CE00C94C1770C94AF
:103DE0003E1C892B59F0FB01828193810E94558CE6
:103DF00064E07FE084EE9CE00C94CA7890E080E080
:103E0000F5CF892B59F0FB01828193810E94078CA9
:103E10006DEE7EE084EE9CE00C94CA7890E080E049
:103E2000F5CF8091C70C9091C80C892B51F00E945E
:103E30004C8B882331F06DED7EE084EE9CE00C9499
:103E4000CA780895EF92FF920F931F93CF93DF9359
:103E5000CDB7DEB72C970FB6F894DEBF0FBECDBF3F
:103E60008C017B0180E094E09A8389831B821C8211
:103E70001D821E8298878F8319861A861B861C8650
:103E800005301105ECF0BE01695F7F4FF7018085B9
:103E900091850E94140F892B99F0CE0107960E94FC
:103EA000F88CBE01695F7F4FF701868197810E9480
:103EB000140F892B61F0CE0107960E94A28D0EC0CF
:103EC000CE0101960E94F88C0430110554F7CE0102
:103ED00001960E94A28D033011057CF1BE01695F3D
:103EE0007F4FF701848195810E94140F892B29F15E
:103EF000CE0107960E944D8DBE01695F7F4FF7018D
:103F0000828193810E94140F892BF1F0CE010796D4
:103F10000E94A38C66EC7EE084EE9CE00E94CA784E
:103F20002C960FB6F894DEBF0FBECDBFDF91CF91B8
:103F30001F910F91FF90EF900895CE0101960E947E
:103F40004D8D02301105C4F6CE0101960E94A38C5E
:103F500001301105F9F6CE0101960E94A38C6DEC9B
:103F60007EE084EE9CE00E94CA78D4CF2F923F92EC
:103F70004F925F926F927F928F929F92AF92BF9279
:103F8000CF92DF92EF92FF920F93CF93DF9300D007
:103F90001F92CDB7DEB77C017A8369835C834B8344
:103FA000DB011C92FC016081662309F4C2C130FF71
:103FB000C0C1F9E06F9FB00111246251764FCD016D
:103FC0000E940DB64B815C816AE676E089819A8118
:103FD0000E9474C3E981FA8101900020E9F73197CA
:103FE00089819A81E81BF90B1C012E0E3F1EAB81C3
:103FF000BC81AE1BBF0B1197BC83AB83D70112965C
:10400000EC91E295EF70E150EC3008F0B3C0F0E0D5
:104010008827E25FFF4D8F4F0C940BBF1A20892039
:10402000EF205621722156200621062106214A2022
:104030003E208F21F7018481282F30E050E040E0BE
:10404000002359F030E0A4E6B0E00E94D4BE2FEF88
:1040500030E040E050E00E94A2BE5F934F933F9358
:104060002F9386EB94E09F938F93FC81FF938B813A
:104070008F933F922F920E94ACC377C0F701878144
:104080008F9386818F9385818F9384818F9389EB22
:1040900094E0E9CFF70187818F9386818F938581A3
:1040A0008F9384818F938DEB94E0DDCFF701C480F3
:1040B000D580E680F780C701B6012AE030E040E015
:1040C00050E00E94A2BE97FF07C090958095709522
:1040D00061957F4F8F4F9F4F9F938F937F936F93E8
:1040E000C701B6012AE030E040E050E00E94A2BEE5
:1040F0005F934F933F932F9381EC94E09F938F9323
:10410000FC81FF938B818F933F922F920E94ACC3CF
:104110002CC0C7010E94C111BC01F701C680D78025
:10412000D0FADD24D0F89481F580EB80BC80292F73
:1041300030E050E040E077FD35C0011135C07F939D
:104140006F931F921F921F929F931F92FF92DF9275
:10415000CF9288EC94E09F938F939C819F93AB8147
:10416000AF933F922F920E94ACC30FB6F894DEBF7C
:104170000FBECDBF89819A810F900F900F900F9045
:10418000DF91CF910F91FF90EF90DF90CF90BF9094
:10419000AF909F908F907F906F905F904F903F90E7
:1041A0002F900895002361F0292F30E0A4E6B0E0BD
:1041B0000E94D4BE2FEF30E040E050E00E94A2BE4B
:1041C0005F934F933F932F931F92FF92DF92CF9273
:1041D0008BEC94E09F938F93BF92EF9295CFD70192
:1041E00015968C9115971F928F9316969C91169702
:1041F00017968C9181708F939F938EEC94E09F9390
:104200008F93BC81BF93EB81EF9333CFD70114968B
:104210008D909D90AD90BC90179720E030E0A90163
:10422000C501B4010E9436BD2401350187FF04C0D9
:1042300077FA709477F87094C301B2010E9408C0B5
:104240006B01072E000C880B990B0E943DBD9B0152
:10425000AC01C301B2010E9429BF20E030E048EC6C
:1042600052E40E949CBD0E9493C00E9408C0062F89
:10427000772E20E030E0A901C501B4010E9436BDCF
:1042800087FF07C07F920F93DF92CF9284ED94E077
:10429000B6CF7F920F93DF92CF9285ED94E09F93FC
:1042A0008F939C819F93AB81AF93E3CED7011496FC
:1042B0008C9114971F928F9315968C9115971F923E
:1042C0008F9316968C911F928F938BEC94E09F9313
:1042D0008F93BC81BF93EB81EF933F922F920E940B
:1042E000ACC343CFD70117968C9117971F928F932A
:1042F00014968C9114971F928F9315968C91159705
:104300001F928F9316968C911F928F9388EC94E056
:104310009F938F93BC81BF93EB81EF93F5CED70131
:1043200014966D917C914B815C81C1010E9492C376
:1043300021CF29803A8062CECF92DF92EF92FF9216
:104340000F931F93CF93DF93EC01888199810E9493
:104350002D8B082F10E0043011059CF40E94C180C1
:10436000009739F0DC0118962C911897207F189649
:104370002C93BC01888199810E94FD8D0F5F1F4F96
:10438000EACFC880D98060E0C6010E94188BFC018A
:10439000F184F88661E0C6010E94188B8C019B8332
:1043A0008A8362E0C6010E94188B9D838C8364E03F
:1043B000C6010E94188B6C019F838E83FAE0FF1662
:1043C00009F46EC0FF1560F083E0F81659F1DF9133
:1043D000CF911F910F91FF90EF90DF90CF900895B4
:1043E000A0E1FA1609F46CC0B2E1FB12F0CF86E04E
:1043F00090E00E94A9B2FC01D383C28386EA92E0D6
:1044000091838083158214820115110541F0D80132
:1044100018968C918F70863011F415830483FA8777
:10442000E987D5CF8AE090E00E94A9B27C01FC0127
:10443000D383C2838EE592E09183808370E060E055
:10444000CE010E94A91C97FD1EC0D70115969C9312
:104450008E9314970115110501F1D80118968C91CE
:104460008F708230B9F08530C1F4C8010E942D8B65
:1044700090E0F7019783868382E892E091838083BE
:10448000FA86E986A4CF919581959109F7019583E4
:104490008483E0CF81E090E0ECCF90E080E0E9CF52
:1044A00084E090E00E94A9B2DC011396DC93CE93E5
:1044B000129728EC32E02D933C939A87898787CF17
:1044C00086E090E00E94A9B2FC01D383C2838CE312
:1044D00092E091838083C114D10469F0D6011896CB
:1044E0008C9118978F70823031F416968D919C9133
:1044F0009583848394CF90E080E0FACFCF93DF93CD
:10450000EC01798368831A8619861B861E8A1D8AA8
:104510000E943612882329F0CE01DF91CF910C94AE
:104520009C21DF91CF910895EF92FF920F931F93FB
:10453000CF93DF93EC017B018E819F81892BD9F48E
:10454000888199810E942D8B082F10E0053011057C
:1045500094F40E94C180009721F0FC012085207F07
:1045600020879F838E83BC01888199810E94FD8D65
:104570000F5F1F4FEBCFEE81FF813097D9F0808521
:10458000982F9F70A9F4807F82608087EE81FF81E1
:104590001186128613861486EE81FF81F782E682E9
:1045A000C701DF91CF911F910F91FF90EF90089578
:1045B000923061F3F12CE12CF3CFCF93DF93EC0138
:1045C0006DED74E085E99DE00E94C5778C819D8149
:1045D0000E9445B370E060E08A819B810E94942232
:1045E0001D821C8281E090E0DF91CF910895CF92EF
:1045F000DF92EF92FF920F931F93CF93DF93EC0123
:104600000E94B11D8C819D81892B61F40A811B81DF
:1046100085E090E00E94A9B2BC01C8010E949422EA
:104620009D838C83EC80FD80E114F104A9F469E39F
:1046300074E18EEE9CE00E94CA788EEE9CE00E94AF
:10464000C17790E080E0DF91CF911F910F91FF90B3
:10465000EF90DF90CF90089510923C0810923B08A5
:10466000109236081092350810923D0810923E08BC
:1046700010923F08109240081092370810923808A4
:104680001092390810923A081092B3071092F50769
:10469000EA81FB81309759F082819381009739F04C
:1046A000DC0118962C912F70263009F468C062EF57
:1046B00073E18EEE9CE00E94CA7861E070E08C812C
:1046C0009D81892B11F470E060E08EEE9CE00E94E9
:1046D000258B60EF73E18EEE9CE00E94CA7861E06A
:1046E00070E08A819B81892B11F470E060E08EEE8E
:1046F0009CE00E94258B6EEE73E18EEE9CE00E94A2
:10470000CA78EA81FB8161E070E082819381892B24
:1047100011F470E060E08EEE9CE00E94258B6CEE60
:1047200073E18EEE9CE00E94CA78EA81FB810280F0
:10473000F381E02D80858F7061E070E0863011F4A8
:1047400070E060E08EEE9CE00E94258B6AEE73E1E3
:104750008EEE9CE00E94CA788EEE9CE00E94C177AB
:104760006BE074E18EEE9CE00E94CA788EEE9CE0D5
:104770000E94C177EC81FD8182E0808362CF6EEE82
:1047800074E00E949C8A009709F4A8C0FC0120856F
:104790002F70243009F0A2C0C184D284B60185E90B
:1047A0009DE00E94647866EE73E185E99DE00E94D9
:1047B000CA7810E000E0C114D10409F486C0B80141
:1047C00062567C4EC6010E94D6B5892B09F077C08F
:1047D000F801EE55FC4E25913491922F832FD7018D
:1047E00013969C93139714968C93EA81FB8165EF43
:1047F00074E0828193810E949C8AEC81FD81009704
:1048000009F472C0DC0118962C9118972F70223091
:1048100009F06AC019964D915D916D917C911C973C
:10482000411551056105710509F45EC0528341834C
:1048300041815281052E000C660B770B23818CE998
:104840009BE00E94817DEC81FD8141815281052E9A
:10485000000C660B770B23818FEF9AE00E94817D1D
:10486000EA81FB8162E675E0828193810E949C8AE5
:10487000009739F0FC01818592859093F40780932D
:10488000F30761E274E184EE9CE00E94CA78EA8159
:10489000FB810190F081E02D6081718184EE9CE0CC
:1048A0000E94647884EE9CE00E94C177EC81FD81D7
:1048B00081E080838093290281E090E0C4CE0A5F8A
:1048C0001F4F0834110509F076CF61E873E185E9DF
:1048D0009DE00E94CA7896E080E081CF86E090E07B
:1048E000F7019483838381CF80E09BE4928381836B
:1048F0009FCFCF92DF92EF92FF920F931F93CF93B0
:10490000DF93EC016A017B018E819F81892BD9F4B1
:10491000888199810E942D8B082F10E005301105A8
:1049200094F40E94C180009721F0FC012085207F33
:1049300020879F838E83BC01888199810E94FD8D91
:104940000F5F1F4FEBCFEE81FF81309749F18085DC
:10495000982F9F7019F5807F82608087EE81FF819C
:10496000C186D286E386F4866AEF76E085E99DE02B
:104970000E94CA782AE030E0B701A60185E99DE0EF
:104980000E94DE7785E99DE0DF91CF911F910F9125
:10499000FF90EF90DF90CF900C94C1779230F1F2BE
:1049A000DF91CF911F910F91FF90EF90DF90CF900B
:1049B00008950F931F93CF93DF938C01FC01C08167
:1049C000D1816FE270E0CE010E94A1C30097D9F0BF
:1049D000FC011192CF010E94A019EC0166E077E082
:1049E00085E99DE00E94CA78BE0185E99DE00E94AC
:1049F000258B85E99DE00E94C177CE01DF91CF91A3
:104A00001F910F910895CE010E94A019EC01892BEE
:104A1000A1F3F80111821082F0CF8F929F92AF9292
:104A2000BF92CF92DF92EF92FF920F931F93CF939B
:104A3000DF93CDB7DEB767970FB6F894DEBF0FBE32
:104A4000CDBF8C017B014C018BE0880E911C9F8AAD
:104A50008E8AF801128611861386168A158A672BAC
:104A600009F463C0A0901009B0901109A114B10419
:104A700009F45BC06FE270E0C7010E9459C36C018A
:104A8000892B09F44AC0F701DE01119690E080E01D
:104A9000BD012191222341F02F3231F08431910563
:104AA00019F02D930196F5CF860F971FFC01108208
:104AB000C5010E949C8AF80191838083B6016F5FD3
:104AC0007F4F4AE050E0C4010E9492C3CE01469657
:104AD0000E94D924F801968B858B8E899F89892B1A
:104AE00009F41386C8010E943612882319F0C80100
:104AF0000E949C2167960FB6F894DEBF0FBECDBF13
:104B0000DF91CF911F910F91FF90EF90DF90CF90A9
:104B1000BF90AF909F908F900895B701C5010E94FC
:104B20009C8AF80191838083DDCFF8011182108285
:104B3000D9CF1F93CF93DF93FC01162FC389D4895C
:104B4000818992899C012F5F3F4F328B218BC80F47
:104B5000D91FCE010E945ABE181721F0612FCE0135
:104B60000E9462BE81E090E0DF91CF911F91089595
:104B7000FC0181899289248535858217930740F449
:104B800023893489820F931F0E945ABE90E00895B2
:104B90008FEF9FEF08952F923F924F925F926F9207
:104BA0007F928F929F92AF92BF92CF92DF92EF92BD
:104BB000FF920F931F93CF93DF93CDB7DEB762972A
:104BC0000FB6F894DEBF0FBECDBF5C014B012901CB
:104BD0003A01CA01B9010E9408C01B013F926F93BC
:104BE00081ED94E09F938F93CE0101967C019F937A
:104BF0008F930E94E9C30F900F900F900F900F902A
:104C00000F9020E030E0A901C301B2010E943EC034
:104C1000181624F077FA709477F87094F7010190E1
:104C20000020E9F731976F01CE18DF088EE280830C
:104C3000A2E0B0E0AC0FBD1FAC0DBD1DBA8BA98BBF
:104C4000B10137FE03C0719561957109072E000C03
:104C5000880B990B0E943DBD9B01AC01C301B201C1
:104C60000E9429BF20E030E040E251E40E949CBD58
:104C70000E9408C0605DE989FA896083FE01EC0D3D
:104C8000FD1D1382D501ED91FC910288F389E02D81
:104C90009801A701B401C501199562960FB6F89461
:104CA000DEBF0FBECDBFDF91CF911F910F91FF905F
:104CB000EF90DF90CF90BF90AF909F908F907F90BC
:104CC0006F905F904F903F902F900895DA01E091A0
:104CD0000609F0E0FE2FEE27E60FF71F90E0982F71
:104CE0008827A901BD018E0F9F1F0C944582CF9389
:104CF000DF931F92CDB7DEB72091060930E0322F47
:104D00002227260F371F90E0982F8827498341E0FC
:104D100050E0BE016F5F7F4F820F931F0E9445825C
:104D20000F90DF91CF910895CF93DF931F92CDB76E
:104D3000DEB741E050E0BE016F5F7F4F0E94BA8155
:104D400089810F90DF91CF9108952091060930E07D
:104D5000322F2227620F731F90E0982F8827860F2B
:104D6000971F0C94942663E070E00C94A5269F9204
:104D7000AF92BF92CF92DF92EF92FF920F931F9369
:104D8000CF93DF93EC017B0180914F0A811121C009
:104D90001B821A8288EE93E0A0E0B0E08C839D83B2
:104DA000AE83BF838CE893E09983888388E08C8707
:104DB00088EE93E09E878D87CE01DF91CF911F9182
:104DC0000F91FF90EF90DF90CF90BF90AF909F90AA
:104DD000089534E0932E833311F028E0922E8FE370
:104DE000C82E8AE0D82E10E098E0B92EA12CD6016A
:104DF0002D913D916D01F701848195812817390727
:104E000091F4812F0E948E86082F873111F08C310A
:104E100039F5812F0E947A85892B59F50C3119F4C7
:104E2000812F0E9472861F5F9112E1CFA11008C0EE
:104E3000D701ED91FC910084F185E02DC701199512
:104E40001B821A8288EE93E0A0E0B0E08C839D8301
:104E5000AE83BF838CE893E099838883BC86A8CF18
:104E6000843149F08111DFCFF6013297118210822F
:104E7000DACFB12ED8CFAA24A394D5CF8F929F9208
:104E8000AF92BF92CF92DF92EF92FF920F931F9358
:104E9000CF93DF93CDB7DEB72F970FB6F894DEBF71
:104EA0000FBECDBF5C014B017A0180914F0A882370
:104EB000C9F104E0833309F008E0B501CE010196A1
:104EC0000E94B7268FE3C82E8AE0D82E10E0F601A4
:104ED000219131916F01F50184819581281739075E
:104EE00051F4812F0E948E86873129F4A701B401E5
:104EF000812F0E94F0841F5F0113E9CFC7012F9615
:104F00000FB6F894DEBF0FBECDBFDF91CF911F91DA
:104F10000F91FF90EF90DF90CF90BF90AF909F9058
:104F20008F900895F12CE12CE9CFDA01E091060988
:104F3000F0E0FE2FEE27E60FF71F90E0982F88276E
:104F4000A901BD018E0F9F1F0C94BA8144E050E06F
:104F5000BC018FE090E00C94458244E050E0BC013D
:104F600085E090E00C94458244E050E0BC0181E093
:104F700090E00C94458208959F92AF92BF92CF9299
:104F8000DF92EF92FF920F931F93CF93DF938C01E9
:104F90005B01942EE52EFC01C688D788F08C80E555
:104FA00091E00E9401908F2D0E949684C92DDE2DE4
:104FB0008C179D0708F4EC019E01A501B6018F2D09
:104FC0000E941384F801868997898C0F9D1F978B07
:104FD000868BCE01DF91CF911F910F91FF90EF90C3
:104FE000DF90CF90BF90AF909F900895CF93FC013A
:104FF000C08D80E591E00E94019060E270E08C2F0E
:105000000E94AA8162E070E08C2F0E94A52684FD98
:1050100016C062E070E08C2F0E94A52683FF0AC0B4
:1050200048E162E070E08C2F0E94772680E090E0FB
:10503000CF91089580E591E00E940190E3CF40E197
:1050400062E070E08C2F0E94772681E0F0CFFF9223
:105050000F931F93CF93DF93EB01FC01178A168AFE
:105060002A81211109C02B81211106C02C81211117
:1050700003C02D81222301F141155105E9F08A0178
:10508000FC01F08C80E591E00E940190AE014E5F42
:105090005F4F24E030E06CE070E08F2D0E946626C8
:1050A000B8018F2D0E949D8681E090E0DF91CF9125
:1050B0001F910F91FF90089580E0F7CF0F931F93FA
:1050C000CF938C01FC016481758181E20E94C986C5
:1050D000C82F8830F8F480E591E00E9401908C2F71
:1050E0000E94B326833131F08C2FCF911F910F9105
:1050F0000C94728662E070E08C2F0E94AA81F80105
:1051000084819581EC2FF0E0EE0FFF1FE15CF54FFD
:1051100091838083CF911F910F9108950F931F93D7
:10512000CF93DF931F921F92CDB7DEB7FC0124858A
:105130002830E0F48C0180E591E00E94019022E0AB
:1051400030E0AE014F5F5F4F60E170E0F8018485B1
:105150000E94952789819A819827892798270F90FF
:105160000F90DF91CF911F910F91089590E080E013
:10517000F6CF0F931F93CF93DF931F921F92CDB75C
:10518000DEB7FC0124852830E0F48C0180E591E055
:105190000E94019022E030E0AE014F5F5F4F64E07B
:1051A00070E0F80184850E94952789819A8198276B
:1051B000892798270F900F90DF91CF911F910F9122
:1051C000089590E080E0F6CFCF93DF93EC0180E08C
:1051D00094E0998388831A821B821C821D8280E559
:1051E00091E00E940190BE016E5F7F4F44E050E06D
:1051F0008FE090E00E94BA81CE01DF91CF910895B7
:105200000E940683882331F080914F0A843329F06D
:10521000873381F090E080E0089580E591E00E947E
:10522000019085E390E00E94942685FD0DC082E008
:1052300090E0089580E591E00E9401908EE290E078
:105240000E94942680FFF3CF81E090E008951F92A2
:105250000F920FB60F9211240BB60F922F933F931C
:105260004F935F936F937F938F939F93AF93BF936E
:10527000EF93FF938091B900887F803609F44DC089
:1052800008F040C0883209F4A7C028F5803109F43D
:105290009BC0C8F4882309F4F7C0883009F494C08F
:1052A000FF91EF91BF91AF919F918F917F916F91FE
:1052B0005F914F913F912F910F900BBE0F900FBEBA
:1052C0000F901F901895883109F486C0803241F7FD
:1052D0008093DF0814C0803409F49BC040F480330D
:1052E000B9F38833E9F68093DF0885ECAEC08035EA
:1052F00009F483C0883509F494C0883489F60E9483
:10530000630ECECF883909F48AC038F5883729F082
:1053100050F4883611F0803719F683E08093E00866
:105320001092DE0855C0883809F479C0803919F028
:10533000803809F0B5CF8091DE08803208F06FC068
:10534000E091DE0881E08E0F8093DE088091BB0043
:10535000F0E0E254F74F80833BC0803B39F0D0F45B
:10536000803A09F477C0883A09F09ACF84E08093B4
:10537000E0081092BD081092BC08F0E0E0E019953A
:105380008091BC0881110FC081E08093BC0810920D
:105390009C0809C0803C09F4A8CF883C09F4A5CF3B
:1053A000883B09F07DCFE091BD0881E08E0F8093AE
:1053B000BD08F0E0E456F74F80818093BB009091E8
:1053C000BD088091BC0829C0809105098093BB006D
:1053D00085EC8093BC0064CF90910409809103090F
:1053E000981758F5E091040981E08E0F8093040925
:1053F000F0E0ED51F74F8081E9CFE091040981E0C1
:105400008E0F809304098091BB00F0E0ED51F74FBF
:10541000808390910409809103099817C8F285E868
:10542000D8CFE091040981E08E0F80930409809128
:10543000BB00F0E0ED51F74F80838091E2088111CD
:105440005ECF81E08093E10884EA8093BC001092F3
:10545000E00826CF85EC8093BC001092E008809194
:10546000DE08803230F4E091DE08F0E0E254F74FDD
:1054700010826091DE0870E08EEB98E0F0E0E0E0F2
:1054800019951092DE080CCF1092DF0838CF4F929A
:105490005F926F927F92AF92BF92CF92DF92EF9224
:1054A000FF920F931F93CF93DF9300D01F92CDB73E
:1054B000DEB72B013C0129833A834B835C83A60131
:1054C00095016E0D7F1D801F911F0E9480BE298156
:1054D0003A814B815C81621773078407950708F551
:1054E0002415350546055705A8F421E0822F0F90B5
:1054F0000F900F900F90DF91CF911F910F91FF9020
:10550000EF90DF90CF90BF90AF907F906F905F90C3
:105510004F90089521E0461657066806790630F345
:105520000FC0461657066806790650F421E08981B7
:105530009A81AB81BC8184159505A605B705B0F2AB
:1055400020E0D4CF8F929F92AF92BF92CF92DF9202
:10555000EF92FF920F931F93CF93DF9300D000D071
:1055600000D01F92CDB7DEB76130710509F07DC262
:105570004C010E94B0959B01AC016091860770912F
:1055800087078091880790918907AA24AA94BA2C4A
:10559000650118E8E12E13E1F12E00E010E00E9411
:1055A000472A8823B9F080E00E94FE1560938607A1
:1055B0007093870780938807909389076AEF74E058
:1055C00085E99DE00E94C5776DE070E082E092E0A1
:1055D0000E942C1A64E670E080E090E00E94A8949B
:1055E00082E69AE00E94706F18161906ACF088EEF9
:1055F00093E02A960FB6F894DEBF0FBECDBFDF91C1
:10560000CF911F910F91FF90EF90DF90CF90BF90BF
:10561000AF909F908F90089545E250E06CE877E05E
:1056200082E69AE00E94437782E69AE00E94706FD9
:10563000892B59F062E070E080E090E00E94A8942D
:1056400082E69AE00E944E6FEFCF8091B007909172
:105650008507891761F2809385078091AF0790E0F5
:1056600040969093B2078093B1078091990790E09C
:1056700090938407809383078091A30790E0909391
:105680008207809381078091A50790E0909380071F
:1056900080937F078091A70790E090937E07809387
:1056A0007D078091A90790E090938B0780938A07EC
:1056B0008091A80790E090937C0780937B07D401AA
:1056C000ED91FC9111970288F389E02D12968D914E
:1056D0009C91DC018D919C91DC016D917C9180917C
:1056E000AB0722E035E049E954E080FD02C04CE917
:1056F00054E0C401199580917B0790917C07803814
:105700009105A9F4D4011296ED91FC9113970190A3
:10571000F081E02D60817181ED91FC910288F38927
:10572000E02D29E035E049E954E0C4011995809164
:105730007B0790917C07892BA9F4D4011296ED91F7
:10574000FC9113970190F081E02D60817181ED91C2
:10575000FC910288F389E02D29E035E04CE954E022
:10576000C40119956FE075E085E99DE00E946478B9
:1057700060918A0770918B0785E99DE00E94258BD7
:1057800085E99DE00E94C17780918A07F40120811C
:105790003181A281B3810D90BC91A02D6D917C913E
:1057A000D9015296ED91FC9126E135E049E954E0AA
:1057B00083FD02C04CE954E0C4011995D401ED9178
:1057C000FC9111970288F389E02D12968D919C919E
:1057D000DC018D919C91DC016D917C9180918A0717
:1057E0002DE135E049E954E081FD02C04CE954E087
:1057F000C401199520917D0730917E07032E000C7E
:10580000440B550BD4011296ED91FC911397019026
:10581000F081E02D60817181ED91FC910684F78526
:10582000E02D09E215E0C401199580917F07909160
:105830008007892BA9F4D4011296ED91FC9113975E
:105840000190F081E02D60817181ED91FC910288E1
:10585000F389E02D25EA34E040E355E0C4011995D1
:1058600080917F07909180070197A9F4D401129647
:10587000ED91FC9113970190F081E02D6081718191
:10588000ED91FC910288F389E02D25EA34E045E3AF
:1058900055E0C401199580917F0790918007029788
:1058A000A9F4D4011296ED91FC9113970190F08127
:1058B000E02D60817181ED91FC910288F389E02DEA
:1058C00025EA34E04CE355E0C401199580917F0747
:1058D000909180070397A9F4D4011296ED91FC9161
:1058E00013970190F081E02D60817181ED91FC9121
:1058F0000288F389E02D25EA34E040E455E0C40154
:105900001995D401ED91FC9111970288F389E02D4E
:1059100012968D919C91DC018D919C91DC016D9191
:105920007C9180917D0790917E0729E235E04CE9DA
:1059300054E0892B11F049E954E0C40119952091F4
:10594000B1073091B207032E000C440B550BD40164
:105950001296ED91FC9113970190F081E02D6081FA
:105960007181ED91FC910684F785E02D0FE814E03C
:10597000C401199520918307309184072F3F310589
:10598000B9F0032E000C440B550BD4011296ED9187
:10599000FC9113970190F081E02D60817181ED9170
:1059A000FC910684F785E02D05E415E0C401199506
:1059B0001982809181079091820767E673E10097D1
:1059C000C9F062E673E181309105A1F06DE573E104
:1059D0008230910579F060E573E18330910551F0F3
:1059E00069E573E18430910529F08D36910531F434
:1059F0006CE373E1CE0101960E94DFB5209181072F
:105A000030918207032E000C440B550BD4011296E3
:105A1000ED91FC9113970190F081E02D60817181EF
:105A2000ED91FC910684F785E02D0BE415E0C401AF
:105A3000199580918A07F40120813181A281B38177
:105A40000D90BC91A02D6D917C91D9015296ED9154
:105A5000FC9124E934E0AE014F5F5F4F80FD02C04E
:105A60004CE954E0C4011995C2CD90E080E0C1CD6D
:105A70008F929F92AF92BF92CF92DF92EF92FF925E
:105A80000F931F93CF93DF937C014A015901C0917B
:105A90009808D0919908062F660F110B209709F4EA
:105AA0005CC088858F70863009F055C061E575E06F
:105AB000CE010E949C8A6C0182E08816910449F014
:105AC0006AEA74E0E3E08E16910429F0D0E0C0E0C9
:105AD00006C066E575E0CE010E949C8AEC01C11407
:105AE000D104D9F1F60180858F708430B1F56185DC
:105AF0007285A801C7010E9492C3A8016BE575E0F9
:105B0000C7010E9474C3209779F188858F70843013
:105B100059F569857A85A801C7010E9474C3A80157
:105B20006BE575E0C7010E9474C3A114B10429F0AC
:105B3000A801B501C7010E9474C3C701DF91CF91CD
:105B40001F910F91FF90EF90DF90CF90BF90AF909B
:105B50009F908F900895D0E0C0E0A80167E675E1BE
:105B6000C7010E940DB6C9CFF2E08F16910481F0F3
:105B700083E08816910429F0609107097091080963
:105B8000CACFA80161E675E1C7010E94EFB5C7CF92
:105B9000A8016EE575E1F8CFCF92DF92EF92FF9208
:105BA0000F931F93CF93DF93CDB7DEB7C154D109C5
:105BB0000FB6F894DEBF0FBECDBF6C01AB0130E075
:105BC00020E060E4CE0101967C010E94382DF701AF
:105BD00001900020E9F731978F010E191F09A801E4
:105BE000B701C6010E9484C3892B11F010E000E0C8
:105BF000C801CF5BDF4F0FB6F894DEBF0FBECDBF3D
:105C0000DF91CF911F910F91FF90EF90DF90CF9098
:105C10000895CF92DF92EF92FF920F931F93CF934D
:105C2000DF93CDB7DEB7C054D1090FB6F894DEBF0D
:105C30000FBECDBF80910E0990910F09059709F411
:105C400049C06115710509F445C069017A018B01EC
:105C500040E450E0CE0101960E9492C36FE270E0F2
:105C6000CE0101960E9459C3892B41F4980143E06B
:105C700050E060E4CE0101960E94382D4FE350E0E1
:105C8000B601CE0101960E9474C30E94B78A882390
:105C900009F180910E0990910F090697D9F480912E
:105CA0009A08811117C0B701CE0101960E947E9615
:105CB00081E090E0C05CDF4F0FB6F894DEBF0FBE0E
:105CC000CDBFDF91CF911F910F91FF90EF90DF90AB
:105CD000CF90089590E080E0EDCFAF92BF92CF9249
:105CE000DF92EF92FF921F93CF93DF9300D000D00B
:105CF000CDB7DEB76C017C0110E08AE0A82EB12C94
:105D0000133061F1F701828190E0B0E0A0E0898377
:105D10009A83AB83BC83BE82AD82BE016F5F7F4F2F
:105D200085E99DE00E9479186CE575E10E94CA78CA
:105D30001F5FFFEFEF1AFF0A143011F726960FB618
:105D4000F894DEBF0FBECDBFDF91CF911F91FF90C2
:105D5000EF90DF90CF90BF90AF900895F6018581CE
:105D600090E0B0E0A0E089839A83AB83BC83BE82DD
:105D7000AD82BE016F5F7F4F84EE9CE00E94791878
:105D80006AE575E1D3CF69E072E184EE9CE00E94A0
:105D9000CA7866EF71E184EE9CE00E94CA7868EEF2
:105DA00071E184EE9CE00E94CA7860EE71E184EEBD
:105DB0009CE00E94CA7884EE9CE00E94C17763ED6B
:105DC00071E184EE9CE00E94CA7863EC71E184EE9C
:105DD0009CE00E94CA7867EB71E184EE9CE00E942F
:105DE000CA7860EA71E184EE9CE00E94CA786EE8AD
:105DF00071E184EE9CE00E94CA7869E771E184EE6B
:105E00009CE00E94CA786AE671E184EE9CE00E9400
:105E1000CA786BE571E184EE9CE00E94CA7863E584
:105E200071E184EE9CE00E94CA7868E471E184EE3E
:105E30009CE00E94CA786EE371E184EE9CE00E94CF
:105E4000CA7866E371E184EE9CE00E94CA786AE257
:105E500071E184EE9CE00E94CA7860E171E184EE19
:105E60009CE00E94CA7861EF70E184EE9CE00E94A1
:105E7000CA786CED70E184EE9CE00E94CA786FEC09
:105E800070E184EE9CE00E94CA7861EC70E184EEDF
:105E90009CE00E94CA7865EB70E184EE9CE00E9471
:105EA000CA786DEA70E184EE9CE00E94CA7862EAEA
:105EB00070E184EE9CE00E94CA7865E970E184EEAE
:105EC0009CE00E94CA786DE870E184EE9CE00E943C
:105ED000CA7862E870E184EE9CE00E94CA7863E7C9
:105EE00070E184EE9CE00E94CA786AE670E184EE7C
:105EF0009CE00E94CA7884EE9CE00C94C1770F93DA
:105F00001F93CF93DF9300D000D0CDB7DEB70E94B0
:105F1000C32E62E87BE084EE9CE00E94CA78CE014A
:105F200001960E94E428CE0101960E946D2E00E0A9
:105F300014E01A8309838091600C9091610CA09108
:105F4000620CB091630C8B839C83AD83BE83CE01C6
:105F500001960E946D2E1A8309831B821C821D826A
:105F60001E8280E591E00E94019044E050E0BE0175
:105F70006D5F7F4F81E090E00E94BA81CE01019673
:105F80000E946D2E1A8309831B821C821D821E8231
:105F900080E591E00E94019044E050E0BE016D5F19
:105FA0007F4F85E090E00E94BA81CE0101960E9469
:105FB0006D2E68EA7BE084EE9CE00E94CA7826960B
:105FC0000FB6F894DEBF0FBECDBFDF91CF911F910A
:105FD0000F910895009789F0FC0120852F702530DE
:105FE00061F40E94188B009741F0FC0120852F700E
:105FF000243019F481859285089590E080E0089519
:10600000CF92DF92EF92FF920F931F93CF93DF9384
:1060100000D000D0CDB7DEB78091970881119CC029
:1060200080910E0990910F0902970CF495C0009190
:106030007407109175070115110509F48DC062E010
:1060400072E083EB9DE00E94EC146FE575E0C801FF
:106050000E949C8A8C01009709F47EC00E942D8BBF
:10606000E82EF12CE114F10409F476C070E060E050
:10607000C8010E94EA2F6C01EA94EF2809F47BC062
:1060800061E0C8010E94188BFC0101851285CE01D8
:1060900001960E94E428CE0101960E94099063E7D0
:1060A0007BE084EE9CE00E94CA78B60184EE9CE01E
:1060B0000E9464786FE177E084EE9CE00E9464784F
:1060C000B80184EE9CE00E94258B6FE177E084EEBE
:1060D0009CE00E94647860E57AE084EE9CE00E9497
:1060E000647884EE9CE00E94C177D092A90DC092A2
:1060F000A80D1093AB0D0093AA0D80E59AE0892BB3
:10610000E9F58DE595E09093AD0D8093AC0D809110
:10611000090990910A09009741F070E060E00E943F
:10612000EA2F9093080980930709809107099091BD
:106130000809009721F09093AF0D8093AE0D109257
:10614000B10D1092B00D81E0809397086AE57BE075
:1061500084EE9CE00E94CA7826960FB6F894DEBFC3
:106160000FBECDBFDF91CF911F910F91FF90EF90A8
:10617000DF90CF90089502E012E089CF80E59AE0A9
:10618000C2CFCF92DF92EF92FF921F93CF93DF9314
:1061900000D000D0CDB7DEB765E57BE084EE9CE0B3
:1061A0000E94CA7889ECE82E8CE0F82E10E090E18D
:1061B000C92ED12CF70181917F01803130F466E640
:1061C00075E084EE9CE00E946478153041F1F7019F
:1061D0003197808190E0B0E0A0E089839A83AB831F
:1061E000BC83DE82CD82BE016F5F7F4F84EE9CE078
:1061F0000E94791863E57BE00E94CA781F5F163021
:10620000C9F626960FB6F894DEBF0FBECDBFDF915C
:10621000CF911F91FF90EF90DF90CF9008958091E4
:10622000CE0C90E0B0E0A0E089839A83AB83BC837E
:10623000DE82CD82BE016F5F7F4F84EE9CE00E94C4
:1062400079180E94C177DACFEF92FF920F931F93D4
:10625000CF93DF9300D000D01F92CDB7DEB77B0184
:10626000CE0107969F938F9301979F938F930197EA
:106270009F938F9301979F938F9301979F938F93F2
:1062800001979F938F938E010F5F1F4F1F930F9363
:1062900088E695E09F938F93DB0113968C9113977B
:1062A0008F9312968C918F930E9419C40FB6F89415
:1062B000DEBF0FBECDBF0697DCF46AE17FE08EEE55
:1062C0009CE00E94CA78D70112966D917C918EEE67
:1062D0009CE00E94647827960FB6F894DEBF0FBE4C
:1062E000CDBFDF91CF911F910F91FF90EF90089557
:1062F0008091C70C9091C80C892BA9F10E949C8BAE
:10630000882389F181E60E943A8B8091C70C909195
:10631000C80CDC01ED91FC910684F785E02D64E06A
:1063200070E019958091C70C9091C80CDC01ED913B
:10633000FC910280F381E02D46E050E0B801199510
:1063400086E0F801A9ECBCE001900D928A95E1F796
:106350008091C70C9091C80CDC01ED91FC910288F2
:10636000F389E02D19950E94C1306CE27FE084EE44
:106370009CE00E94CA78AFCFEF92FF920F93CF9329
:10638000DF93CDB7DEB7A0970FB6F894DEBF0FBE90
:10639000CDBF7C0100E020E033E040E250E0BE01F0
:1063A0006F5F7F4F0E94B61FBE016F5F7F4F85E911
:1063B0009DE00E94647866ED7AE085E99DE00E94A8
:1063C000CA78F701628162956F7085E99DE00E944D
:1063D000118B6FEC7AE085E99DE00E94CA78F701A5
:1063E00062816F7085E99DE00E94118B85E99DE0D7
:1063F0000E94C177A0960FB6F894DEBF0FBECDBF46
:10640000DF91CF910F91FF90EF9008952F923F92DF
:106410004F925F926F927F928F929F92AF92BF92B4
:10642000CF92DF92EF92FF920F931F93CF93DF9360
:10643000CDB7DEB768970FB6F894DEBF0FBECDBFFD
:106440001C0109871A872B873C874D875E876F87DA
:10645000788B2DE0E216F10408F035C0F701E05E1C
:10646000FC4F3081398BCE0109960E94C11197FDF6
:1064700004C0BC01C1010E94E3119B85892F8F706C
:10648000D1011296EC911297E07FE82B1296EC93D3
:10649000129789858C93E295EF70EC3008F063C019
:1064A000F0E08827E95AFD4C8F4F0C940BBF5B340A
:1064B00080328032FA3365328534C3330434043495
:1064C0000434C333C333198ACECFB12C92959F7055
:1064D0009D3008F0BEC4E92FF0E08827ED58FD4C50
:1064E0008F4F0C940BBFB332BF34DF34BF348834CA
:1064F0008834BF34BF3429372937BF34BF3493338E
:1065000092959F709D3008F01EC1E92FF0E088271A
:10651000E357FD4C8F4F0C940BBFB33267335B33A3
:106520001D339D329A323E336B33A333A33328336A
:10653000283393338889F10187838F85D10116969B
:106540008C9316978E8515968C9315978D8514963A
:106550008C9314979295907F12968C9112978F70CE
:10656000982B12969C93B989BB2309F463C0F1015F
:10657000828182958F702B2F30E08217130609F4E9
:1065800059C065E579E085E99DE00E94CA78D101AE
:1065900012966C9162956F7085E99DE00E94118B57
:1065A00062E579E085E99DE00E94CA78698985E91C
:1065B0009DE00E94118B60E579E085E99DE00E94F5
:1065C000CA78F101008119821A821B821C821D8205
:1065D0001E821F82188689898295807F9B819F7089
:1065E000892B8B830983EE24EA94FE2C118122816E
:1065F00033814481558166817781CE0101960E9465
:106600000632D1012C9311963C93119712964C931C
:10661000129713965C93139714966C931497159690
:106620007C93159716968C93169717969C93C10199
:106630000E94BC3188E0F1017BC18F859889F1010E
:106640008683878190FB80F987838E8585838BCFB6
:106650008D859E85AF85B8898F3F9105A105B105D0
:1066600029F024F08FEF90E0A0E0B0E0B7FF03C086
:1066700080E090E0DC01F101848375CF6D857E853B
:106680008F8598892AE030E040E050E00E94A2BE69
:106690002F3F31054105510529F024F02FEF30E05F
:1066A00040E050E057FF03C020E030E0A901D101F5
:1066B00014962C9358CF8F859889F1018683878112
:1066C00090FB80F987838E8585838D85D5CF8D85D9
:1066D00014968C9348CFCD84DE84EF84F88820E034
:1066E00030E0A901C701B6010E9436BD87FD17C081
:1066F00020E030E04FE753E4C701B6010E943EC0FE
:10670000181634F4C12CD12CAFE7EA2EA3E4FA2EEC
:10671000C701B6010E940FC0F101648324CFC12CD0
:10672000D12C7601F5CFD10112968C9112978F70F2
:10673000806C12968C9312978D859E8515969C93EE
:106740008E93149710CF65ED79E085E99DE00E9466
:10675000CA786B8562956F7085E99DE00E94118B08
:1067600062ED79E085E99DE00E94CA78F1016281DD
:1067700062956F7085E99DE00E94118B85E99DE02F
:106780000E94C177F0CE92959F70933091F09C302B
:1067900051F24D855E856F857889F101448355837B
:1067A000668377839295907F82818F70982B9283F6
:1067B000DACE60E0C1010E946810D10114968C937A
:1067C00014978F85988916968C93169717968C91A7
:1067D000179790FB80F917968C9317978E851596CF
:1067E0008C93159712968C9112978F7080621296E7
:1067F0008C93B9CE60E0CE0109960E946810D10159
:1068000014968C931497EECF92959F709D3008F05C
:1068100065C0E92FF0E08827EF5EFB4C8F4F0C94AA
:106820000BBFB33230345A34D9335A345A341E344D
:106830004A344A344A343E34453493336D857E8538
:106840008F8598890E943DBD20E030E040E251E410
:106850000E9496BFF101648375838683978383CEFC
:106860006D8570E090E080E00E943BBDD101149600
:106870006D937D938D939C93179775CE6D857E85D3
:106880008F8598890E943DBDE5CF6D857E858F857A
:106890009889EACF9295907FF10182818F70982B31
:1068A00092838D859E85AF85B88984839583A683E1
:1068B000B78359CE9295907FD10112968C91129701
:1068C0008F70982B12969C938D859E85AF85B88985
:1068D000F10184839583A683B78345CE60EC79E08C
:1068E00085E99DE00E94CA786B8562956F7085E9A5
:1068F0009DE00E94118B6DEB79E085E99DE00E949F
:10690000CA78D10112966C9133CFBB24B394DECDFB
:106910004D855E856F857889F10144835583668353
:1069200077839295907F82818F70982B928388E0F5
:10693000DE01119601900D928A95E1F729813A8145
:106940004B815C816D817E818F81988568960FB6C1
:10695000F894DEBF0FBECDBFDF91CF911F910F9195
:10696000FF90EF90DF90CF90BF90AF909F908F906F
:106970007F906F905F904F903F902F90089596304A
:1069800009F43AC148F46D85913071F06FEF70E011
:10699000933051F060E008C0973009F439C19A5043
:1069A0006D857E859230B0F784E68F8788898E7FEB
:1069B000888B1E868B858F7080628B876D872E8576
:1069C00030E0AFEFB0E00E94D4BE24E630E040E01B
:1069D00050E00E94A2BE69017A01FFEFCF16D104F8
:1069E000E104F10429F024F0C12CD12C7601CA94E1
:1069F00086012D852A8B622E712CBB2009F471C073
:106A000088898695A82FA150BB0B2D01BFEF4B168F
:106A10005B0609F01EC1003811050CF000C18FE7BC
:106A200090E08C199D09869DD001879DB00D969DA3
:106A3000B00D11242FEF30E00E9422BF21E83EE785
:106A400040E050E00E94A2BEF1012783ABE9B0E034
:106A5000A70196010E94C1BEEFE78E2E912CA12CBA
:106A6000B12CA50194010E94A2BE89019A010C5982
:106A70001F4F2F4F3F4FAEEFB1E0A70196010E948D
:106A8000C1BEA50194010E94A2BED3010E94C1BE55
:106A90002FEF30E040E050E00E94A2BE39012FEF1E
:106AA0006216710421F01CF066246A94712C60EB6C
:106AB00079E085E99DE00E94CA78B80185E99DE00A
:106AC0000E94258B62EA79E085E99DE00E94CA7800
:106AD000B30185E99DE00E94258B85E99DE00E9438
:106AE000C177EDE6F9E1E491F0E0EE0FFF1FED5A1A
:106AF000F64E85919491E3ECF9E1E4912F85388984
:106B00003170AFEFBFEF0E94D4BE2DE631E040E020
:106B100050E00E94A2BE44275527AAEFB5E00E948C
:106B2000C1BEDC01CB019058AF4FBF4FCD01BB2799
:106B300097FDB095AB2F8E3FE1E09E0708F062C154
:106B4000382F8F3F910508F47FC14EEF481B50E06E
:106B50003FEFF301319678012FEFE21AF20A009528
:106B600010E03E9DC0013F9D900D1124292F332739
:106B7000200F311FDF010E9422BF4B015C018824DE
:106B8000AA24BB245E9D90015F9D300D1124232F0C
:106B90003327200F311F0E9422BFBB27A92F982F18
:106BA000872F882A992AAA2A4E9D90014F9D300D41
:106BB0001124232F3327200F311FDF010E9422BF12
:106BC000B82FA72F962F882788279927BB27882992
:106BD0009929AA29F101A6839583848366E779E040
:106BE00085E99DE00E94CA78C1010E94BC3160E045
:106BF00080E00E945093B7CC6D857E858F85988903
:106C00002AE030E040E050E00E94A2BEB901CCCEC4
:106C10006D857E858F8598890E9408C0C5CEA701A5
:106C200096012058310941095109ABE9B0E00E94B1
:106C3000C1BE2FE730E040E050E00E94A2BE8901D3
:106C40009A010C591F4F2F4F3F4FD10117961C929D
:106C50002ECF9201AAEBBFEF0E941ABF44E6842E0A
:106C6000912CA12CB12CA50194010E94A2BEDA01A5
:106C7000C9018C599F4FAF4FBF4F8B8B9C8BAD8BF6
:106C8000BE8B26E430E0D2010E9422BFA501940110
:106C90000E94A2BE49015A019EE1890E911CA11CCD
:106CA000B11C003811050CF093C08FE790E08C19EF
:106CB0009D09869DD001879DB00D969DB00D112434
:106CC000A50194010E94CCBE9B01AC01AFEFB0E0E6
:106CD0000E94C1BE24E63AE640E050E00E94A2BE17
:106CE000D10117962C932B893C894D895E892C0DF7
:106CF0003D1D4E1D5F1DAEEFB1E00E94C1BE23EEF3
:106D000030E040E050E00E94A2BE29013A01388FF5
:106D10002F8BAFEFB0E0A70196010E94C1BE2FE715
:106D200030E040E050E00E94A2BE8901EA89AE2F27
:106D3000B0E0A30192010E94C1BE2FEF30E040E01D
:106D400050E00E94A2BE39012F3F310521F01CF016
:106D500066246A94712C6CE979E085E99DE00E94D3
:106D6000CA782AE030E04B895C896D897E8985E9A3
:106D70009DE00E94DE7766E979E085E99DE00E946A
:106D8000CA782AE030E0B501A40185E99DE00E94BF
:106D9000DE776EE879E085E99DE00E94CA78B80167
:106DA00085E99DE00E94258B66E879E085E99DE014
:106DB0000E94CA78B30185E99DE00E94258B6DE7AA
:106DC00079E085E99DE00E94CA786F89788D81CE4F
:106DD000A70196012058310941095109ABE9B0E0FA
:106DE0000E94C1BE2FE730E040E050E00E94A2BE0A
:106DF00089019A010C591F4F2F4F3F4FD101179610
:106E00001C92A9CF8C3FF3E09F0768F48D3F22E0EE
:106E1000920728F452E0580F3FEF40E09ACE3CEF43
:106E2000381B5FEFFACF8A3F35E0930781F08B3F45
:106E3000E4E09E0728F444E0480F5FEF30E089CE9D
:106E40005AEF581B30E001C050E04FEF82CE50E0C7
:106E5000F9CF64E679E085E99DE00E94CA786B8508
:106E600062956F7085E99DE00E94118B61E679E083
:106E700044CDAF92BF92CF92DF92EF92FF920F93E9
:106E80001F93CF93DF93CDB7DEB768970FB6F89413
:106E9000DEBF0FBECDBFFC01098B1A8B2B8B3C8B49
:106EA0004D8B5E8B6F8B788F82819381009709F475
:106EB0009FC024813581232B09F49AC0CC2009F48A
:106EC00097C06F0170E060E00E94A91C192FD601E5
:106ED000ED91FC91028CF38DE02DC60119955C01BA
:106EE0008230910509F478C0039709F447C095E012
:106EF000F1E0AF16B10409F091E019861A861B86FD
:106F00001C861D861E861F86188A9295907F8B850B
:106F10008F70892B8B87EE24EA94FE2C09891A89BD
:106F20002B893C894D895E896F89788DCE010996C0
:106F30000E940632F1E0AF16B10409F44FC082E0BE
:106F4000A816B10409F045C06F8570E0D60114960B
:106F50008C910E948C9361E070E0C6010E94D41C69
:106F60006E8570E00E948C9362E070E0C6010E9422
:106F7000D41C6D8570E00E948C932BC0612F661F1E
:106F80006627661FCE0141960E9468105C01BC0115
:106F9000D60114968C910E948C936CE375E185E97F
:106FA0009DE00E94CA78F6016481758185E99DE0C3
:106FB0000E94258B6AE375E185E99DE00E94CA780D
:106FC000B50185E99DE00E94258B85E99DE00E9441
:106FD000C17781E090E00EC094E08FCF63E070E075
:106FE000C6010E94D41C688970E00E948C93ACCFCB
:106FF00090E080E068960FB6F894DEBF0FBECDBF7C
:10700000DF91CF911F910F91FF90EF90DF90CF9084
:10701000BF90AF900895AF92BF92CF92DF92EF9260
:10702000FF920F931F93CF93DF93CDB7DEB7CC556D
:10703000D1090FB6F894DEBF0FBECDBF5C016696D6
:107040000FAF669767961FAF679768962FAF6897E1
:1070500069963FAF69976A964FAF6A976B965FAF35
:107060006B976C966FAF6C976D967FAF6D971AAA02
:1070700019AAFE01F39682E1DF011D928A95E9F7D4
:107080007A961192119286E0DF011D928A95E9F7B6
:10709000CE018B5A9F4F0E94BC31F0FE2CC06696E9
:1070A000EFAD6697E83108F08DC0F0E08827E45A2C
:1070B000F74C8F4F0C940BBFE8387438DF38E23848
:1070C000E238DF387438E238E238E238743874383D
:1070D0007438E238E238E238E238E238E238E2384E
:1070E000E238E238E238E8386DE479E0CE01835BDB
:1070F0009F4F0E94DFB568968FAD689782958F701D
:10710000813008F48DC0833018F0883009F088C0D1
:107110000E94B78A882309F423C180919A088111BB
:107120001FC1C114D10409F01BC130E020E043E0CD
:1071300050E060E3CE0101960E94382DD501ED911B
:10714000FC91608171814FE250E0CE0101960E9476
:1071500074C301E020E032E044E150E0BE016F5C26
:107160007F4FCE018B5A9F4F0E94B61FF1FE07C082
:1071700066968FAD6697823011F0853061F5F0FE2E
:107180004FC0BE01635B7F4FCE0101960E947E9689
:107190006CE279E085E99DE00E94CA78BE016F5FEC
:1071A0007F4F85E99DE00E94647869E279E085E996
:1071B0009DE00E94CA78BE01635B7F4F29C069E4ED
:1071C00079E094CF6BE379E085E99DE00E94CA788D
:1071D000E894F0F890CFBE016F5C7F4FCE0101962E
:1071E0000E947E9665E379E085E99DE00E94CA7879
:1071F000BE016F5F7F4F85E99DE00E94647862E386
:1072000079E085E99DE00E94CA78BE016F5C7F4FFE
:1072100085E99DE00E94647885E99DE00E94C17740
:1072200068968FAD6897807F87010027107188234B
:1072300011F0F1FC04C00115110509F4BDC030E0E6
:1072400020E043E050E060E3CE0101960E94382D3B
:10725000D501ED91FC91608171814FE250E0CE014A
:1072600001960E9474C3C114D10469F06BE575E006
:10727000CE0101960E944EC34FE250E0B601CE010E
:1072800001960E9474C36BE575E0CE0101960E94E1
:107290004EC34FE250E065E279E00115110511F4AB
:1072A00061E279E0CE0101960E94EFB568968FAD5C
:1072B000689782958F708450823008F069C067E1CA
:1072C000CE018B5A9F4F0E94111026962FAF269702
:1072D00027963FAF279728964FAF289729965FAFFD
:1072E00029972A966FAF2A972B967FAF2B972C96CC
:1072F0008FAF2C972D969FAF2D9700E020E033E0C5
:1073000044E150E0BE016F5C7F4FCE018B5A9F4F2E
:107310000E94B61F6BE179E085E99DE00E94CA7882
:10732000BE016F5F7F4F85E99DE00E94647868E150
:1073300079E085E99DE00E94CA78BE016F5C7F4FCD
:1073400085E99DE00E94647885E99DE00E94C1770F
:107350000E94B78A882321F080919A08882301F13E
:10736000B701C5010E944F1D90E080E0C45ADF4F75
:107370000FB6F894DEBF0FBECDBFDF91CF911F9146
:107380000F91FF90EF90DF90CF90BF90AF90089556
:1073900020E032E0012B11F020E033E000E0B0CF3C
:1073A000BE016F5C7F4FCE0101960E947E9660E029
:1073B00072E0C5010E942A1DF0FE73C066968FAD73
:1073C00066978A3009F478C008F06EC0813009F4FD
:1073D0007EC0863009F47BC030E020E043E050E01E
:1073E00060E3CE0101960E94382DD501ED91FC910C
:1073F000608171814FE250E0CE0101960E9474C31A
:10740000C114D10469F06BE575E0CE0101960E94CC
:107410004EC34FE250E0B601CE0101960E9474C304
:107420006BE575E0CE0101960E944EC340E350E04B
:1074300065E079E0CE0101960E94EFB56FEF78E04C
:1074400085E99DE00E94CA78BE016F5F7F4F85E9A4
:107450009DE00E9464786CEF78E085E99DE00E94F1
:10746000CA78BE01635B7F4F85E99DE00E94647826
:1074700085E99DE00E94C1770E94B78A882309F4BC
:107480006FCF80919A0881116BCFBE01635B7F4FF4
:10749000CE0101960E947E9660E071E0C5010E94D7
:1074A0002A1D81E090E062CF8B3071F08C3009F0C2
:1074B00093CF63E179E002C06EE079E0CE01835BB7
:1074C0009F4F0E94DFB588CF69E079E0F7CFF501E3
:1074D0008085853009F080CFECCFCF92DF92FF928C
:1074E0000F931F93CF93DF93F12C6115710509F46E
:1074F00058C06A01EB018C01CB010E943612F82EB4
:10750000882309F44EC0D0FE05C0F8016081CE0189
:107510000E94881DD1FE3CC0F801928192959F7017
:107520004481558166817781973030F09930D0F071
:1075300086EF890F823090F0EC81FD81309771F0F9
:1075400080858F702EEF280F223010F0811106C039
:107550009295907F80858F70982B9087CE010E94A6
:10756000421216C0EC81FD81309791F080858F70BA
:107570009EEF980F923010F081110AC04187528718
:1075800063877487EC81FD818085807F836080873D
:1075900067EE79E085E99DE00E94CA78C8010E9403
:1075A000BC318F2DDF91CF911F910F91FF90DF9014
:1075B000CF900895CF92DF92EF92FF920F931F9397
:1075C000CF93DF936115710509F478C06A017B01DF
:1075D0008C01CB010E943612D82F8823E1F1D7010C
:1075E00014968D919C91009709F44AC0FC01C085C6
:1075F0002C2F2F703EEF320F323010F0211135C09A
:10760000C595C595C595C595D0FE76C0C7010E94A4
:107610009E1EF8018083CC2309F441C0C295C07F2F
:1076200082818F70C82BC283D70114968D919C9153
:10763000009789F1FC0120852F70223019F5818592
:107640009285A385B485F80184839583A683B78347
:10765000C8010E94BC318D2FDF91CF911F910F91F6
:10766000FF90EF90DF90CF900895253049F460E0CF
:107670000E94188B009721F0DC011896CC91C0CFA6
:10768000C0E0C2CF253039F460E00E94188B00972B
:1076900011F0FC01D4CF80E090E0DC01D4CFD70121
:1076A0001496ED91FC9180858295807F85958595D6
:1076B00085958595823021F0833081F0D0E0CBCF65
:1076C0004185528563857485F80182818F70806A57
:1076D00082834483558366837783BDCF41855285FA
:1076E00063857485F80182818F708067828344830B
:1076F000558366837783AFCFCC2389F2C295C07F51
:10770000F8018ECF0F931F93CF93DF9300D000D05B
:107710001F921F92CDB7DEB719821A821B821C827C
:107720001D821E821F8218862B812F702B83FC01E5
:1077300002811381C8010E949E1E8230C9F08530EB
:10774000B9F040E052E0B801CE0101960E94DA3A69
:1077500060E0CE0101960E94681028960FB6F8945A
:10776000DEBF0FBECDBFDF91CF911F910F91089566
:1077700090E080E0F2CFAF92BF92CF92DF92EF9293
:10778000FF920F931F93CF93DF9300D000D01F92EF
:107790001F92CDB7DEB75C017B0160FF03C0E894A8
:1077A000E0F8F3F8F3FC0DC00E94520F6639710542
:1077B0008105910530F080910E0990910F09059790
:1077C000F9F4B70166277370C5010E944F1D6BEE77
:1077D00078E085E99DE00E94CA788FEF9FEF2896B8
:1077E0000FB6F894DEBF0FBECDBFDF91CF911F91D2
:1077F0000F91FF90EF90DF90CF90BF90AF900895E2
:1078000019821A821B821C821D821E821F82188688
:107810008B818F708B8340E053E0B501CE010196E0
:107820000E94DA3A60E073E0C5010E94721DE82A06
:10783000F92AD12CC12C09811A812B813C814D81DF
:107840005E816F817885C5010E940B38C8CF3F9259
:107850004F925F926F927F928F929F92AF92BF9260
:10786000CF92DF92EF92FF920F931F93CF93DF930C
:10787000CDB7DEB7CC5BD1090FB6F894DEBF0FBE33
:10788000CDBF4C01C755DF4F0883C95AD040C655FC
:10789000DF4F1883CA5AD040C555DF4F2883CB5AD3
:1078A000D040C455DF4F3883CC5AD040C355DF4F4A
:1078B0004883CD5AD040C255DF4F5883CE5AD0406E
:1078C000C155DF4F6883CF5AD040C055DF4F788312
:1078D000C05BD040CF54DF4FF982E882C15BD0401B
:1078E0005C2C0E94B095C754DF4F688379838A83EC
:1078F0009B83C95BD040C555DF4F8881CB5AD040B0
:107900008F70682E712CC0900E09D0900F09C95449
:10791000DF4FD982C882C75BD040CF54DF4FE881A8
:10792000F981C15BD040309721F0808181110C94A6
:107930008046D4011B968C91882341F0C4010B969C
:10794000CF54DF4F99838883C15BD04061147104A9
:1079500011F00C94C946CF54DF4FE881F981C15B27
:10796000D040309711F00C948446F40165887688F5
:107970006114710411F40C94C946C555DF4F888118
:10798000CB5AD0408F7011F00C94C946662DCE01B1
:1079900087559F4F0E94EA0FC756DF4F2883C9596A
:1079A000D040C656DF4F3883CA59D040C556DF4F46
:1079B0004883CB59D040C456DF4F5883CC59D04070
:1079C000C356DF4F6883CD59D040C256DF4F78830E
:1079D000CE59D040C156DF4F8883CF59D040C056D2
:1079E000DF4F9883C05AD0400C94C946CE018755CA
:1079F0009F4F0E94BC31F40180819181009711F466
:107A00000C940C47FDE06F16710409F0A5C00E94AC
:107A10002D8B082F10E006301105A4F40E94C180C0
:107A2000009739F0DC0118962C911897207F189652
:107A30002C93BC01F401808191810E94FD8D0F5F28
:107A40001F4FE9CF65E0D4018D919C910E94188B66
:107A50008C01892BE1F410E000E0C801C454DF4F31
:107A60000FB6F894DEBF0FBECDBFDF91CF911F914F
:107A70000F91FF90EF90DF90CF90BF90AF909F90CD
:107A80008F907F906F905F904F903F900895C75573
:107A9000DF4F8881C95AD0408031E8F6CE01875542
:107AA0009F4F0E947C1116161706180619060CF037
:107AB00048C00E94B0956B017C01CE0187559F4F55
:107AC0000E947C11C60ED71EE81EF91EF801C18661
:107AD000D286E386F486C755DF4F8881C95AD040E5
:107AE0008295807F8260808767E578E085E99DE008
:107AF0000E94CA78CE0187559F4F0E947C11AB012E
:107B0000BC012AE030E085E99DE00E94DE7761E576
:107B100078E085E99DE00E94CA78D80119964D91D8
:107B20005D916D917C911C972AE030E085E99DE0A4
:107B30000E94DE7785E99DE00E94C17701E010E0B8
:107B40008CCFF80180858F70808767E478E085E9C5
:107B50009DE00E94CA78EECFC755DF4FF880C95A22
:107B6000D040F4E0FF1609F403C3FF1530F0FF2006
:107B700009F477C0B12CA12CB8C288EF8F0D8230E8
:107B8000C8F788E0FE01E755FF4FDE01119601902E
:107B90000D928A95E1F7C555DF4F8881CB5AD040C9
:107BA000807F09F43EC3CE0187559F4F0E947C1110
:107BB0008B01672B09F435C369E0C62EFC1003C0A6
:107BC000119501951109B401CE0187559F4F0E946F
:107BD000588E60E0CE0187559F4F0E9411106A9623
:107BE0002FAF6A976B963FAF6B976C964FAF6C97C2
:107BF0006D965FAF6D976E966FAF6E976F967FAF16
:107C00006F97A0968FAFA097A1969FAFA19722E004
:107C10006216710409F450C30CF006C3CC24C3945B
:107C20006114710409F0A6CFC555DF4FE881CB5A26
:107C3000D040E295EF70E150EB3008F0C3C3F0E0C4
:107C40008827EA5DF14C8F4F0C940BBF5E415E417B
:107C5000E241E241E241BD419941994199417B4173
:107C60007B4119821A821B821C821D821E821F8206
:107C700018868B818F708B83C555DF4F8881CB5AD7
:107C8000D040807F09F476CF29E06216710409F4B0
:107C90002EC20CF015C16114710409F435C192E0D3
:107CA0006916710409F066CFB12CA12CC12C3324C4
:107CB0003A94B401CE0101960E94588E8B81982F80
:107CC00092959F70945F9F70923060F4C555DF4F1E
:107CD0009881CB5AD04092959F70923019F48F7052
:107CE00080628B83F4019085973071F4C555DF4F26
:107CF0008881CB5AD040807E803211F0803421F4CC
:107D00008B818F7080628B83F401A185B285892F6E
:107D100090E0109741F0ED91FC911197028CF38D5A
:107D2000E02DCD0119957C01C755DF4F0881C95A57
:107D3000D040C655DF4F1881CA5AD040C555DF4FD5
:107D40002881CB5AD040C455DF4F3881CC5AD0401F
:107D5000C355DF4F4881CD5AD040C255DF4F5881BF
:107D6000CE5AD040C155DF4F6881CF5AD040C05560
:107D7000DF4F7881C05BD040CE0101960E94063271
:107D8000CF57DF4F2883C158D040CE57DF4F3883BD
:107D9000C258D040CD57DF4F4883C358D040CC574E
:107DA000DF4F5883C458D040CB57DF4F6883C55846
:107DB000D040CA57DF4F7883C658D040C957DF4FED
:107DC0008883C758D040C857DF4F9883C858D040E1
:107DD000CE0101960E94BC31CC2069F1C555DF4F20
:107DE0008881CB5AD04082958F709FE0980F9F700A
:107DF000923020F08A5F8F708230E8F48B81829518
:107E00008F7081508230B8F42D8130E0AFEFB0E058
:107E10000E94D4BE24E630E040E050E00E94A2BEC2
:107E20002F3F31054105510529F024F02FEF30E0B7
:107E300040E050E02D8388E0FE013196DE01A75539
:107E4000BF4F01900D928A95E1F7FAE0BF2AD12C3D
:107E5000D40118968C911897873009F009C45520E1
:107E600009F41DC31296ED91FC9190859F70953099
:107E700009F015C3C954DF4F88819981C75BD04091
:107E8000059709F40CC3CF54DF4F48815981C15B7A
:107E9000D040BE0167557F4FCF010E949D4901E050
:107EA00010E0C755DF4F8881C95AD040853009F4AA
:107EB000B3C308F0F7C2833009F422C3312C90C356
:107EC000AAE06A16710409F4BFC0BBE06B16710426
:107ED00009F050CEB401CE0101960E94588ECE0119
:107EE00087559F4F0E94C111BC01CE0101960E948F
:107EF000E31188E0FE013196DE01A755BF4F0190E6
:107F00000D928A95E1F7EEC0C4010E945D4A8C0192
:107F100061E070E01816190614F070E060E085E981
:107F20009DE00E94258B6AE676E085E99DE00E944F
:107F30006478CE0187559F4F0E947C11AB01BC0134
:107F40002AE030E085E99DE00E94DE7785E99DE04A
:107F50000E94C177CE0187559F4F101611060CF075
:107F6000C5C60E947C11B12CA12C672B682B692BF4
:107F700089F562E0CE0187559F4F0E941110CF56C0
:107F8000DF4F2883C159D040CE56DF4F3883C259C6
:107F9000D040CD56DF4F4883C359D040CC56DF4F39
:107FA0005883C459D040CB56DF4F6883C559D04061
:107FB000CA56DF4F7883C659D040C956DF4F8883F1
:107FC000C759D040C856DF4F9883C859D040AA241B
:107FD000A394BA2CCC24C394332433946ACE61E0A6
:107FE000CE0187559F4F0E941110C757DF4F28833E
:107FF000C958D040C657DF4F3883CA58D040C557FC
:10800000DF4F4883CB58D040C457DF4F5883CC58FC
:10801000D040C357DF4F6883CD58D040C257DF4FA1
:108020007883CE58D040C157DF4F8883CF58D04097
:10803000C057DF4F9883C059D040AA24A394BA2CCC
:10804000CC24C394312C35CEB401CE0101960E94CC
:10805000588EC255DF4F9881CE5AD0408B81282F41
:1080600022952F7041F0223049F0B12CA12CDD2453
:10807000D394C12C3DC18F7080628B83892F90E097
:108080008536910514F084E690E08E8388E0FE0149
:108090003196DE01A755BF4F01900D928A95E1F709
:1080A00062E0CE0187559F4F0E94EA0FEA962FAFFC
:1080B000EA97EB963FAFEB97EC964FAFEC97ED96C8
:1080C0005FAFED97EE966FAFEE97EF967FAFEF97BE
:1080D000C158DF4F8883CF57D040C058DF4F9883B7
:1080E000C058D040A12CFAE0BF2ED12CC2CFB40191
:1080F000CE0101960E94588EC155DF4F6881CF5A3C
:10810000D040C055DF4F7881C05BD0407170CE0148
:1081100001960E941712C82E882309F45DC188E0D9
:10812000FE013196DE01A755BF4F01900D928A9551
:10813000E1F762E0CE0187559F4F0E94EA0FE29679
:108140002FAFE297E3963FAFE397E4964FAFE49704
:10815000E5965FAFE597E6966FAFE697E7967FAF58
:10816000E797E8968FAFE897E9969FAFE997BACF80
:10817000C4010E945D4A181619063CF562E0CE0162
:1081800087559F4F0E941110AA962FAFAA97AB96C2
:108190003FAFAB97AC964FAFAC97AD965FAFAD9797
:1081A000AE966FAFAE97AF967FAFAF97E0968FAFBB
:1081B000E097E1969FAFE197AA24A394BA2CD12C23
:1081C000CC24C3943324339443CEB401CE018755D9
:1081D0009F4F0E94588E61E0CE0187559F4F0E94AD
:1081E0001110A2962FAFA297A3963FAFA397A49684
:1081F0004FAFA497A5965FAFA597A6966FAFA6972A
:10820000A7967FAFA797A8968FAFA897A9969FAF7D
:10821000A997AA24A394BA2CD12CCC24C394312C92
:1082200017CE05E010E0C8CC99E06916710409F496
:10823000D8C0AAE06A16710409F09CCCC555DF4F7E
:108240008881CB5AD04082958F70823009F01CC152
:10825000C255DF4F6881CE5AD040060F111D17FF5F
:1082600002C010E000E00536110514F004E610E04D
:10827000C255DF4F0883CE5AD04062E0CE01875509
:108280009F4F0E94EA0F2A962FAF2A972B963FAF57
:108290002B972C964FAF2C972D965FAF2D972E9640
:1082A0006FAF2E972F967FAF2F9760968FAF609707
:1082B00061969FAF619716CFC12CB6CCC355DF4FE7
:1082C0006881CD5AD040060F111D17FF02C010E083
:1082D00000E00F3F110519F014F00FEF10E0C35547
:1082E000DF4F0883CD5AD040A12C5AE0B52ED12CB7
:1082F00033243A94ADCDC355DF4F68817981CD5A8F
:10830000D040060F171F17FF02C010E000E005362F
:10831000110514F004E610E0012E000C220B330BC3
:10832000C355DF4F088319832A833B83CD5AD0403E
:10833000DBCFC355DF4F688179818A819B81CD5A1C
:10834000D0400E9408C0600F711F77FF02C070E02C
:1083500060E06536710514F064E670E0072E000CED
:10836000880B990B0E943DBDC355DF4F688379830D
:108370008A839B83CD5AD040B7CFC355DF4F288126
:108380003981CD5AD0404AE0409FC001419F900DB5
:108390001124820F931F97FF02C090E080E0893E76
:1083A000B3E09B0714F088EE93E0092E000CAA0BB3
:1083B000BB0BC355DF4F88839983AA83BB83CD5AF8
:1083C000D04092CF88E0FE013196DE01A755BF4F25
:1083D00001900D928A95E1F7B12CA12CDD24D39464
:1083E00087CFC555DF4F8881CB5AD04082958F709B
:1083F000823009F049C0C155DF4F6881CF5AD04063
:10840000C055DF4F8881C05BD040782F7170060F58
:10841000171F0E36E1E01E072CF417FF05C00DE60E
:1084200011E002C010E000E0C155DF4F0883CF5AD1
:10843000D040C055DF4F8881C05BD04010FB80F931
:10844000C055DF4F8883C05BD04062E0CE018755C6
:108450009F4F0E94EA0F62962FAF629763963FAFDD
:10846000639764964FAF649765965FAF659766961E
:108470006FAF669767967FAF679768968FAF68977D
:1084800069969FAF69972ECE88E0FE013196DE0196
:10849000A755BF4F01900D928A95E1F7E6CD0FEFFA
:1084A0001FEFFFCC863009F47CC0873009F006CD81
:1084B000C4010E949E1EF82E96E0891361C067E2F7
:1084C00078E085E99DE00E94CA7866E070E085E981
:1084D0009DE00E94258B85E99DE00E94C17762E0C6
:1084E000CE0187559F4F0E94111029AF3AAF4BAF75
:1084F0005CAF6DAF7EAF8FAF21969FAF21973CC031
:10850000C4010E949E1E853019F00DEF1FEFA5CA11
:1085100068E378E085E99DE00E94CA7865E070E054
:1085200085E99DE00E94258B85E99DE00E94C17749
:10853000B401CE0187559F4F0E94588E61E0CE0155
:1085400087559F4F0E94111022962FAF2297239696
:108550003FAF239724964FAF249725965FAF25977B
:1085600026966FAF269727967FAF279728968FAFCF
:10857000289729969FAF29976894A0F8B0F89ECCC9
:108580006FE078E085E99DE00E94CA786F2D70E089
:1085900085E99DE00E94258B85E99DE00E94C177D9
:1085A000B4CFC4010E945D4A1816190674F1B401D3
:1085B000CE0187559F4F0E94588E61E0CE018755AE
:1085C0009F4F0E94111029AB3AAB4BAB5CAB6DAB2C
:1085D0007EAB8FAB98AF6894A0F8B0F846E0342E2D
:1085E000C755DF4F8881C95AD040811132C0689485
:1085F000A0F8C555DF4F8881CB5AD040807F69F104
:108600006894B1F8D11017C220C26BEF77E085E90A
:108610009DE00E94CA7879CFC4010E945D4A181675
:108620001906A4F462E0CE0187559F4F0E941110F5
:1086300029A73AA74BA75CA76DA77EA78FA798ABE2
:108640006894A0F8B0F835E0332ECACF64EE77E036
:10865000DECF6894A0F8B0F8CCCF40E052E0B4018F
:10866000CE0187559F4F0E94DA3A8111C9CFCACFF8
:10867000AFEF3A12B1C0C4010E945D4A3324339473
:10868000181619060CF4ABC0312C6CED77E085E9B7
:108690009DE00E94CA78E32C032C000CFF08CD5407
:1086A000DF4FF982E882C35BD040B70185E99DE0E6
:1086B0000E94258B65ED77E085E99DE00E94CA78F0
:1086C0006C2D70E085E99DE00E94258B85E99DE099
:1086D0000E94C177CF54DF4F48805980C15BD040A2
:1086E0004114510409F484C06DE479E0C2010E9490
:1086F000D6B501E010E0892B09F44BC069E479E0BC
:10870000C2010E94D6B502E010E0892B09F441C0F5
:1087100063E277E0C2010E94D6B505E010E0892B44
:10872000C1F16FE177E0C2010E94D6B506E010E02A
:10873000892B79F16EE079E0C2010E94D6B50AE09A
:1087400010E0892B31F169E079E0C2010E94D6B5D1
:108750000BE010E0892BE9F063E179E0C2010E94AF
:10876000D6B50CE010E0892BA1F066E177E0C201FC
:108770000E94D6B50DE010E0892B59F062E177E058
:10878000C2010E94D6B510E000E0892B11F40EE082
:1087900010E0C4010E949E1EE82EF12CE114F104A9
:1087A00031F4CD54DF4FE880F980C35BD040011530
:1087B000110509F436C0E016F106A1F06FEB77E081
:1087C00085E99DE00E94CA78B70185E99DE00E9495
:1087D000258B85E99DE01EC3332009F456CFCC24B8
:1087E000C39453CFCF54DF4F19821882C15BD0405E
:1087F000C755DF4FE881C95AD040EA3008F00CC1B4
:10880000F0E08827E95FFB4B8F4F0C940BBF1945B5
:10881000FC44F5444A441945DC44B9448C441945A8
:108820001945D40119968D919C91009709F413C9AB
:10883000DC01ED91FC910488F589E02D7201C755AA
:10884000DF4F0881C95AD040C655DF4F1881CA5A38
:10885000D040C555DF4F2881CB5AD040C455DF4F9B
:108860003881CC5AD040C355DF4F4881CD5AD040D3
:10887000C255DF4F5881CE5AD040C155DF4F688175
:10888000CF5AD040C055DF4F7881C05BD04019959A
:108890008C01E3C8C4010E949E1E853009F035CECC
:1088A00060EB77E085E99DE00E94CA7865E070E0C2
:1088B00085E99DE00E94258B85E99DE00E94C177B6
:1088C000B401CE0187559F4F0E94588EF4018085D8
:1088D000853099F46CE0CE0187559F4F0E941110AE
:1088E00029A33AA34BA35CA36DA37EA38FA398A750
:1088F0006894A0F8B0F8312C57C061E0CE018755DC
:108900009F4F0E941110298F3A8F4B8F5C8F6D8F74
:108910007E8F8F8F98A3ECCFC4010E949E1E182FCC
:108920008630F9F46FE977E085E99DE00E94CA7826
:1089300066E070E085E99DE00E94258B85E99DE079
:108940000E94C17762E0CE0187559F4F0E941110AF
:10895000298B3A8B4B8B5C8B6D8B7E8B8F8B988F9F
:10896000C7CF67E877E085E99DE00E94CA78612F6C
:108970000ECE31101EC0B401CE0187559F4F0E940C
:10898000588E61E0CE0187559F4F0E9411102987B4
:108990003A874B875C876D877E878F87988B689433
:1089A000A0F8B0F826E0322E0FEF1FEFCC24C394CE
:1089B00029CE63E777E02BCE3320A1F062E0CE0131
:1089C00087559F4F0E94111029833A834B835C8304
:1089D0006D837E838F8398876894A0F8B0F895E0C4
:1089E000392EE2CF6CE577E012CEC4010E949E1EC4
:1089F000853009F07DCF89CD332019F069E477E027
:108A000006CEB401CE0187559F4F0E94588E6894C0
:108A1000A0F8F3E0BF2A6FCFC555DF4F8881CB5A4E
:108A2000D040807F19F46894B0F865CF23E0B22A73
:108A300062CFDD2021F00CEF1FEF0C942D3D312C87
:108A40000FEF1FEFA114B10439F0A501B401CE015D
:108A500087559F4F0E946D3AD40119968D919C9134
:108A6000009709F474C0CF54DF4FE880F980C15BF0
:108A7000D040DC01ED91FC910488F589E02DC755CB
:108A8000DF4F0881C95AD040C655DF4F1881CA5AF6
:108A9000D040C555DF4F2881CB5AD040C455DF4F59
:108AA0003881CC5AD040C355DF4F4881CD5AD04091
:108AB000C255DF4F5881CE5AD040C155DF4F688133
:108AC000CF5AD040C055DF4F7881C05BD040199558
:108AD0008C01332021F0632DC4010E94881DC954EC
:108AE000DF4FE881F981C75BD040359721F0B501B0
:108AF000C4010E94BB3B6FE277E085E99DE00E94E4
:108B0000CA78B80185E99DE00E94258B68E277E08C
:108B100085E99DE00E94CA780E94B095AB01BC0136
:108B2000C754DF4FC880D980EA80FB80C95BD04042
:108B30004C195D096E097F092AE085E99DE00E94D4
:108B4000757785E99DE00E94C1770C942D3DF40175
:108B50008085853009F464C0863009F0BACF70E0B2
:108B600060E0C4010E94A91C7C01009709F4B1CF08
:108B7000712C612C97FF06C0F194E194F1086624F2
:108B80006394712CC70101978635910508F0A1CF38
:108B9000C755DF4F0881C95AD04010E0DE2C61E094
:108BA0008E2D0E945093672859F10130110521F054
:108BB00061E00C30110509F460E0062F10E08D2D06
:108BC0000E94229364E477E085E99DE00E94CA78E0
:108BD000B70185E99DE00E94258B62E477E085E995
:108BE0009DE00E94CA78B80185E99DE00E94258B2E
:108BF00085E99DE00E94C1776894A0F8B0F86FC045
:108C00000130110551F091E080E00C30110509F0C0
:108C100090E0092F182F602FD2CF01E010E0FBCF9A
:108C2000F2E06F16710409F45DC02CE06216710465
:108C300029F06A94672809F04CCFDECFC4010E9466
:108C40008D1C892B49F4D401ED91FC9160817181D7
:108C50008CE795E00E949996CE0187559F4F0E9420
:108C6000351120E030E048EC52E40E949CBD0E94A7
:108C700008C02B0188E00E94FE15CD54DF4F6883A9
:108C800079838A839B83C35BD040CD54DF4FE880D8
:108C9000F980C35BD0406EE377E085E99DE00E94F8
:108CA000CA78B20185E99DE00E94258B69E377E0EF
:108CB00085E99DE00E94CA78CD54DF4F68817981B3
:108CC000C35BD04085E99DE00E94F78D85E99DE07A
:108CD0000E94C177B701A201C4010E94792401E07A
:108CE00010E0F7CE6894A0F8B1F8F9CF0E947C119B
:108CF000672B682B692B09F072C9B12CA12CA0C974
:108D00006114710409F045C08081882311F40C942A
:108D1000B53CCE018F549F4F0E94D9243C01C555CC
:108D2000DF4F8881CB5AD0408F7071F5662DCE0110
:108D300087559F4F0E94EA0FCF55DF4F2883C15AB6
:108D4000D040CE55DF4F3883C25AD040CD55DF4F8B
:108D50004883C35AD040CC55DF4F5883C45AD040C3
:108D6000CB55DF4F6883C55AD040CA55DF4F788353
:108D7000C65AD040C955DF4F8883C75AD040C8551E
:108D8000DF4F9883C85AD0406114710411F40C94D9
:108D9000B53C0E94520F6B018B0163E878E085E9D6
:108DA0009DE00E94CA78B60185E99DE00E94258B6E
:108DB0006CE778E085E99DE00E94CA78D401ED91E6
:108DC000FC916081718185E99DE00E94647866E78D
:108DD00078E085E99DE00E94CA78CF54DF4F688132
:108DE0007981C15BD04085E99DE00E94647860E7AD
:108DF00078E085E99DE00E94CA78083C110514F0EE
:108E00000C94F63C62E678E08EEE9CE00E94CA7814
:108E10008EEE9CE00E94C1770FEF1FEF0C942D3D6A
:108E20002F923F924F925F926F927F928F929F927A
:108E3000AF92BF92CF92DF92EF92FF920F931F9368
:108E4000CF93DF93CDB7DEB7A5970FB6F894DEBF0B
:108E50000FBECDBF5C0179A368A370905C0777203B
:108E600009F4B8C080910C098F5F80930C09E091E0
:108E70001009F0911109309709F4A4C086809780F9
:108E800040901009509011094114510409F496C002
:108E90008114910409F492C0D40118968C918F70BA
:108EA000853091F7C4010E942D8B823068F3B401A4
:108EB000CE0101960E947E22CE0101960E943612BA
:108EC000882309F45EC060E074E0CE0101960E9440
:108ED000721D892B09F455C0188E198E1A8E1B8E9F
:108EE0001C8E1D8E1E8E1F8E8A8D8F708A8F40E085
:108EF00053E0BE016F5F7F4FCE0148960E94DA3A81
:108F000067EC78E085E99DE00E94CA7860E074E053
:108F1000CE0101960E942A1D8A859B85009789F1C2
:108F2000DC01ED91FC910488F589E02DCC24C394FB
:108F3000F12CE12C088D198D2A8D3B8D4C8D5D8D8A
:108F40006E8D7F8D19958F3F9807D9F0E981FA8151
:108F500060817181892BE9F485E99DE00E94647844
:108F600065EC78E085E99DE00E94CA786DEB78E0D9
:108F700085E99DE00E94CA7885E99DE00E94C1775D
:108F8000712CF40182809380CE0101960E945D12C3
:108F900077CF85E99DE00E9464786BEB78E085E906
:108FA0009DE00E94CA7867EB78E085E99DE00E9429
:108FB000CA7885E99DE00E94C177E3CF85E99DE00D
:108FC0000E94C17780910C09815080930C09711027
:108FD00010925C0765E0D5018D919C910E94188BE1
:108FE0001C01009709F48FC0FC018084859485944E
:108FF0008594859441845284638474840E94B095DE
:10900000882009F480C0461A570A680A790A188E1F
:10901000198E1A8E1B8E888E8A8D8F70806A982E7C
:109020008A8F4C8E5D8E6E8E7F8EC301B20128EECC
:1090300033E040E050E00E94A2BE2AA33BA34CA331
:109040005DA3672B682B692B21F5D12CC12CE12C5A
:1090500090E1F92E082D198D292D3B8D4C8D5D8DBC
:109060006E8D7F8DC5010E940B382AE030E04AA149
:109070005BA16CA17DA185E99DE00E94DE776CED8E
:1090800078E085E99DE00E94CA7885E99DE00E942C
:10909000C17777FE38C0F2E04F1651046104F0E862
:1090A0007F068CF1D12CC12CE12C80E1F82E088DAB
:1090B000198D2A8D3B8D4C8D5D8D6E8D7F8DC501FB
:1090C0000E940B3819821A821B821C821D821E820A
:1090D0001F8218862B812F702B838982CC24C39406
:1090E000F12CE12C082D1A813C8140E05E816F81DA
:1090F0007885C5010E94273CD10118968C9118975C
:109100008F7018968C93E8A1F9A13197B9F460E0BB
:1091100073E0C5010E94721D009781F020910E0935
:1091200030910F092630310549F4BC01C5010E9478
:10913000BB3B60E073E0C5010E942A1DD501199672
:109140008D919C910097D9F490E080E0A5960FB6A0
:10915000F894DEBF0FBECDBFDF91CF911F910F916D
:10916000FF90EF90DF90CF90BF90AF909F908F9047
:109170007F906F905F904F903F902F900895DC010B
:10918000ED91FC910484F585E02D1995892BE1F290
:10919000F50181859285DC01ED91FC910480F581DA
:1091A000E02D68A179A11995D1CFAF92BF92CF924E
:1091B000DF92EF92FF920F931F93CF93DF93CDB780
:1091C000DEB767970FB6F894DEBF0FBECDBFE09154
:1091D0001009F0911109309709F49EC080910C0993
:1091E0008F5F80930C0906811781E0901009F09041
:1091F0001109E114F10431F10115110519F1F8011A
:1092000080858F708530A9F7C8010E942D8B823030
:1092100080F3B801CE0101960E947E22CE01019614
:109220000E943612882331F062E070E0CE01019690
:109230000E941047F80102811381CE0101960E941D
:109240005D12D3CF80910C09815080930C098091DD
:109250000E0990910F09059709F45EC00E94B09520
:109260009B01AC0160916607709167078091680768
:1092700090916907AA24AA94BA2C650118EEE12EF0
:1092800013E0F12E00E010E00E94472A082F882307
:1092900009F442C010E0609176077091770761157C
:1092A0007105D1F1111138C0FB0180858F708530B7
:1092B000D9F4CE0101960E947E2261E070E0CE01D9
:1092C00001960E941047892B59F00E94B095609337
:1092D0006607709367078093680790936907102F5C
:1092E000CE0101960E945D12E0917607F09177071A
:1092F000309791F0828193819093770780937607DE
:10930000892B49F6E0911009F09111098681978126
:10931000909377078093760767960FB6F894DEBF31
:109320000FBECDBFDF91CF911F910F91FF90EF90B6
:10933000DF90CF90BF90AF9008954F925F926F9261
:109340007F928F929F92AF92BF92CF92EF92FF92B5
:109350000F931F93CF93DF93CDB7DEB767970FB609
:10936000F894DEBF0FBECDBF009709F4A4C0FC0186
:1093700020852F70253009F09EC02A015B01868070
:10938000978080910C098F5F80930C098114910460
:1093900009F48CC0F40180858F70843009F082C09C
:1093A0006185728580911009909111090E949C8AB3
:1093B0003C01009709F476C0FC0180858F708530F0
:1093C00009F070C0B301CE0101960E947E22A11463
:1093D000B104A9F0CE0101960E943612882379F0DB
:1093E000C12C7201F50100811181228133814481F8
:1093F000558166817781CE0101960E94273C60E00D
:10940000C3010E94188B0097D1F1FC0120852F70B9
:109410002230A9F581859285A385B4850797A1059A
:10942000B10569F561E0C3010E94188BA201B50185
:109430000E949D49A114B10489F5882379F1809196
:109440000C09815080930C09CE0101960E945D1297
:1094500081E067960FB6F894DEBF0FBECDBFDF91F7
:10946000CF911F910F91FF90EF90CF90BF90AF9051
:109470009F908F907F906F905F904F900895A11470
:10948000B10461F4CE0101960E943612882331F0B6
:10949000CE0101960E945D4A892B89F6CE01019684
:1094A0000E945D12F4018280938070CF80910C093C
:1094B000815080930C0980E0CCCFFF920F931F93D3
:1094C000CF93DF9300D000D01F921F92CDB7DEB7AD
:1094D0008C0119821A821B821C821D821E821F82AD
:1094E00018868B818F708B83D801ED91FC91608100
:1094F000718185E99DE00E94647865EB78E085E9FB
:109500009DE00E94CA78C8010E943612811119C0DC
:109510006CEA78E085E99DE00E94CA7885E99DE0E3
:109520000E94C1770FEF1FEFC80128960FB6F8947D
:10953000DEBF0FBECDBFDF91CF911F910F91FF9086
:109540000895C8010E949E1EF8019085973039F059
:10955000853049F1D0F48130E9F0823021F1D80131
:1095600019968D919C91009721F1DC01ED91FC9170
:109570000688F789E02D199501E0892B09F400E0B0
:10958000802F0E94561610E0CFCF863019F08A50F7
:10959000833028F76DE878E085E99DE00E94CA787D
:1095A00001E010E0C1CF80E00E94561610E000E01C
:1095B000BBCF40E052E0B801CE0101960E94DA3AFA
:1095C000F8018085873079F160F4833009F452C066
:1095D000843061F06DE978E085E99DE00E94CA7809
:1095E000E5CF883009F446C08930A1F760E0CE01AC
:1095F00001960E9468108C0162E978E085E99DE09F
:109600000E94CA78B80185E99DE00E94258B85E912
:109610009DE00E94C17791E080E0012B09F490E089
:10962000092F182F81CF0280F381E02D80858F7064
:10963000853031F56AEA78E085E99DE00E94CA78D4
:1096400050E040E070E060E0F801828193810E9488
:109650009D49F82E082F10E067EA78E085E99DE043
:109660000E94CA788F2D0E94561685E99DE00E94BF
:10967000C1775ACFCE0101960E947C118B01BCCFDD
:1096800010E000E0B9CF2F923F924F925F926F921D
:109690007F928F929F92AF92BF92CF92DF92EF9282
:1096A000FF920F931F93CF93DF93CDB7DEB7C955CA
:1096B000D1090FB6F894DEBF0FBECDBF0E94B095A2
:1096C0009B01AC0160916E0770916F0780917007EC
:1096D00090917107AA24AA94BA2C650110E3E12E97
:1096E00015E7F12E00E010E00E94472A882309F4D4
:1096F000FEC1E0911009F0911109309709F4F7C10A
:1097000080910C098F5F80930C092680378010E0D0
:109710002114310409F431C1F10180858F70853045
:10972000F9F460E0C1010E94188BFC0181859285EB
:10973000A385B4850597A105B10591F4B101CE01CA
:1097400001960E947E22CE0101960E9436126696F4
:109750008FAF6697811108C0CE0101960E945D12FD
:10976000F10122803380D4CF25961CAE1DAE1EAEF3
:109770001FAE259729961CAE1DAE1EAE1FAE2997B3
:1097800040E052E0BE016F5F7F4FCE018F5B9F4F85
:109790000E94DA3ACE0101960E948D1C6B017C0179
:1097A00069966FAF69976A96DFAE6A9770E060E07E
:1097B000CE0101960E94A91C4C01CE018F5B9F4FE8
:1097C0000E94351165966CAF7DAF8EAF9FAF6597E8
:1097D000CE0101960E949E1E182FB601DD0C880B4B
:1097E000990B0E943DBD20E030E048EC52E40E941D
:1097F00096BF2B013C01CE0101960E945D4A6896FE
:109800009FAF8EAF689769E972E185E99DE00E949C
:10981000CA7865966CAD7DAD8EAD9FAD65970E94A3
:10982000EB8E63E972E185E99DE00E94CA78C3018D
:10983000B2010E94EB8E6DE872E185E99DE00E9425
:10984000CA78612F70E085E99DE00E94258BE114C4
:10985000F10409F48BC088E00E94FE159B01AC0165
:1098600044275527B70190E080E0AA24AA94BA2C97
:10987000C12CD12C17E2E12E19E0F12E00E010E00E
:109880000E94472A882319F1F101608171818EEECF
:109890009CE00E9464786DE772E18EEE9CE00E948D
:1098A000CA78F101608171818BE895E00E949996F8
:1098B00090E080E0BC0169964FAD69976A965FAD14
:1098C0006A97CE0101960E94792460E02CC020E0C6
:1098D00030E048E152E4C301B2010E943EC01816D4
:1098E0003CF4F1016081718187E995E00E949996CD
:1098F00068968EAD9FAD6897892B39F320E030E0F4
:1099000040E85FE365966CAD7DAD8EAD9FAD65972C
:109910000E9429BF9B01AC01C301B2010E9436BD68
:1099200087FF0CC061E0C4010E94AB1ECE0101960E
:109930000E945D1266961FAD669712CFA301920139
:1099400065966CAD7DAD8EAD9FAD65970E9436BDC1
:1099500018160CF0BACF6EE672E185E99DE00E9420
:10996000CA7885E99DE00E94C177E0CF64E672E1A4
:1099700085E99DE00E94CA78D9CF80910C09815079
:1099800080930C090E94B09560936E0770936F07E7
:1099900080937007909371070E94520F2B013C0136
:1099A0000E94B0956B017C010E94B78A882309F45C
:1099B00066C080919A08811162C030E020E041E0E9
:1099C00050E060E4CE0101960E94382D40E450E062
:1099D00066E477E1CE0101960E94EFB56BE575E094
:1099E000CE0101960E944EC340E450E06BE372E169
:1099F000CE0101960E94EFB5B301A201CE018F5BAB
:109A00009F4F0E94BD0EBE016F5B7F4FCE0101963E
:109A10000E947E9630E020E041E050E060E4CE011C
:109A200001960E94382D40E450E066E477E1CE01D3
:109A300001960E94EFB56BE575E0CE0101960E949C
:109A40004EC340E450E064E372E1CE0101960E940F
:109A5000EFB5C701B60128EE33E040E050E00E94C8
:109A600080BEBA01A901CE018F5B9F4F0E94BD0E3F
:109A7000BE016F5B7F4FCE0101960E947E9611233F
:109A800009F44FC06EE572E185E99DE00E94CA7855
:109A90000E94520FAB01BC012AE085E99DE00E94C3
:109AA000757766E572E185E99DE00E94CA7860916C
:109AB0000C09062E000C770B85E99DE00E94258B92
:109AC00064E472E185E99DE00E94CA7840916A07EA
:109AD00050916B0760916C0770916D072AE085E9E2
:109AE0009DE00E94757785E99DE00E94C177C75A85
:109AF000DF4F0FB6F894DEBF0FBECDBFDF91CF9121
:109B00001F910F91FF90EF90DF90CF90BF90AF909B
:109B10009F908F907F906F905F904F903F902F908D
:109B2000089564E572E185E99DE00E94CA780E948B
:109B3000520FAB01BC012AE085E99DE00E947577D8
:109B40006CE472E1B0CF6F927F929F92AF92BF921E
:109B5000CF92DF92EF92FF920F931F93CF93DF93F9
:109B6000CDB7DEB7E2970FB6F894DEBF0FBECDBF1C
:109B700078AB6FA75AAB49AB672B09F480C2FA01E7
:109B8000309719F02081211109C0FC01238522237F
:109B900029F09C01255F3F4F3AAB29AB5C01E9A955
:109BA000FAA93097E1F4F501E588F688E114F104AB
:109BB00001F510E000E0CFA4D8A83601600E711EB8
:109BC000F3018081882309F458C0082E000C990BFA
:109BD0000E94F1C2F30180830F5F1F4FECCF8081A1
:109BE000882309F3CE01C1960E94D9247C01892BD8
:109BF000D1F2FEE0EF16F104E1F62FA538A91982A3
:109C00001A821B821C821D821E821F8218868B81F3
:109C10008F70806C8B833E832D836EE0CE01019626
:109C20000E94EA0F29A33AA34BA35CA36DA37EA3D2
:109C30008FA398A7E9A8FAA8CC24C39409811A8114
:109C40002B813C814D815E816F817885C5010E94A9
:109C5000273CE2960FB6F894DEBF0FBECDBFDF9172
:109C6000CF911F910F91FF90EF90DF90CF90BF9019
:109C7000AF909F907F906F900895C114D10481F1AF
:109C8000F6018081882361F18D3209F46DC090ED79
:109C9000980F9A3008F468C008E010E0853211F19E
:109CA0000EEF1FEF8B37F1F007E110E08332D1F0B8
:109CB00097EF692E99E0792E01E010E0C3010E9430
:109CC000E6B5AC01B301C6010E94FFB5892B51F086
:109CD0000F5F1F4FF9E06F0E711C0931110571F70D
:109CE0000FEF1FEF19A21AA21BA21CA21DA21EA2F7
:109CF0001FA218A68BA18F708BA309A385E0E8167D
:109D0000F104A9F1E6E0EE16F10411F407E110E028
:109D10009E2C6E2DCE0181960E94EA0F298F3A8FDC
:109D20004B8F5C8F6D8F7E8F8F8F98A301151105E0
:109D3000A9F104F50E3F1F4F0CF0A1C1CE018F9683
:109D40000E946016092E000CAA0BBB0B0097A10500
:109D5000B10509F4D2C02BA12F70206A2BA38DA3CB
:109D60009EA3AFA3B8A7C9C010E000E0BBCF08E135
:109D700010E0CECF0731110509F43DC108311105BE
:109D8000E9F660E0CE0181960E941110298B3A8B92
:109D90004B8B5C8B6D8B7E8B8F8B988F19821A828D
:109DA0001B821C828B818F7080668B83EFA5F8A944
:109DB000309709F48AC08081882309F486C06FA493
:109DC00078A8F3018081882359F08D3249F08053BF
:109DD0008A3030F0FFEF6F1A7F0A78AA6FA6EFCFB4
:109DE000C3010E9475B56C016EE270E0C3010E9470
:109DF00059C3009771F0FC010181002E000C110B7A
:109E0000005311090A30110514F009E010E017FFA2
:109E100002C010E000E06CE270E0C3010E9459C390
:109E2000009709F045C018AA1FA60115110509F4ED
:109E300043C02AE02C9DC0012D9D900D11241C14BF
:109E40001D041CF0119501951109080F191F012E11
:109E5000000C220B330B0D831E832F833887692D53
:109E6000CE0101960E94EA0F29873A874B875C87CB
:109E70006D877E878F87988BDB80D2948FE0D82286
:109E80003E01F9E26F0E711C10E000E08FA598A969
:109E9000892BF9F003301105E1F00F5F1F4FCE0160
:109EA0008F960E946016F301819391933F01EECF4C
:109EB000019698AB8FA7B9CF8601DD0C220B330B2F
:109EC0008B818F70806A8B83C6CF00E010E0980191
:109ED000C2CFFAE0EF16F104E9F08BE0E816F104E6
:109EE00069F1E9E0EE16F10491F5CE0101960E94C8
:109EF0007C11CE0181960E941712E9A8FAA8CC2401
:109F0000C39409A11AA12BA13CA14DA15EA16FA1EF
:109F100078A59CCECE0101960E947C118BA1982F32
:109F200092959F7039F0923041F7653608F064E6FB
:109F30006EA3E3CF8F7080628BA3F7CFCE01019623
:109F40000E947C11CE0181960E94E311D6CF81E060
:109F500090E0D11002C090E080E0800F911F82302D
:109F6000910539F164F4019741F688E0FE013196DC
:109F7000DE01919601900D928A95E1F7BECF833074
:109F8000910539F1049709F0B8CF1BA509A5CE01B9
:109F900001960E947C118BA18F7080628BA36FA3AE
:109FA00088A570FB80F988A70EA31DA36DA57EA5CB
:109FB000C9CF19A5CE0101960E947C118BA18F708B
:109FC00080638BA36FA388A570FB80F988A71EA36D
:109FD00094CF1BA509A5CE0101960E947C118BA1EF
:109FE0008F7080628BA36FA388A570FB80F988A710
:109FF0000EA31DA382CF60E0CE0181960E941110B6
:10A0000029833A834B835C836D837E838F83988718
:10A010007E01F9E0EF0EF11C10E000E08FA598A999
:10A02000892B71F00430110591F00F5F1F4FCE01A5
:10A030008F960E946016F701819391937F01EECF76
:10A040000330110589F00430110509F056CF9F85C2
:10A050002D853B8549858BA18F7080658BA34FA390
:10A060003EA32DA398A749CF9D852B8539858BA12C
:10A070008F7080648BA33FA32EA39DA33ECF90E05F
:10A0800080E0E7CD2F923F924F925F926F927F9246
:10A090008F929F92AF92BF92CF92DF92EF92FF92F8
:10A0A0000F931F93CF93DF93CDB7DEB7C955D10977
:10A0B0000FB6F894DEBF0FBECDBF3C01562E6296A0
:10A0C000EFAE62976396FFAE639764960FAF6497A7
:10A0D00065961FAF659766962FAF669767963FAFF9
:10A0E000679768964FAF689769965FAF69976A966A
:10A0F000CFAE6A972D2C4A2C3B2C009709F45EC1F9
:10A10000FC0180858295807F8595859585958595CF
:10A11000843009F43EC12CF4882309F443C180E063
:10A120002DC0853009F444C08630C9F764EA75E073
:10A13000C3010E949C8A4C01009709F46FC0B12CA6
:10A14000A12CD12CC12C6296EFAC62976396FFAC28
:10A15000639764960FAD649765961FAD6597669695
:10A160002FAD669767963FAD679768964FAD689736
:10A1700069965FAD6997652D0E944250C75ADF4FBF
:10A180000FB6F894DEBF0FBECDBFDF91CF911F9108
:10A190000F91FF90EF90DF90CF90BF90AF909F9086
:10A1A0008F907F906F905F904F903F902F90089589
:10A1B00080910C098F5F80930C09868097808114B1
:10A1C000910431F1A42CB32C6A96CFAC6A97D22CAF
:10A1D0006296EFAC62976396FFAC639764960FAD9F
:10A1E000649765961FAD659766962FAD66976796DF
:10A1F0003FAD679768964FAD689769965FAD699771
:10A20000652DC4010E944250F40182809380D7CF13
:10A2100080910C09815080930C0981CF68EA75E028
:10A22000C3010E949C8A7C016DEA75E0C3010E9413
:10A230009C8A6C01552039F0F1E05F1609F48AC060
:10A2400010E000E00CC062EB75E0C3010E949C8A44
:10A250004C0167EB75E0C3010E949C8A8C0181145C
:10A26000910409F443010115110509F48301E11476
:10A27000F10421F46A96EFAC6A97F22CC114D10470
:10A2800011F4C42CD32C8114910409F494C0F4016A
:10A2900080858F70843009F08EC08184928401158E
:10A2A000110509F493C0F80180858F70843009F09E
:10A2B0008DC001851285E114F10409F4CBC081142D
:10A2C000910409F492C06EE875E185E99DE00E9471
:10A2D000CA78F7016185728585E99DE00E946478FE
:10A2E00069E875E185E99DE00E94CA78B40185E9D5
:10A2F0009DE00E94647885E99DE00E94C177CE01CF
:10A300008F5A9F4F0E94BC31C114D10409F0FAC08A
:10A31000F70180858F70843009F0F2C06185728505
:10A32000CE0101960E940D25CE0101960E943612A3
:10A33000882359F08114910409F46BC050E040E087
:10A34000B401CE0101960E94A34DCE0101960E9458
:10A350005D12D6C06CEB75E0C3010E949C8A4C0173
:10A3600061EC75E0C3010E949C8A8C018114910408
:10A3700009F0CDC062EB75E0C3010E949C8A4C01DC
:10A380000115110509F465CF892B09F070CF430140
:10A390006ECF10E000E0912C812CD12CC12CF12C3F
:10A3A000E12C5DCF10E000E0912C812CD12CC12C50
:10A3B000F12CE12C5CCF912C812C71CFCA2CDB2CA1
:10A3C0006A96EFAC6A97F22C912C812C00E020E089
:10A3D00033E040E150E0BE016F5B7F4FCE018F5A0A
:10A3E0009F4F0E94B61F8C0166CF6FE775E185E92C
:10A3F0009DE00E94CA78F7016185728585E99DE03C
:10A400000E9464786AE775E185E99DE00E94CA7858
:10A4100076CFCC24C394F12CE12C62960FAD6297D9
:10A4200063961FAD639764962FAD649765963FADB5
:10A43000659766964FAD669767965FAD6797689626
:10A440006FAD689769967FAD6997CE0101960E94BE
:10A45000273C7BCFC114D10409F452C0011511056A
:10A4600009F44EC0F60180858F70843009F044C035
:10A4700063E775E185E99DE00E94CA78F601618590
:10A48000728585E99DE00E9464786EE675E185E954
:10A490009DE00E94CA78B80185E99DE00E94647839
:10A4A00085E99DE00E94C177F6016185728540E4EF
:10A4B00050E0CE0101960E9492C30E94B78A882381
:10A4C000D9F080919A08811117C06FE270E0CE0137
:10A4D00001960E9459C3892B51F4F60121853285DA
:10A4E00043E050E060E4CE0101960E94382DB801AF
:10A4F000CE0101960E947E96E114F10409F008CF86
:10A5000081E03CCE0115110509F0ACCF01CF892BBC
:10A5100009F0ADCE9ECE2F923F924F925F926F92F6
:10A520007F928F929F92AF92BF92CF92DF92EF92E3
:10A53000FF920F931F93CF93DF93CDB7DEB7E297D0
:10A540000FB6F894DEBF0FBECDBF9AA389A3098FC3
:10A550001A8F2B8F3C8F4D8F5E8F6F8F78A3FAAA47
:10A56000E9AADC011496ED91FC91309709F4D8C06A
:10A570006680778018AA1FA61AA619A6312C212C4E
:10A58000912C812C512C412C6114710409F4D0C000
:10A5900060E974E0C3010E949C8A5C0165E974E093
:10A5A000C3010E949C8A9EA38DA3A114B10409F447
:10A5B000AFC0892B09F4ACC0F50180858F70823063
:10A5C00009F0A6C0ADA1BEA118968C918F70823003
:10A5D00009F09EC066EC75E0C3010E949C8ADC0114
:10A5E00019962D913D914D915C911C972BA73CA7FD
:10A5F0004DA75EA7E9A9FAA9309709F459C0D3017C
:10A60000CD90DC90BF01C6010E9464C3892B09F084
:10A610004FC0098D002309F1802F90E0B0E0A0E049
:10A62000EDA1FEA181879287A387B48780910E094F
:10A6300090910F09059789F0E12CFF24F3941A8D6E
:10A640002B8D3C8D4D8D5E8D6F8D78A1A9A1BAA10A
:10A6500012968D919C910E940B388B8D807F41F1D9
:10A6600060E0CE0149960E946810092E000CAA0BEA
:10A67000BB0BF50181879287A387B48780910E0970
:10A6800090910F090597A1F0D301CD90DC90E12CBA
:10A6900092E0F92E098D1A8D2B8D3C8D4D8D5E8D9E
:10A6A0006F8D78A1E9A1FAA1828193810E940B3874
:10A6B000D50119964D915D916D917C911C97EDA1FD
:10A6C000FEA181859285A385B4850297A105B10578
:10A6D00021F12BA53CA5429FC001439F900D529FA5
:10A6E000900D1124480E591EABA5BCA58A0E9B1EC9
:10A6F000EFA5F8A98F01FF0F220B330B04171507E5
:10A70000260737072CF458AB4FA79AA789A71D0136
:10A71000D30112966D907C9037CF90E080E0E4CF2B
:10A720001AA619A6312C212C912C812C512C412CAC
:10A730008114910409F486C0C201B4010E94F7BEDD
:10A740007B0161E075E185E99DE00E94CA78B40172
:10A7500085E99DE00E94258B66EF74E185E99DE027
:10A760000E94CA780FEF10E0C201B8010E94F7BE44
:10A7700085E99DE00E94258B6FEE74E185E99DE0FF
:10A780000E94CA78B70185E99DE00E94258B61EEA1
:10A7900074E185E99DE00E94CA7889A59AA5B8016F
:10A7A0000E94F7BE85E99DE00E94258B6AED74E169
:10A7B00085E99DE00E94CA78B10185E99DE00E948B
:10A7C000258B66ED74E185E99DE00E94CA7885E9F4
:10A7D0009DE00E94C17719821A821B821C821D8211
:10A7E0001E821F8218868B818F708B83B701CE01EA
:10A7F00001960E94331079018A013B014C01298B9B
:10A80000FA8A4B8B1C8B6D8B7E8A8F8B988E66EAB7
:10A8100076E0E9A1FAA1848195810E949C8AB12CFD
:10A82000A12CD12CC12C9301A4016FEF0E944250A6
:10A83000A9A1BAA11496ED91FC913097E9F488246E
:10A840008394912CC401E2960FB6F894DEBF0FBE3C
:10A85000CDBFDF91CF911F910F91FF90EF90DF90CF
:10A86000CF90BF90AF909F908F907F906F905F90B0
:10A870004F903F902F900895868097809101330CE0
:10A88000440B550B29A33AA34BA35CA389A59AA516
:10A89000092E000CAA0BBB0B8DA39EA3AFA3B8A7D8
:10A8A0008114910461F266EC75E0C4010E949C8AF7
:10A8B0007C016AEA74E0C4010E949C8A3C0160E960
:10A8C00074E0C4010E949C8A5C0165E974E0C401E3
:10A8D0000E949C8A6114710409F4B6C0A114B104E9
:10A8E00009F4B2C0009709F4AFC0D30118962C91B7
:10A8F0002F70223009F0A8C0F50120852F7022307A
:10A9000009F0A2C0DC0118962C9118972F70223004
:10A9100009F09AC0F701C184D284E384F484C1149D
:10A92000D10409F491C019968D919D910D90BC911F
:10A93000A02D0297A105B10509F48AC029A53AA561
:10A94000232B09F485C0D50119968D919C918C9D7E
:10A9500050018D9DB00C9C9DB00C11242FEF30E068
:10A96000D5010E9422BF9601DD0C440B550B0E94BD
:10A97000A2BE69A17AA18BA19CA10E9470BE2DA14B
:10A980003EA14FA158A50E94A2BE19012A01F401BF
:10A990006081718185E99DE00E94647868EC75E0D2
:10A9A00085E99DE00E946478C5016FEF70E00E9428
:10A9B000F7BE85E99DE00E94258B60ED74E185E995
:10A9C0009DE00E94CA782AE030E0B201A10185E949
:10A9D0009DE00E94DE7785E99DE00E94C177F3014A
:10A9E00081859285A385B48582159305A405B50557
:10A9F00059F119861A861B861C861D861E861F869F
:10AA0000188A8B858F708B87B101CE0109960E94C1
:10AA1000331029833A834B835C836D837E838F83DA
:10AA20009887B12CA12CD12CC12C79018A019B01D2
:10AA3000AC016FEFC4010E944250D30119962D92D0
:10AA40003D924D925C921C97F4018280938028CFB6
:10AA5000212C312C2101C3CF6F927F928F929F9234
:10AA6000AF92BF92CF92DF92EF92FF920F931F931C
:10AA7000CF93DF93CDB7DEB7A0970FB6F894DEBFC4
:10AA80000FBECDBF8C01862E7A01DC018D919C9189
:10AA90001197892B09F460C01496ED91FC913097C1
:10AAA00009F45AC080818071BFEF6B1357C0B1F4B5
:10AAB00081E0A0960FB6F894DEBF0FBECDBFDF9148
:10AAC000CF911F910F91FF90EF90DF90CF90BF90AB
:10AAD000AF909F908F907F906F9008954330510575
:10AAE00039F3818082942FE0822262EC76E085E95E
:10AAF0009DE00E94CA78D80113966C9185E99DE08B
:10AB00000E94118B60EC76E085E99DE00E94CA7896
:10AB1000D8011496ED91FC9161816F7085E99DE0FB
:10AB20000E94118B6DEB76E085E99DE00E94CA786A
:10AB3000682D85E99DE00E94118B85E99DE00E94CA
:10AB4000C177D8011496ED91FC9181818F708812A4
:10AB500007C080818F7E808380E0ABCF8111FCCFE6
:10AB6000198E1A8E1B8E1C8E1D8E1E8E1F8E18A285
:10AB70008B8D8F708B8FD8011496ED91FC91818114
:10AB80008F70881579F1B3E0EB16F10459F16BEB96
:10AB900076E085E99DE00E94CA78F801638185E945
:10ABA0009DE00E94118B69EB76E085E99DE00E94B3
:10ABB000CA78D8011496ED91FC9161816F7085E996
:10ABC0009DE00E94118B66EB76E085E99DE00E9496
:10ABD000CA78682D85E99DE00E94118B85E99DE08A
:10ABE0000E94C177F80120813181FCE0F81508F45A
:10ABF00016C1E82DF0E08827EF5FF94A8F4F0C94DB
:10AC00000BBF0E564B56CC56E356EF56CC56A556B8
:10AC1000CC56F256FD56B95600570C57D80114962B
:10AC2000CD90DC90F60181818F70853009F4F7C0FA
:10AC300050F48230C1F06CED75E0C9010E949C8A2D
:10AC40003C01912C4BC08730D1F08A30A1F765EDE3
:10AC500075E0C9010E949C8A3C01D6019C9092FA41
:10AC6000992490F83BC06FEC75E0C9010E949C8A62
:10AC70003C01D6019C9090FA992490F82FC06EEC7C
:10AC800075E0C9010E949C8A3C01F601908091FA0E
:10AC9000992490F823C061EE75E0C9010E949C8A56
:10ACA0003C01D8011496ED91FC91808180FB9924A0
:10ACB00090F8982F9E7F80FF9160908361147104BB
:10ACC00069F461E0CE0149960E941110298B3A8BFC
:10ACD0004B8B5C8B6D8B7E8B8F8B988FF801A0805C
:10ACE000B18068EA75E0C5010E949C8A6C016DEA3A
:10ACF00075E0C5010E949C8A5C01892B81F4C11416
:10AD0000D10469F460E0CE0149960E9411102983B4
:10AD10003A834B835C836D837E838F839887D801CE
:10AD20001496ED91FC916114710409F07CC0898D39
:10AD3000811179C0B82DBF708B2E8181807F882AC8
:10AD4000818280818F7E8083B3CE66EE75E0C901FB
:10AD50000E949C8A3C01D8011496ED91FC9180815F
:10AD600081FB992490F8982F9D7F81FF92609083BA
:10AD7000B5CF6CEE75E0C9010E949C8A3C01D801F8
:10AD80001496ED91FC91808182FB992490F8982F84
:10AD90009B7F82FF9460EBCF6CED75E0C9010E9450
:10ADA0009C8A3C01892B09F04CCF62E0CE01499688
:10ADB0000E94111029873A874B875C876D877E87B1
:10ADC0008F87988B3ECF62EF75E0C9010E949C8A05
:10ADD0003C01D8011496ED91FC9190804CCF67EF27
:10ADE00075E0F3CF6DEF75E0C9010E949C8A3C01CC
:10ADF000D8011496ED91FC9149CF63E076E0F4CF51
:10AE00006AE076E0C9010E949C8A3C01D801149650
:10AE1000ED91FC91908023CF60E176E0F3CF912C0F
:10AE2000712C612C5BCF83E0E816F104B9F0982D0A
:10AE30009F70892E8181807F882A818280818F7E88
:10AE40008083E98CFA8C0B8D1C8D2D8D3E8D4F8D62
:10AE500058A1692DC3010E9442502ACE81818F7072
:10AE6000881509F425CE829490EF8922882A818260
:10AE70008081806168CF8F929F92AF92BF92CF9274
:10AE8000DF92EF92FF920F931F93CF93DF93CDB793
:10AE9000DEB767970FB6F894DEBF0FBECDBF611562
:10AEA000710599F1FA017B016C01E60FF71F108221
:10AEB0000E94520F4B018B0161E57BE085E99DE02B
:10AEC0000E94CA78B40185E99DE00E94258B6EE45A
:10AED0007BE085E99DE00E94CA78B60185E99DE0A6
:10AEE0000E9464786BE47BE085E99DE00E94CA786B
:10AEF0000A3F1105ECF46EE37BE08EEE9CE00E94CD
:10AF0000CA788EEE9CE00E94C17767960FB6F894DF
:10AF1000DEBF0FBECDBFDF91CF911F910F91FF908C
:10AF2000EF90DF90CF90BF90AF909F908F9008955B
:10AF3000B70185E99DE00E94647885E99DE00E9463
:10AF4000C17780910E0990910F0963E070E0059739
:10AF500049F062E070E0C6010E94CC2D009781F4B8
:10AF600061E070E0C6010E94CC2D009749F463E3D4
:10AF70007BE085E99DE00E94CA7885E99DE0C3CF2A
:10AF8000C80ED91E67E176E0C6010E9464C3892B12
:10AF900069F4F70101900020E9F73197EE19FF09F4
:10AFA000329720F0C7010E94077EAFCF6FE270E0BA
:10AFB000C6010E9459C38C01009741F0FC01108228
:10AFC0008181843209F4A1CF0F5F1F4FF601808188
:10AFD000843209F49ACFB601CE0101960E940D2564
:10AFE000CE0101960E943612882331F0A801B701E4
:10AFF000CE0101960E94A34DCE0101960E945D12E2
:10B0000084CF2F923F924F925F926F927F928F9256
:10B010009F92AF92BF92CF92DF92EF92FF920F93E7
:10B020001F93CF93DF93CDB7DEB7C556D1090FB6C7
:10B03000F894DEBF0FBECDBFDC0114962D913C917C
:10B04000232B09F4FEC59B01225031092230310522
:10B0500008F091C23B014C01FC018281803409F46B
:10B06000F7C208F04AC0843008F085C280915B07BF
:10B070008F5F80935B07A3016FEFC4010E942C5583
:10B08000D40112960C9112970695017013961C919B
:10B0900013978AEC810F803108F043C060E276E0BC
:10B0A0008D919C910E949C8A7C010097D1F1FC01BA
:10B0B00080858F708530A9F58091640C181324C0A9
:10B0C0008091650C803401F58091660C9091670C3D
:10B0D0005C01990FCC08DD0860E0C7010E94188B65
:10B0E000FC0181859285A385B485A816B906CA0698
:10B0F000DB060CF065C0512C3EC0823409F4A8C2B6
:10B1000008F439C28058AFCF1093640C80E4809368
:10B11000650C812F0E9463949093670C8093660C5A
:10B12000D7CF212F30E0F901E75EF54E8491F90188
:10B13000ED53F64E1491F901E359F64EF490FF20C9
:10B1400009F43BC081110E94BB92EF2DF0E0EE0F9D
:10B15000FF1FE456F94FA591B491EC911E2331E005
:10B1600020E009F430E0832F922F552453940817E0
:10B17000190609F0C0CFF3E06F16710409F488C016
:10B18000D4011496ED91FC91E181EF70E150EC3027
:10B1900008F07EC0F0E08827EF52F74A8F4F0C94FA
:10B1A0000BBFF2586E5A28595E596E5A77596E5A2B
:10B1B000AB59D859F159335A555A90E080E0D5CF60
:10B1C00061E0C7010E94188B55245394FC018185CE
:10B1D0009285A385B4858A159B05AC05BD050CF049
:10B1E000CACF89CF0E94B0959B01AC014427552757
:10B1F000D4011496ED91FC916281738190E080E01E
:10B20000AA24AA94BA2CC12CD12C18EEE12E13E05A
:10B21000F12E00E010E00E94472A8823C9F1F401D2
:10B220000081118162EF75E0C8010E949C8A892B20
:10B2300041F467EF75E0C8010E949C8A892B09F4EC
:10B240000EC142E050E063E0C4010E942C5520C0D2
:10B250000E94B0959B01AC0144275527D401149658
:10B26000ED91FC916281738190E080E0AA24AA9420
:10B27000BA2CC12CD12C1CE2E12EFF24F39400E067
:10B2800010E00E94472A42E050E064E0811184C04F
:10B29000D4011496ED91FC91808183FB992790F95C
:10B2A000951509F4D2C1982F907E09F439C1982FD1
:10B2B000907E90528F71892B808358C10E94B095E7
:10B2C0009B01AC0144275527D4011496ED91FC91C4
:10B2D0006281738190E080E0AA24AA94BA2CC12CE8
:10B2E000D12C16E9E12EF12C00E010E0CACF0E942B
:10B2F000B0959B01AC0144275527D4011496ED91DC
:10B30000FC916281738190E080E0AA24AA94BA2C17
:10B31000C12CD12C18EEE12E13E0F12E00E010E04C
:10B320000E94472A882309F4B3CFF40100811181D8
:10B330006DEF75E0C8010E949C8A892B41F463E09F
:10B3400076E0C8010E949C8A892B09F488C042E0FB
:10B3500050E068E079CF0E94B0959B01AC01442792
:10B360005527D4011496ED91FC916281738190E090
:10B3700080E0AA24AA94BA2CC12CD12C1CE2E12E84
:10B38000FF24F39400E010E00E94472A42E050E0DE
:10B3900069E0882309F47CCFC4010E942C550E94E7
:10B3A000B095D4011496ED91FC917383628370CFB4
:10B3B0000E94B0959B01AC0144275527D4011496F7
:10B3C000ED91FC916281738190E080E0AA24AA94BF
:10B3D000BA2CC12CD12C16E9E12EF12C00E010E0A2
:10B3E000D3CF0E94B0959B01AC0144275527D401CF
:10B3F0001496ED91FC916281738190E080E0AA2423
:10B40000AA94BA2CC12CD12C18EEE12E13E0F12E07
:10B4100000E010E00E94472A882309F439CFF401A4
:10B42000008111816AE076E0C8010E949C8A892B24
:10B4300039F460E176E0C8010E949C8A892B21F0F2
:10B4400042E050E06BE000CF6CEE75E0C8010E9476
:10B450009C8A42E050E066E0892B09F4F5CE42E098
:10B4600050E06DE0F1CE0E94B0959B01AC01442705
:10B470005527D4011496ED91FC916281738190E07F
:10B4800080E0AA24AA94BA2CC12CD12C1CE2E12E73
:10B49000FF24F39400E010E00E94472A882309F477
:10B4A000F7CE42E050E06CE077CF0E94B0959B0170
:10B4B000AC0144275527D4011496ED91FC9162818B
:10B4C000738190E080E0AA24AA94BA2CC12CD12CDC
:10B4D00016E9E12EF12C00E010E0DECF0E94B095DD
:10B4E0009B01AC0144275527D4011496ED91FC91A2
:10B4F0006281738190E080E0AA24AA94BA2CC12CC6
:10B50000D12C18E5E12E12E0F12E00E010E00E94AF
:10B51000472A882309F4BCCE42E050E060E094CE94
:10B520000E94B095D4011496ED91FC911597738308
:10B530006283E181EF70552009F445C0E230F1F0FB
:10B5400050F4EE23E9F1D4011496ED91FC91808141
:10B5500050FA83F9B1CEE53089F0A3016AE0E73013
:10B5600091F7C4010E942C558111EDCF80915B07AA
:10B57000815080935B0790E080E065C3F401008117
:10B58000118166EE75E0C8010E949C8A892BA9F49E
:10B590006DEF75E0C8010E949C8A892B71F463E00D
:10B5A00076E0C8010E949C8A892B39F46EEC75E024
:10B5B000C8010E949C8A892B19F0A30166E0D1CFB3
:10B5C000A30161E0CECFE150ED3008F0BCCFF0E058
:10B5D0008827E251F54A8F4F0C940BBFFB5AA35AB0
:10B5E000FE5AFE5AA35A015BA35A225B225B225BDE
:10B5F000225B225BFE5AA30162E0B3CFA30165E0A8
:10B60000B0CF0D911C9166EE75E0C8010E949C8A36
:10B61000892BA9F46DEF75E0C8010E949C8A892BE3
:10B6200071F463E076E0C8010E949C8A892B39F4AA
:10B630006EEC75E0C8010E949C8A892B19F0A30169
:10B6400067E08FCFA30160E08CCF8F71806434CE30
:10B65000B3E06B16710409F48ECF60E276E0F4017A
:10B66000808191810E949C8A8C01D40113968C91D7
:10B670009091640C8913CEC09091650C903409F0C0
:10B68000C9C08091660C9091670C3C0101151105B1
:10B6900009F4F0C0F80120852F70253009F0EAC0C8
:10B6A000C8010E942D8BA4968FAFA497843008F414
:10B6B000BDC063E0C8010E94188BDC0119968D9112
:10B6C0009C913AE0D32ED89EF001D99EF00D112422
:10B6D000A396FFAFEEAFA39762E0C8010E94188B5C
:10B6E000DC0119968D919C91D89E7001D99EF00C29
:10B6F000112457010F2C000CCC08DD0861E0C801B3
:10B700000E94188BA6969FAF8EAFA69760E0C801E7
:10B710000E94188BFC012184328443845484930159
:10B72000072C000C440B550B221933094409550909
:10B73000A396AEADBFADA397BD01BB0F880B990B10
:10B740006A197B098C099D090E9470BEA696EEAD10
:10B75000FFADA6972185328543855485221933098B
:10B76000440955090E94A2BEA20EB31EC41ED51ED6
:10B77000A496FFADA497F53009F46BC081E090E08A
:10B78000A396EEADFFADA397AF01FF0F660B770B4E
:10B790004A155B056C057D050CF464C0B601A50176
:10B7A00057010F2C000CCC08DD084A155B056C0511
:10B7B0007D050CF45CC05A016B01A496FFADA49703
:10B7C000F23009F06BC06301770CEE08FF0860E00F
:10B7D000C8010E94188BFC0181859285A385B485E0
:10B7E000C816D906EA06FB060CF447C261E0C80198
:10B7F0000E94188BFC0181859285A385B4858C15E8
:10B800009D05AE05BF050CF0B6CE81E090E0A0E04E
:10B81000B0E036C28093640C90E49093650C0E9473
:10B8200063949093670C8093660C2FCF8AE0869D7B
:10B830005001879DB00C11240B2C000CCC08DD08A6
:10B84000F12CE12C20E038E2A3963FAF2EAFA39776
:10B8500095CF64E0C8010E94188BDC0119968D9188
:10B860009C918ECF66246A9423E0722E99CF712C1E
:10B87000612CA3CF2AE0289F5001299FB00C1124EE
:10B880000B2C000CCC08DD08F12CE12C20E038E278
:10B89000A3963FAF2EAFA39781E090E0D40114961A
:10B8A000ED91FC91428153819301241B350B37FFAD
:10B8B00003C0319521953109821793070CF4C1C05B
:10B8C0008081982F929596959770963008F0BCC01D
:10B8D0009F5F9295990F907E8F71892BB4C0F7016D
:10B8E00061857285DB018C91811157C2A114B1046D
:10B8F00009F474C0D50118968C9118978F70843014
:10B9000009F06CC019966D917C91CE0101960E9450
:10B910000D25CE0101960E943612882309F45AC0E3
:10B920006114710409F461C0E114F10431F0F7010C
:10B9300080858F70843009F441C025961CAE1DAE01
:10B940001EAE1FAE259729961CAE1DAE1EAE1FAEB5
:10B95000299724962FAD24972F7024962FAF2497E4
:10B9600081E022968FAF2297CC24C394F12CE12C56
:10B9700001E023961FAD239725963FAD259740E024
:10B9800027965FAD279728966FAD289729967FADAC
:10B990002997CE0101960E94273C1CC00115110574
:10B9A00029F0F80180858F70843019F06CE974E01B
:10B9B000F4C161857285FB01808196CF61857285B6
:10B9C000FB018081882331F050E040E0CE010196F8
:10B9D0000E94A34DCE0101960E945D12D4011496DF
:10B9E000ED91FC9173826282C6CD0115110531F093
:10B9F000D80118968C918F708430E9F025961CAE92
:10BA00001DAE1EAE1FAE259729961CAE1DAE1EAEF6
:10BA10001FAE299724962FAD24972F7024962FAF11
:10BA2000249782E022968FAF2297CC24C394F12CE6
:10BA3000E12C02E09ECFF80161857285DB018C91DB
:10BA4000C1CF80818F7180838081803AB8F0C70137
:10BA5000FF0CAA0BBB0B8A159B05AC05BD0571F04D
:10BA6000A396EEADFFADA397CF01FF0FAA0BBB0BC3
:10BA70008A159B05AC05BD0509F07DCD461557051A
:10BA800009F479CD6D961CAE1DAE1EAE1FAE6D973E
:10BA90006C968FAD6C978F7080666C968FAF6C973D
:10BAA0006D968CAD9DADAEADBFAD6D9765968CAF0F
:10BAB0009DAFAEAFBFAF65976996ACAEBDAECEAE33
:10BAC000DFAE69976BE876E085E99DE00E94CA7871
:10BAD000D40113966C9185E99DE00E94118B69E871
:10BAE00076E085E99DE00E94CA78CE018F5A9F4F8B
:10BAF0000E94BC3164EA75E0F401808191810E946A
:10BB00009C8AB12CA12CD12CC12C6296EFAC6297EF
:10BB10006396FFAC639764960FAD649765961FAD0F
:10BB2000659766962FAD669767963FAD679768965F
:10BB30004FAD689769965FAD69976FEF0E9442506D
:10BB4000D4010D911C9168EA75E0C8010E949C8A9D
:10BB50007C016DEA75E0C8010E949C8A8C01009707
:10BB6000E1F1FC0180858F708430B9F561857285C3
:10BB700040E450E0CE0101960E9492C36FE270E073
:10BB8000CE0101960E9459C3892B59F4D801199608
:10BB90002D913C9143E050E060E4CE0101960E947B
:10BBA000382D00E020E032E040E150E0BE016F5B64
:10BBB0007F4FCE018F5A9F4F0E94B61F0E94B78AB7
:10BBC000882359F080919A08811107C0BE016F5BEC
:10BBD0007F4FCE0101960E947E96E114F10409F494
:10BBE000FDCEF70180858F70843009F0F7CE618536
:10BBF0007285CE0101960E940D25CE0101960E940C
:10BC00003612882309F4E6CECC24C394F12CE12C1F
:10BC100062960FAD629763961FAD639764962FADE2
:10BC2000649765963FAD659766964FAD6697679644
:10BC30005FAD679768966FAD689769967FAD6997B6
:10BC4000A8CE8FEF9FEFCB59DF4F0FB6F894DEBF32
:10BC50000FBECDBFDF91CF911F910F91FF90EF905D
:10BC6000DF90CF90BF90AF909F908F907F906F901C
:10BC70005F904F903F902F90089580E090E0DC011E
:10BC8000F40124813581F90142815381052E000C94
:10BC9000660B770B481759076A077B0709F46BCCCB
:10BCA0003C01D4010D911C9168EA75E0C8010E9425
:10BCB0009C8A5C016DEA75E0C8010E949C8A6C0157
:10BCC000A114B10419F4892B09F488CE61EE75E052
:10BCD000C8010E949C8A7C016CED75E0C8010E943D
:10BCE0009C8A8C0161E976E085E99DE00E94CA7832
:10BCF000F401638185E99DE00E94118B6FE876E095
:10BD000085E99DE00E94CA78B30185E99DE00E9423
:10BD1000258B85E99DE00E94C177C114D10409F407
:10BD2000E5CDD60118968C9118978F70843009F064
:10BD3000DDCD19966D917C9140E450E0CE010196E5
:10BD40000E9492C30E94B78A882309F4CFCD8091C4
:10BD50009A088111CBCD6FE270E0CE0101960E946E
:10BD600059C3892B51F4F6012185328543E050E017
:10BD700060E4CE0101960E94382D6114710409F42B
:10BD80000DCEE114F10439F0D70118968C918F7023
:10BD9000843009F4A4CD69E974E0CE0101960E94D3
:10BDA0007E96A4CD8F929F92AF92BF92CF92DF9258
:10BDB000EF92FF920F931F93CF93DF9300D000D0A9
:10BDC000CDB7DEB72091720730917307232B09F4AA
:10BDD000C7C0209165072111C3C04C018091650740
:10BDE0008F5F8093650780910C098F5F80930C09AA
:10BDF0000E94B0959B01AC01609161077091620750
:10BE00008091630790916407AA24AA94BA2C6501D3
:10BE10001BE0E12EF12C00E010E00E94472A88236D
:10BE200009F452C0E0917207F091730706811781FF
:10BE300001151105B9F1F80180858F70863071F513
:10BE400064EA75E0C8010E949C8A0097D1F0FC0169
:10BE500020852F702530A9F4E680F780E114F104E5
:10BE6000E9F0FA82E982B801CE0101960E948918B0
:10BE7000B401CE0101960E940158F701E280F380DF
:10BE8000EDCF1A83098370E060E0CE0101960E9435
:10BE90008918B401CE0101960E940158F80102816F
:10BEA0001381C6CFF3E08F16910451F00E94B09534
:10BEB00060936107709362078093630790936407B0
:10BEC0001092640C1092650C83E088169104F1F1D5
:10BED0000E94B0959B01AC0160915D0770915E0777
:10BEE00080915F0790916007AA24AA94BA2C6501FB
:10BEF00018E8E12E13E1F12E00E010E00E94472A3D
:10BF0000882321F1E0917207F09173070681178170
:10BF10000115110589F0F80180858F70863041F494
:10BF20001A83098370E060E0CE0101960E948918AF
:10BF3000F80102811381ECCF0E94B09560935D07F8
:10BF400070935E0780935F079093600780910C0960
:10BF5000815080930C09809165078150809365071B
:10BF600026960FB6F894DEBF0FBECDBFDF91CF91FE
:10BF70001F910F91FF90EF90DF90CF90BF90AF9007
:10BF80009F908F9008954F925F926F927F92AF92A1
:10BF9000BF92CF92DF92EF92FF920F931F93CF93B6
:10BFA000DF93CDB7DEB767970FB6F894DEBF0FBE4D
:10BFB000CDBF67E273E185E99DE00E94CA7885E91B
:10BFC0009DE00E94C1770E94B0952B013C018091B9
:10BFD0000C09882329F10E94B0959B01AC01AA2489
:10BFE000AA94BA2C650110E1E12E17E2F12E00E0CF
:10BFF00010E0C301B2010E94472A811111C00E94C2
:10C000007A7E80910E0990910F09059711F00E9498
:10C01000D5480E94434B82E090E00E94D25ED7CF89
:10C0200080910C09882351F064E073E18EEE9CE06E
:10C030000E94CA788EEE9CE00E94C1776EEE72E19B
:10C0400085E99DE00E94CA7885E99DE00E94C1775C
:10C05000809178078F5F80937807E0911009F091C5
:10C060001109309781F1068117810115110559F1E8
:10C07000D80118968C918F708530B9F7C8010E944D
:10C080002D8B882391F3F80160817181CE01019697
:10C090000E940D25CE0101960E943612882359F088
:10C0A0008A859B85009739F0DC01ED91FC91028433
:10C0B000F385E02D1995CE0101960E945D12F801DD
:10C0C00002811381D2CF109277071092760766EE25
:10C0D00072E185E99DE00E94CA7885E99DE00E94B1
:10C0E000C1771092970810920D096EEC72E185E904
:10C0F0009DE00E94CA780E94520FAB01BC012AE069
:10C1000085E99DE00E94757780917407909175078D
:10C110000E94B18F109275071092740710927307E6
:10C12000109272071092110910921009109299083A
:10C130001092980810920A091092090969EC72E1AC
:10C1400085E99DE00E94CA780E94520FAB01BC01B4
:10C150002AE085E99DE00E94757785E99DE00E94CF
:10C16000C17710920B0980917807815080937807EE
:10C1700067960FB6F894DEBF0FBECDBFDF91CF91AB
:10C180001F910F91FF90EF90DF90CF90BF90AF90F5
:10C190007F906F905F904F90089580919A088F5F85
:10C1A00080939A08A89583E090E00E94D25E0E9456
:10C1B0007A7E80919A08815080939A080895CF9250
:10C1C000DF92EF92FF92CF93DF93EC018C85883062
:10C1D00068F40E9472860E94B0956B017C018C8588
:10C1E0000E948E86811109C088E08C87DF91CF91F3
:10C1F000FF90EF90DF90CF9008950E94CD6061E0B6
:10C2000070E080E090E00E94A8940E94B095AB019D
:10C21000BC014C195D096E097F098D859E85B0E0D2
:10C22000A0E0481759076A077B07C8F28C850E946F
:10C230008086DACFCF92DF92EF92FF921F93CF9357
:10C24000DF93EC017B016A018C85883048F40E9401
:10C250008E86882319F08C850E94728688E08C87F0
:10C26000F70182819381A481B5810097A105B10571
:10C2700051F490E080E0DF91CF911F91FF90EF901B
:10C28000DF90CF9008958F3F9F4FAF4FBF4F89F3FF
:10C2900070E060E081E20E94C986182F8C878830A8
:10C2A00040F780E591E00E940190A7014E5F5F4F4B
:10C2B00024E030E06CE070E0812F0E946626B60139
:10C2C000812F0E949D8664E070E0812F0E94AA81E8
:10C2D0000E94B0956B017C018C850E948E8687310F
:10C2E00021F18C3111F1882321F20E94B095AB012C
:10C2F000BC014C195D096E097F098D859E85B0E0F2
:10C30000A0E084179507A607B70748F00E94CD6004
:10C3100061E070E080E090E00E94A894DDCF8C8521
:10C320000E94808688E08C87A4CF81E090E0A3CF34
:10C330008F929F92BF92CF92DF92EF92FF920F93D4
:10C340001F93CF93DF93CDB7DEB76D970FB6F894F9
:10C35000DEBF0FBECDBF00917407109175070115A8
:10C36000110509F4ECC180910C098F5F80930C09D1
:10C3700064E276E0C8010E949C8A90931109809340
:10C3800010096AE276E0C8010E949C8A909399089D
:10C390008093980861E874E0C8010E949C8A909399
:10C3A00073078093720761E376E0C8010E949C8A5C
:10C3B00090930A09809309090E9400301092770730
:10C3C00010927607E0911009F0911109309709F465
:10C3D000C8C0E680F780009110091091110901157D
:10C3E000110509F4B7C0E114F10409F4B3C0D70191
:10C3F00018968C918F70853091F7C7010E942D8B14
:10C40000823068F3B701CE0101960E947E22CE01F0
:10C4100001960E943612882309F44AC08A859B85BA
:10C42000009759F570E060E0CE0101960E94A91CCA
:10C430008C01912C812C97FF06C011950195110953
:10C4400088248394912CCE0101960E949E1EC82EB2
:10C45000D12C89858530A9F1863051F5B02E61E067
:10C46000802F0E94509361E0892809F451C0CA943A
:10C47000CD2809F051C060E04FC0DC01ED91FC9186
:10C480000484F585E02D1995892B49F08A859B85D3
:10C49000DC01ED91FC910284F385E02D19958A85EC
:10C4A0009B85DC01ED91FC910680F781E02D1995CB
:10C4B000D7011296ED90FC90CE0101960E945D127C
:10C4C0008ACFCD2829F462E0CE0101960E94881D12
:10C4D00061E0802F0E94509360E0802F0E942293A1
:10C4E00065E47EE085E99DE00E94CA78B80185E9AF
:10C4F0009DE00E94258B60E47EE085E99DE00E943E
:10C50000CA786EE37EE085E99DE00E94CA78D0CFCC
:10C51000CA94CD2809F0AFCFC62ED12C8B2D0E9406
:10C52000229369E37EE085E99DE00E94CA78B80124
:10C5300085E99DE00E94258B67E37EE085E99DE02B
:10C540000E94CA78B60185E99DE00E94258B65E3CB
:10C550007EE0D9CFF8018681978190937707809309
:10C56000760785E99DE00E94C177E0917207F0911E
:10C570007307309709F48AC080910C098F5F80930C
:10C580000C09068117810115110509F47AC0D8013B
:10C5900018968C918F70863009F069C0198F088FBA
:10C5A00070E060E0CE0148960E9489188C8D9D8DC8
:10C5B000892B09F45CC08091740790917507892BD1
:10C5C00009F455C0E88CF98CF70180858F708630AE
:10C5D00099F564EA75E0C7010E949C8A0097F1F022
:10C5E000DC0118962C9118972F702530B9F4169607
:10C5F000CD90DC90C114D104F9F0DA82C982B70180
:10C60000CE0101960E948918ED81FE81108211826F
:10C6100012821382F601C280D380ECCFFA82E982C3
:10C6200070E060E0CE0101960E94891862E070E03F
:10C63000CE0101960E940158EC8DFD8D1082118271
:10C64000128213828A8D843068F462E0823008F0AE
:10C6500060E08B8D0E945093EC8DFD8D8181807FF9
:10C66000818305C0803441F060E0823431F0D8012C
:10C6700012960D911C9187CF62E08B8D0E94509392
:10C68000F6CF80910C09815080930C0968E27EE01E
:10C6900084EE9CE00E94CA7860E27EE084EE9CE03A
:10C6A0000E94CA7881E02091100930911109232B52
:10C6B00009F480E00E94431667E17EE084EE9CE08E
:10C6C0000E94CA7881E02091720730917307232B72
:10C6D00009F480E00E94431660E17EE084EE9CE075
:10C6E0000E94CA7881E02091090930910A09232B20
:10C6F00009F480E00E94431684EE9CE00E94C1771A
:10C700006BE07EE084EE9CE00E94CA780E94520FAB
:10C71000AB01BC012AE084EE9CE00E94757784EEB8
:10C720009CE00E94C17781E080930D0980910C0903
:10C73000815080930C0988EB9CE00E94DF606D962D
:10C740000FB6F894DEBF0FBECDBFDF91CF911F9122
:10C750000F91FF90EF90DF90CF90BF909F908F90C0
:10C760000895CF93DF9300D000D01F921F92CDB7D2
:10C77000DEB761E77EE084EE9CE00E94CA7884EE3A
:10C780009CE00E94C1771092E10C1092E00C80E0D6
:10C7900090E19093DC0C8093DB0C84E690E0909326
:10C7A000E30C8093E20C81E08093DD0C80E090E26A
:10C7B0009093DF0C8093DE0C8FEC9CE00E94B825F8
:10C7C0008B37910509F04CC01C821B8280E093E0FE
:10C7D0009A8389838FEC9CE09E838D838FEF9FEFFC
:10C7E00098878F838091740790917507892B11F03A
:10C7F0000E94C35FCE0101960E94E38F909375075C
:10C80000809374078FEC9CE00E94741280917407EF
:10C8100090917507892B69F464E57EE08EEE9CE0CB
:10C820000E94CA788EEE9CE00E94C17790E080E082
:10C830000EC06DE47EE084EE9CE00E94CA7884EE37
:10C840009CE00E94C1770E94986181E090E0289668
:10C850000FB6F894DEBF0FBECDBFDF91CF91089524
:10C860008FEC9CE00E94AD1260E67EE084EE9CE0DE
:10C870000E94CA7884EE9CE00E94C1778FEC9CE015
:10C880000E947412D3CF0E94B163892B31F486EFDA
:10C890009FEF90930F0980930E0908954F925F9236
:10C8A0006F927F92AF92BF92CF92EF92FF920F93CF
:10C8B0001F93CF93DF9300D000D01F921F92CDB76C
:10C8C000DEB75C0109831A832B833C834D835E832F
:10C8D0006F83788763E776E085E99DE00E94CA78F8
:10C8E000CE0101960E94BC318981811134C00B8137
:10C8F0000F700130A9F160F1023021F010E0053035
:10C9000009F03FC0D501ED91FC91068CF78DE02D2B
:10C9100009811A812B813C814D815E816F817885EF
:10C92000C501199581E090E028960FB6F894DEBF16
:10C930000FBECDBFDF91CF911F910F91FF90EF9070
:10C94000CF90BF90AF907F906F905F904F90089581
:10C95000CC24C394D7CF813051F1823009F4DEC0AA
:10C9600066E676E085E99DE00E94CA78698185E9FE
:10C970009DE00E94118B85E99DE00E94C17701E056
:10C9800010E066E576E085E99DE00E94CA78B8018E
:10C9900085E99DE00E94258B85E99DE00E94C17795
:10C9A000CE0101960E94BC3190E080E0BDCF1B819A
:10C9B00012951F70163009F478C088F48FEF810F3C
:10C9C000823048F52D8130E0A4E6B0E00E94D4BE6C
:10C9D0002FEF30E040E050E00E94A2BE19C01730B7
:10C9E000E9F186EF810F8230B0F48D819E81AF81B5
:10C9F000B88585369105A105B10524F084E690E05F
:10CA0000A0E0B0E0B7FF03C080E090E0DC019C0153
:10CA100029313105D4F4163009F47BC008F05EC02A
:10CA20001150123008F469C0F5016281738140E051
:10CA300052E0CE0101960E946D3A60E07AE0D501A5
:10CA400012968D919C910E94BB3BD501ED91FC917A
:10CA5000068CF78DE02DCC24C3945ACF4D805E8098
:10CA60006F80788420E030E0A901C301B2010E9408
:10CA700036BD87FD11C020E030E048EC52E4C30130
:10CA8000B2010E943EC0181654F4412C512C88EC7F
:10CA9000682E82E4782E03C0412C512C3201C30150
:10CAA000B2010E9408C09B01B3CF6D817E818F814E
:10CAB00098852AE030E040E050E00E94A2BE253692
:10CAC00031054105510524F024E630E040E050E016
:10CAD00057FF9ECF20E030E0A9019ACF173081F0B8
:10CAE0001A5086E690E0A0E0B0E0123008F09CCF4B
:10CAF0008D839E83AF83B88797CF86E68D8394CF4F
:10CB000080E090E0ACECB2E48D839E83AF83B88785
:10CB10008BCF8CEF93E0A0E0B0E0EACF1D821E82C5
:10CB20001F821886D501ED91FC91068CF78DE02DC2
:10CB3000CC24C39402E01A812B813C8140E0EDCEED
:10CB4000EF92FF920F931F93CF93DF9300D01F922A
:10CB5000CDB7DEB78C017B01FB0184858830A8F05E
:10CB600080E094E0F8019183808312821382148222
:10CB70001582C8010F900F900F900F90DF91CF9109
:10CB80001F910F91FF90EF90089580E591E00E9432
:10CB9000019024E030E0AE014F5F5F4F6CE070E049
:10CBA000F70184850E949527BE016F5F7F4FC80102
:10CBB0000E940079DECFAF92BF92CF92DF92EF92C8
:10CBC000FF920F931F93CF93DF93CDB7DEB7C25879
:10CBD000D1090FB6F894DEBF0FBECDBF8E010F5B3B
:10CBE0001F4FD8011D921C92FE01ED5BFF4F2EE1FD
:10CBF000DF011D922A95E9F7E090C70CF090C80C70
:10CC000002970CF455C0FB01628173814FE150E043
:10CC1000C8010E9492C3EF28D9F10E949C8B8823FF
:10CC2000B9F1F80101900020E9F73197E01BF10B11
:10CC3000B09770F582E70E943A8B8091C70C909173
:10CC4000C80CDC01ED91FC910684F785E02D6CE1C8
:10CC500070E01995B8018091C70C9091C80C0E94A2
:10CC600064788091C70C9091C80CDC01ED91FC9127
:10CC70000190F081E02D60E019958091C70C9091B2
:10CC8000C80CDC01ED91FC910288F389E02D199527
:10CC9000B80184EE9CE00E94647863E670E184EE63
:10CCA0009CE00E94CA7884EE9CE00E94C17735C067
:10CCB000EF2809F46EC10E949C8B882309F469C196
:10CCC00082E70E943A8B8091C70C9091C80CDC01DE
:10CCD000ED91FC910684F785E02D6CE170E01995EB
:10CCE0004FE150E0B8018091C70C9091C80C0E94B0
:10CCF000DD8B7C018091C70C9091C80CDC01ED911B
:10CD0000FC910288F389E02D1995E114F10409F4EE
:10CD100040C1F801EE0DFF1D10828091CE0C1F92D4
:10CD20008F938091CD0C1F928F938091CC0C1F928A
:10CD30008F938091CB0C1F928F938091CA0C1F927E
:10CD40008F938091C90C1F928F9386E396E09F93F7
:10CD50008F931F9280E48F93FE0131966F01FF93B2
:10CD6000EF930E94ACC365E270E184EE9CE00E9408
:10CD7000CA78B80184EE9CE00E946478B60184EE23
:10CD80009CE00E94647884EE9CE00E94C1777E0162
:10CD9000F1E6EF0EF11CD70113961C921E9212972A
:10CDA00088EE93E0A0E0B0E0F70184839583A6834A
:10CDB000B78388E0848788EE93E0968785878CE840
:10CDC00093E091838083108B0787128A118A80E514
:10CDD00090E0948B838B178A6FE170E185E99DE089
:10CDE0000E94CA780E94520FAB01BC012AE085E97B
:10CDF0009DE00E94757785E99DE00E94C17764E619
:10CE000070E080E090E00E94A89465EE72E784EF05
:10CE100090E80E94BEB68C010FB6F894DEBF0FBE3C
:10CE2000CDBF892BB1F183E090E00E94A9B2D80177
:10CE30001D969C938E931C97FC01F182E0821282D6
:10CE4000C7010E945115882319F0C7010E94DF60B5
:10CE5000D70151966D917C9152975396AD90BC90AD
:10CE60006115710509F4A8C0CE0187589F4F0E9433
:10CE70000079A501BE0167587F4FC7010E941A6162
:10CE8000181619060CF414C1C8010E94CD8010E0D8
:10CE900000E067E170E185E99DE00E94CA7885E9DC
:10CEA0009DE00E94C17764E670E080E090E00E941F
:10CEB000A894D7015596ED90FC906EE070E185E95D
:10CEC0009DE00E94CA78B70185E99DE00E94258B0C
:10CED00085E99DE00E94C17764E670E080E090E023
:10CEE0000E94A8940115110509F4DBC0B8ECEB16FB
:10CEF000F10409F0C1C062E070E184EE9CE00E94A0
:10CF0000CA7864EF71E080E090E00E94A894ED960A
:10CF10001FAE1EAEED97EF961FAE1EAEEF978FEFD2
:10CF20009FEFC158DF4F99838883CF57D0408AEE57
:10CF300092E0EB969FAF8EAFEB97CF57DF4F198301
:10CF40000883C158D040F894809174079091750778
:10CF5000892B11F00E94C35FCE0187589F4F0E941A
:10CF6000E38F90937507809374077894C8010E94AB
:10CF7000CD808091740790917507892B09F05AC074
:10CF80006BEE7FE08EEE9CE00E94CA788EE090E02F
:10CF900061C040E250E067E570E1C8010E940DB653
:10CFA00069E370E184EE9CE00E94CA78B80184EEE7
:10CFB0009CE00E94647877CEF70167857089A501AF
:10CFC000C7010E9473155CCF6E01E9E7CE0ED11C3C
:10CFD000DF92CF9280E69FE09F938F931F930F93F2
:10CFE0000E9462B70F900F900F900F900F900F90CC
:10CFF000019709F04ECFD6018D919C91F701968B48
:10D00000858B90E0D12CFAE0DF120FC09A3009F442
:10D0100040CFC8010E9409B78F3F21F4C8010E9488
:10D02000CD8037CF9D2DD82EEECF8DE0D812F1CF09
:10D03000D92EEFCF60EE7FE084EE9CE00E94CA78AC
:10D040000E94986169ED7FE084EE9CE00E94CA78BE
:10D0500084E090E0CE57DF4F0FB6F894DEBF0FBEEE
:10D06000CDBFDF91CF911F910F91FF90EF90DF9097
:10D07000CF90BF90AF90089561EC7FE08EEE9CE082
:10D080000E94CA78B7018EEE9CE00E94258B8EEE3E
:10D090009CE00E94C17780910D09882309F476CF26
:10D0A000D7CF6EEA7FE085E99DE00E94CA78F3CF92
:10D0B000F701B784A088DF92CF928AEA9FE09F931E
:10D0C0008F931F930F930E9445B7DF92CF9285EA0B
:10D0D0009FE09F938F931F930F930E9445B7D801B2
:10D0E0001C96ED91FC9181E08283DF92CF9282EADF
:10D0F0009FE09F938F931F930F930E9445B7D80192
:10D100001C96ED91FC911282AF92BF928CE69FE04B
:10D110009F938F931F930F930E9445B787EA9FE0D9
:10D120009F938F931F930F930E9445B7F701168A21
:10D13000158AD8011C96ED91FC91A080B1800FB6A4
:10D14000F894DEBF0FBECDBF83E3C82ED12CD5012E
:10D15000ED91FC910084F185E02DC5011995419771
:10D160000CF032CFB1E0CB1AD10809F42DCF64E135
:10D1700070E080E090E00E94A894E9CFEF92FF92E7
:10D180000F931F93CF93DF93EC018B0102970CF168
:10D19000FB01E280F38069E57FE0C7010E94C3B52F
:10D1A000892BF9F065E57FE0C7010E94C3B5892BA3
:10D1B000C1F065E37FE084EE9CE00E94CA7870E0F5
:10D1C00060E084EE9CE00E94258B84EE9CE00E944F
:10D1D000C177B801CE010E94DB6590930F0980935F
:10D1E0000E09DF91CF911F910F91FF90EF9008955D
:10D1F000EF92FF920F931F93CF93DF93CDB7DEB7DC
:10D2000064970FB6F894DEBF0FBECDBF0D871E87A3
:10D210002F87388B498B5A8B6B8B7C8B65E676E03E
:10D2200085E99DE00E946478CE010D960E94BC3194
:10D230009F85892F8F70082F10E02D85222309F4F8
:10D24000A6C00115110509F474C0813009F471C03C
:10D250008130A0F18230C1F18E3009F07FC092950B
:10D260009F7069897A899C3011F070E060E0CE018E
:10D2700001960E9400776EE776E0C7010E9464C3C2
:10D28000892B09F03FC0BE016F5F7F4FCE0107962B
:10D290000E94F776CE0107960E94C891BC018CE9E6
:10D2A0009BE00E94BC78CE0107960E94C47601E004
:10D2B00010E0CE0101960E94C47616C066E874E1C3
:10D2C00085E99DE00E94CA7862E774E185E99DE006
:10D2D0000E94CA7885E99DE00E94C1778F85807F92
:10D2E00001E010E009F400E0C80164960FB6F8947C
:10D2F000DEBF0FBECDBFDF91CF911F910F91FF9089
:10D30000EF9008956EE876E0C7010E9464C300E0E4
:10D31000892B71F6BE016F5F7F4FCE0107960E9489
:10D32000F776CE0107960E94C891BC018FEF9AE074
:10D33000B8CF213021F1223039F165E674E185E979
:10D340009DE00E94CA786D8585E99DE00E94118B61
:10D3500085E99DE00E94C17701E010E065E574E198
:10D3600085E99DE00E94CA78B80185E99DE00E94A8
:10D37000258B85E99DE00E94C17700E003C02093E2
:10D38000290201E010E0B0CF10922902FACF8130DB
:10D3900009F05ECFD2CF6F927F928F929F92AF9221
:10D3A000BF92CF92DF92EF92FF920F931F93CF9392
:10D3B000DF93CDB7DEB72C970FB6F894DEBF0FBE64
:10D3C000CDBF4C018CE99BE00E94706F892B39F135
:10D3D00080E00E94FE1560933D0870933E088093A4
:10D3E0003F08909340088CE99BE00E944E6F682EA6
:10D3F0008DE290E09A83898369824FE350E0BE0119
:10D400006F5F7F4F83EB97E00E9474C380913B086E
:10D4100090913C08019690933C0880933B088FEFD5
:10D420009AE00E94706F892B39F180E00E94FE150E
:10D4300060933708709338088093390890933A08BE
:10D440008FEF9AE00E944E6F782E8DE290E09A83E3
:10D45000898379824FE350E0BE016F5F7F4F85EF94
:10D4600097E00E9474C38091350890913608019628
:10D47000909336088093350880913D0890913E083E
:10D48000A0913F08B0914008892B8A2B8B2B09F083
:10D49000C7C08AE26812DFC010923D0810923E08B1
:10D4A00010923F081092400810923C0810923B08DE
:10D4B00063EB77E0CE0107960E9400771092B307E6
:10D4C000CE0107960E9423758B859C85892B09F4D4
:10D4D000DFC16CE676E0CE0101960E940077BE01C6
:10D4E0006F5F7F4FCE0107960E94C375182FCE0144
:10D4F00001960E94C476112321F08091290288238D
:10D50000A1F0BE01695F7F4FCE0101960E94F776C0
:10D51000CE0101960E94C891BC018FEF9AE00E9453
:10D52000BC78CE0101960E94C476BE01695F7F4F30
:10D53000CE0101960E94F776BE016F5F7F4FC40156
:10D540000E940119CE0101960E94C47665E776E03B
:10D55000CE0101960E940077BE016F5F7F4FCE0122
:10D5600007960E94C375182FCE0101960E94C476BB
:10D57000112309F450C1BE01695F7F4F8EEC9DE01D
:10D580000E94F375811184C1BE01695F7F4F8EECEB
:10D590009DE00E94AD764F815885D4011296ED91A1
:10D5A000FC9113970190F081E02D60817181ED91E4
:10D5B000FC910288F389E02D2BE736E0C401199530
:10D5C0008091F3079091F407892B09F461C161E51B
:10D5D00074E185E99DE00E94CA7810E000E0A0E1D6
:10D5E000EA2EF12CB801CE0107960E94B175FC011C
:10D5F0008081882309F448C18B859C850817190709
:10D6000008F042C18091F3079091F40781309105B1
:10D6100009F443C1029709F46BC10F5F1F4FE2CFBA
:10D620000E94B0959B01AC0160913D0870913E084D
:10D6300080913F0890914008AA24AA94BA2C6501D1
:10D640001AE0E12EF12C00E010E00E94472A882326
:10D6500009F41FCF21CFADE06A1609F41DCF8091E8
:10D660003B0890913C088034910508F015CF8091DB
:10D67000370890913808A0913908B0913A08892B61
:10D680008A2B8B2B09F040C1BAE27B1258C1109251
:10D690003708109238081092390810923A08109200
:10D6A00036081092350865EF77E0CE0107960E94A4
:10D6B00000771092F507CE0107960E9423758B859F
:10D6C0009C85892B09F49BC16CE676E0CE0101961E
:10D6D0000E940077BE016F5F7F4FCE0107960E94C8
:10D6E000C375182FCE0101960E94C476112321F034
:10D6F000809129028823A1F0BE01695F7F4FCE018E
:10D7000001960E94F776CE0101960E94C891BC0155
:10D710008CE99BE00E94BC78CE0101960E94C47601
:10D72000BE01695F7F4FCE0101960E94F776BE0170
:10D730006F5F7F4FC4010E940119CE0101960E94C4
:10D74000C47665E776E0CE0101960E940077BE01BF
:10D750006F5F7F4FCE0107960E94C375182FCE01D1
:10D7600001960E94C476112309F40CC1BE01695FC1
:10D770007F4F8AED9DE00E94F375811140C1BE018B
:10D78000695F7F4F8AED9DE00E94AD764F8158859D
:10D79000D4011296ED91FC9113970190F081E02D48
:10D7A00060817181ED91FC910288F389E02D2BE875
:10D7B00036E0C40119958091F3079091F407892B05
:10D7C00009F41DC163E574E185E99DE00E94CA7812
:10D7D000912C812C00E110E0B401CE0107960E944B
:10D7E000B175FC018081882309F405C18B859C8576
:10D7F0008816990608F0FFC08091F3079091F4070E
:10D800008130910509F400C1029709F428C1BFEFE6
:10D810008B1A9B0AE1CF60E876E0CE0101960E9468
:10D820000077BE016F5F7F4FCE0107960E94C375E0
:10D83000182FCE0101960E94C476112309F4C0CEA0
:10D84000BE01695F7F4F84ED9DE00E94F3758111F9
:10D850001FC0BE01695F7F4F84ED9DE00E94AD76E1
:10D860004F815885D4011296ED91FC911397019048
:10D87000F081E02D60817181ED91FC910288F38946
:10D88000E02D26E836E09ACE85E99DE00E94C1773A
:10D89000CE0107960E94C476EACEB801CE01079663
:10D8A0000E94B175DC018C9166EA76E0803114F457
:10D8B00066E675E085E99DE00E946478B801CE01D6
:10D8C00007960E94B175FC018081082E000C990B0F
:10D8D000AA0BBB0B89839A83AB83BC83FE82ED8248
:10D8E000BE016F5F7F4F85E99DE00E94791895CE5C
:10D8F000B801CE0107960E94B175DC016C9185E9F3
:10D900009DE00E94D77789CE0E94B0959B01AC0123
:10D9100060913708709138088091390890913A08E1
:10D92000AA24AA94BA2C65011AE0E12EF12C00E099
:10D9300010E00E94472A882309F4A6CEA8CEEDE085
:10D940007E1609F4A4CE8091350890913608803473
:10D95000910508F09CCE81E090E02C960FB6F894EB
:10D96000DEBF0FBECDBFDF91CF911F910F91FF9012
:10D97000EF90DF90CF90BF90AF909F908F907F906F
:10D980006F90089560E876E0CE0101960E940077DE
:10D99000BE016F5F7F4FCE0107960E94C375182F9F
:10D9A000CE0101960E94C476112309F404CFBE0172
:10D9B000695F7F4F80EE9DE00E94F37581111FC06B
:10D9C000BE01695F7F4F80EE9DE00E94AD764F8182
:10D9D0005885D4011296ED91FC9113970190F08136
:10D9E000E02D60817181ED91FC910288F389E02D39
:10D9F00020E936E0DECE85E99DE00E94C177CE01C8
:10DA000007960E94C476A7CFB401CE0107960E9464
:10DA1000B175DC018C9166EA76E0803114F466E63B
:10DA200075E085E99DE00E946478B401CE01079617
:10DA30000E94B175FC018081082E000C990BAA0B85
:10DA4000BB0B89839A83AB83BC831E830D83BE018A
:10DA50006F5F7F4F85E99DE00E947918D8CEB401B1
:10DA6000CE0107960E94B175DC016C9185E99DE0BD
:10DA70000E94D777CCCEAF92BF92CF92DF92EF9237
:10DA8000FF920F931F93CF93DF93CDB7DEB7C554AB
:10DA9000D1090FB6F894DEBF0FBECDBF5C016B019C
:10DAA000CE0101960E94F776BE016F5F7F4F85E938
:10DAB0009DE00E94BC7885E99DE00E94C177CE017F
:10DAC00001960E94C4766DE27BE0CE0101960E9431
:10DAD000C976BE016F5F7F4FC6010E94F375182F94
:10DAE000CE0101960E94C476112399F120E04DE207
:10DAF00051E0B50186E99CE00E94D97D67E07BE0BA
:10DB0000C5010E94EE78C5010E94C17764E670E00D
:10DB100080E090E00E94A894D501ED91FC910488EA
:10DB2000F589E02DC501199501E010E0C801CB5B36
:10DB3000DF4F0FB6F894DEBF0FBECDBFDF91CF91A0
:10DB40001F910F91FF90EF90DF90CF90BF90AF901B
:10DB50000895002309F434C16BEF7AE0CE010196F9
:10DB60000E94C976BE016F5F7F4FC6010E94C375D8
:10DB7000182FCE0101960E94C476112309F459C0D2
:10DB80004BE050E070E060E0C6010E948075B50196
:10DB9000CE01805C9F4F0E94529BF6016081718193
:10DBA000CE0181960E940D25CE0181960E943612EB
:10DBB00081110CC000E911E0CE0181960E945D1236
:10DBC000CE01805C9F4F0E94C476B0CF22966EAD8E
:10DBD0007FAD229750E040E0CE0181960E94A34D98
:10DBE000892B41F318AE19AE1AAE1BAE1CAE1DAE9A
:10DBF0001EAE1FAE8AAD8F708AAF40E053E0BE010B
:10DC00006F5D7F4FCE01C8960E94DA3A00E020E0B7
:10DC100033E040E250E0BE016F5F7F4FCE01C89617
:10DC20000E94B61FBC01C7010E94967608EC10E165
:10DC3000C3CF60EF7AE0CE0101960E94C976BE01A3
:10DC40006F5F7F4FC6010E94C375182FCE010196EA
:10DC50000E94C476112309F450C04AE050E070E0FD
:10DC600060E0C6010E948075D6016D917C91CE0165
:10DC700081960E940D25CE0181960E94361200E900
:10DC800011E08823A9F189A5873061F4CE0181963E
:10DC90000E945D4A61E0892B09F462E0CE01819621
:10DCA0000E94881D18AE19AE1AAE1BAE1CAE1DAE7A
:10DCB0001EAE1FAE8AAD8F708AAF40E053E0BE014A
:10DCC0006F5D7F4FCE01C8960E94DA3A00E020E0F7
:10DCD00033E040E250E0BE016F5F7F4FCE01C89657
:10DCE0000E94B61FBC01C7010E94967608EC10E1A5
:10DCF000CE0181960E945D1219CF61EE7AE0CE01CD
:10DD000001960E94C976BE016F5F7F4FC6010E94D7
:10DD1000C375182FCE0101960E94C476112309F411
:10DD200052C04EE050E070E060E0C6010E94807595
:10DD3000B501CE0101960E94529B41E050E06AE697
:10DD400076E0C6010E9423764D815E8169817A81E9
:10DD5000C6010E9423766BED7AE085E99DE00E9482
:10DD6000CA78B601CE0181960E94F776BE016F5D3A
:10DD70007F4F85E99DE00E94BC7885E99DE00E9487
:10DD8000C177CE0181960E94C47665E976E0C6012E
:10DD90000E94DE75882341F021E048EC50E0B50197
:10DDA00086E99CE00E94D97DF601808191810E94E4
:10DDB000077ECE0101960E94C47608EC10E0B6CE34
:10DDC00001E911E0B3CE10E000E0B0CE0895FC010F
:10DDD000248135816217730748F48081918100970F
:10DDE00029F0860F971FFC018081089580E0089537
:10DDF0000895AF92BF92CF92DF92EF92FF920F936E
:10DE00001F93CF93DF936C017B018B01040F151FD0
:10DE1000EB015E01AE18BF08C017D10759F0699138
:10DE2000D601ED91FC910190F081E02DC60119958C
:10DE3000892B79F7C501DF91CF911F910F91FF9049
:10DE4000EF90DF90CF90BF90AF900895FC01A08934
:10DE5000B1898C91A689B78982FD0FC09C91818D73
:10DE60008F5F8F73228D821749F0A18DAE0FBF2F68
:10DE7000B11D5D969C93818F08958C910895FC014E
:10DE8000538D448D252F30E0842F90E0821B930B1F
:10DE9000541710F0CF96089501970895FC01918DC5
:10DEA000828D981761F0A28DAE0FBF2FB11D5D96C8
:10DEB0008C91928D9F5F9F73928F90E008958FEF6A
:10DEC0009FEF0895FC01918D828D981731F0828D1E
:10DED000E80FF11D858D90E008958FEF9FEF089575
:10DEE000FC01918D228D892F90E0805C9F4F821BD9
:10DEF00091098F739927089582E69AE00E94706FC6
:10DF000021E0892B09F420E0822F08958FEF9AE019
:10DF10000E94706F21E0892B09F420E0822F089580
:10DF20008CE99BE00E94706F21E0892B09F420E0CE
:10DF3000822F089588EF9CE00E94706F21E0892B6A
:10DF400009F420E0822F0895FC01A48DA80FB92FB9
:10DF5000B11DA35ABF4F2C91848D90E001968F7311
:10DF60009927848FA689B7892C93A089B1898C9130
:10DF700080648C93938D848D981306C00288F389F6
:10DF8000E02D80818F7D80830895EF92FF920F9323
:10DF90001F93CF93DF93EC0181E0888F9B8D8C8D55
:10DFA000981316C0E889F989808185FF11C0EE8930
:10DFB000FF896083E889F98980818064808381E0BA
:10DFC00090E0DF91CF911F910F91FF90EF90089516
:10DFD000F62E0B8D10E00F5F1F4F0F731127E02EF1
:10DFE0008C8D8E110CC00FB607FCFACFE889F98929
:10DFF000808185FFF5CFCE010E94A46FF1CFEB8D1C
:10E00000EC0FFD2FF11DE35AFF4FF0820B8FEA89D1
:10E01000FB8980818062D2CFCF93DF93EC01888D22
:10E020008823B9F0AA89BB89E889F9898C9185FD93
:10E0300003C0808186FD0DC00FB607FCF7CF8C9121
:10E0400085FFF2CF808185FFEDCFCE010E94A46FC6
:10E05000E9CFDF91CF91089580E090E0892B29F0FE
:10E060000E949A6F81110E94000080E090E0892B4D
:10E0700029F00E94906F81110E94000080E090E0E2
:10E08000892B29F00E94866F81110E94000080E098
:10E0900090E0892B29F00E947C6F81110C94000084
:10E0A00008950F931F93FC01628573858485958580
:10E0B0000281138124813581601B710B820B930BCC
:10E0C0000685178520893189601B710B820B930BA4
:10E0D0001F910F910895DC01ED91FC910190F08169
:10E0E000E02D19948FEF9FEF0895FC0162897389E9
:10E0F000848995890895EF920F931F93CF93DF93AF
:10E10000FC01248D222341F0213051F1DF91CF9188
:10E110001F910F91EF900895228933894489558981
:10E1200086899789A08DB18D821B930BA40BB50BAB
:10E13000892F9A2FAB2FBB278C010F5F1F4F628156
:10E14000738184819581CFB7F894DCB7E1E0ECBFAF
:10E15000EE24E394E2E0FEEF1995DCBFCFBFD6CF0B
:10E16000F0E0E0E0DF91CF911F910F91EF901994D3
:10E17000FC01138E128E41110CC082899389A489EF
:10E18000B589868B978BA08FB18F148E81E090E03C
:10E19000089590E080E00895CF92DF92EF92FF9291
:10E1A000CF93DF93DC01CB01642FCFB7F8946D01DF
:10E1B000EE24FF24CBBEDCB741E04CBFA901E1E077
:10E1C000FEEF1995DCBFCFBFDF91CF91FF90EF90AD
:10E1D000DF90CF900895CF93DF93FC01248D211120
:10E1E00010C0EC01828D938D892B49F06689778967
:10E1F000808D918D30E020E045E00E94CC701B8E38
:10E200001A8EDF91CF9108951F93CF93DF93FC0176
:10E21000248D211145C0162FEC01828D938D892B01
:10E2200049F466897789808D918D30E020E043E064
:10E230000E94CC704A8D5B8DCA0181709927FE01C6
:10E24000E80FF91F158F892B69F02D8D3E8D6E8992
:10E250007F89888D998D640F751F811D911D41E007
:10E260000E94CC708A8D9B8D01969B8F8A8F811521
:10E270009140B1F46E897F89888D998D30E020E0DE
:10E2800045E00E94CC701B8E1A8E8E899F89A88DC6
:10E29000B98D9F5FAF4FBF4F8E8B9F8BA88FB98F6C
:10E2A00081E090E0DF91CF911F910895DC01ED9125
:10E2B000FC910280F381E02D40E01994FB01248160
:10E2C0003581428153812417350750F4A081B181F3
:10E2D000A20FB31F8C9384819581019695838483CB
:10E2E00080E00895CF93DF93EC01E881F981028407
:10E2F000F385E02DCE0119950196B9F7DF91CF9105
:10E300000895CF92DF92EF92FF920F931F93CF93D6
:10E31000DF937C016A018B01D0E0C0E0CC15DD0504
:10E3200081F0D701ED91FC910284F385E02DC701C6
:10E3300019958F3F980729F0F80181938F01219655
:10E34000EDCFCE01DF91CF911F910F91FF90EF9014
:10E35000DF90CF900895CF93C62FDC01ED91FC9113
:10E360000088F189E02D1995DC01ED91FC91019077
:10E37000F081E02D6C2FCF911994062E000C770BB5
:10E38000FC01778366830895CF93DF93EC018E8140
:10E390009F81019611F5E881F9810088F189E02DCE
:10E3A000CE011995DC01ED91FC910084F185E02D01
:10E3B0001995892BB1F0E881F9810284F385E02D6C
:10E3C000CE0119958132910534F3E881F9810684F3
:10E3D000F785E02D682FCE01199581E0DF91CF916F
:10E3E000089580E0FBCFFC0120812EBD9B012150D0
:10E3F000310941F051810DB407FEFDCF4EB55EBD30
:10E400004193F5CF61507109860F971F0DB407FE38
:10E41000FDCF2EB5FC0120830895E0911309F09102
:10E420001409808190911209892B80830895E091CD
:10E430001309F09114099081809112098095892324
:10E44000808308958EBD00000DB407FEFDCF8EB50C
:10E45000089590E020914F0A233339F40C96982FB9
:10E46000990F990F990F80E008954896F8CFEF9291
:10E47000FF920F931F93CF93DF93EC018B017A01EF
:10E480000E94B095688B798B8A8B9B8B8C819D8148
:10E49000DC01ED91FC910280F381E02DA701B80130
:10E4A000DF91CF911F910F91FF90EF9019941F93DF
:10E4B000CF93DF93EC01162F0E94B095688B798B78
:10E4C0008A8B9B8B8C819D81DC01ED91FC9101906D
:10E4D000F081E02D612FDF91CF911F911994CF92A0
:10E4E000DF92EF92FF92CF93DF93EC018E819F81B9
:10E4F0008F3F980759F02FEF3FEF3F832E83DF9137
:10E50000CF91FF90EF90DF90CF9008950E94B0954B
:10E510006B017C01A4EFCA0EA1E0DA1EE11CF11C24
:10E52000E881F9810088F189E02DCE011995DC019F
:10E53000ED91FC910084F185E02D1995892B39F43A
:10E540000E94B0956C157D058E059F0548F3E88106
:10E55000F9810088F189E02DCE011995DC01ED915A
:10E56000FC910284F385E02DDF91CF91FF90EF9035
:10E57000DF90CF9019940E94ECC20F931F93CF931A
:10E58000DF93EC0188819981009759F02A813B81C2
:10E590002617370730F081E0DF91CF911F910F915F
:10E5A00008958B016F5F7F4F0E940BC2009759F057
:10E5B000998388831B830A832C813D81232B59F700
:10E5C000FC011082E8CF80E0E7CFEF92FF920F933B
:10E5D0001F93CF93DF93009751F4CFEFDFEFCE017E
:10E5E000DF91CF911F910F91FF90EF900895DC0183
:10E5F0001C96ED90FC90F70100811181D801ED91FE
:10E60000FC910688F789E02DC8011995882329F324
:10E61000D801ED91FC910084F185E02DC801199598
:10E62000D801ED91FC91892B61F30284F385E02DF3
:10E63000C8011995EC01019681F2F80187898823B8
:10E6400029F06C2F88EF9CE00E94118BD701129665
:10E650008C91882321F2C532D10509F6D801ED91BC
:10E66000FC910084F185E02DC801199502975CF0BA
:10E67000D801ED91FC910688F789E02DC801199524
:10E680008111ECCFAACFD1E0C0E0D801ED91FC918F
:10E690000284F385E02DC80119958F3F980709F48E
:10E6A0009CCF9C01215431092A31310570F48D2F02
:10E6B0008295807F829FC00D1124D11104C00C2E41
:10E6C000000CDD0B8CCFD0E0E0CF9C01215631094E
:10E6D0002A31310560F3C0978A30910570F79D2F7C
:10E6E0009295907F989FC00D1124E7CFCF92DF9233
:10E6F000EF92FF920F931F93CF93DF936C018B01E7
:10E7000086E090E00E94A9B2EC0190939409809376
:10E710009309F60101900020E9F7CF018C199D09BA
:10E720000E94A9B27C01B6010E946DC3F60101905E
:10E730000020E9F73197EC19FD09EE0DFF1D10825D
:10E74000F982E8821B830A83809196099091970948
:10E750009D838C83D0939709C0939609DF91CF91C5
:10E760001F910F91FF90EF90DF90CF900895FC01E3
:10E77000868197818F3F980729F02FEF3FEF3783EE
:10E7800026830895808591850C9409B77F928F9296
:10E790009F92AF92BF92CF92DF92EF92FF920F9330
:10E7A0001F93CF93DF93CDB7DEB7A6970FB6F8943C
:10E7B000DEBF0FBECDBF8C01762E942E852E20E2BB
:10E7C000A22ECE0101967C01DC01EA2D1D92EA9574
:10E7D000E9F76801F3E4CF0ED11C80E094E09AA33E
:10E7E00089A38FEF8BA38CA38DA38EA343E450E06A
:10E7F000BE016F5D7F4FC6010E942728019609F474
:10E80000BFC081E089838A8386E0B82EBB821C82E8
:10E81000D80114966D917D918D919C9117970E94CE
:10E8200013BF6D837E838F83988789869A8680E85D
:10E8300090E09C878B874CE150E0B701C6010E94B5
:10E84000BC27FE0137968AE1DF011D928A95E9F720
:10E850004801B8E08B0E911CF401D70101900D9294
:10E86000BA94E1F740E150E0B701C6010E94BC272D
:10E87000F7011192AA94E9F796E0A92EB12C40E293
:10E8800050E0B701C6010E94BC27F1E0AF1AB10801
:10E89000B1F783E6898392E89A8393E59B838C831F
:10E8A00085E38D8381E08E837F829DE3988797E067
:10E8B00099878A8786E0F401DE011B9601900D920C
:10E8C0008A95E1F78CE0898B8A8B6DE976E0CE0141
:10E8D00043960E946DC3D8011B966C91CE01499658
:10E8E0000E94A390F8016485CE014B960E94A390EC
:10E8F000D8011D966C91CE014D960E94A3904EE1D9
:10E9000050E0B701C6010E94BC27B3E07B121EC0D5
:10E9100082E3898384E08A83F80196859B839785C7
:10E920009C8390899D8391899E8396E39F838887AA
:10E93000828D8987838D8A87848D8B87858D8C874F
:10E940004CE050E0B701C6010E94BC2787E38983F1
:10E9500086E08A8391E09B8393E09C838D838FE0A4
:10E960008E838AE38F838BE388878FEF898749E0E3
:10E9700050E0B701C6010E94BC27C6010E94F627DD
:10E98000A6960FB6F894DEBF0FBECDBFDF91CF9134
:10E990001F910F91FF90EF90DF90CF90BF90AF90BD
:10E9A0009F908F907F90089590E080E00C94942643
:10E9B000CF93DF93C4E1D0E00E94D474882361F048
:10E9C00061E070E080E090E00E94A8942197A1F7B8
:10E9D00080E0DF91CF91089581E0FBCFFF920F930C
:10E9E0001F93CF93DF931F921F92CDB7DEB7F82E00
:10E9F00022E030E0AE014F5F5F4F66E270E00E94C0
:10EA0000952709811A8110270127102722E030E07D
:10EA1000AE014F5F5F4F66E270E08F2D0E94952739
:10EA200089819A819827892798270817190749F417
:10EA3000C8010F900F90DF91CF911F910F91FF9020
:10EA400008958C01E3CFAF92BF92CF92DF92EF9205
:10EA5000FF920F931F93CF93DF93DC01CD90DC9057
:10EA60001197C114D10439F01496CD91DC918C0129
:10EA70007601209761F4DF91CF911F910F91FF9064
:10EA8000EF90DF90CF90BF90AF9008957501570140
:10EA9000BFEFAB1ABB0AF7018081082E000C990B5F
:10EAA0000E94BAB5892B91F72197CC0DDD1D888185
:10EAB000082E000C990B0E94BAB5892B29F0CE15AF
:10EAC000DF0510F02197F3CFAE014F5F5F4F4E1976
:10EAD0005F09D80115965C934E931497CE14DF040A
:10EAE00020F4B701C6010E9420C3D801ED91FC912A
:10EAF000119714968D919C91E80FF91F1082BBCF4E
:10EB0000CF93DF93DC011496ED91FC916E177F0794
:10EB100028F54115510511F19F01261B370B4217AE
:10EB2000530708F49A01DB01EC0188819981E21B0B
:10EB3000F30BFD83EC83AF01461B570B260F371FEA
:10EB4000BC01620F731F8A0F9B1F0E9492C3E88152
:10EB5000F9818C819D81E80FF91F1082DF91CF919F
:10EB60000895FC01248135816217730720F48081A8
:10EB70009181009729F41092950985E999E008950B
:10EB8000860F971F0895FB0144815581FC01248164
:10EB900035812417350778F080819181009759F0ED
:10EBA000FB01608171816115710529F00E9484C3A8
:10EBB00021E0892B09F020E0822F0895FC012481B7
:10EBC0003581232B39F421E0FB018081882349F032
:10EBD00020E007C0808191810E9464C321E0892BDD
:10EBE000B9F7822F0895FC0124813581FB0144810E
:10EBF000558124173507E1F4FC0180819181FB01E7
:10EC0000608171810097D1F061157105A1F4232B0A
:10EC1000C1F0FC01808190E008C0232B91F0FB0142
:10EC2000808190E091958195910921E0892B09F0EF
:10EC300020E0822F08950E9464C3F7CF611571050B
:10EC400061F721E0F6CFEF92FF920F931F93CF93DE
:10EC5000DF936115710541F480E0DF91CF911F9141
:10EC60000F91FF90EF90089541155105B1F07B0190
:10EC7000EC010C811D81040F151FB8010E94BD72AB
:10EC8000882351F3288139818C819D81B701820FBE
:10EC9000931F0E946DC31D830C8381E0DECFCF9351
:10ECA000DF931F921F92CDB7DEB769831A8241E0CE
:10ECB00050E0BE016F5F7F4F0E9423760F900F9050
:10ECC000DF91CF910895CF93DF93EC0188819981F3
:10ECD000009711F00E9445B3198218821D821C8290
:10ECE0001B821A82DF91CF910895EF92FF920F93CA
:10ECF0001F93CF93DF93EC017B018A01BA010E943D
:10ED0000BD7281110BC0CE010E946376CE01DF91EE
:10ED1000CF911F910F91FF90EF9008951D830C8369
:10ED2000B701888199810E946DC3F0CFCF93DF93A3
:10ED3000EC016115710571F0FB0101900020E9F70C
:10ED40003197AF01461B570B0E947576CE01DF91BC
:10ED5000CF9108950E946376F9CFCF93DF93EC01B2
:10ED6000FB018617970749F0608171816115710574
:10ED700041F0448155810E947576CE01DF91CF919B
:10ED800008950E946376F9CFFC01808191810C94F3
:10ED900045B3EF92FF920F931F93CF93DF93EC0154
:10EDA0008B01198218821B821A821D821C82CB0160
:10EDB0000E94E6B57C01BC01CE010E94BD728111AA
:10EDC00009C0CE01DF91CF911F910F91FF90EF907D
:10EDD0000C946376FD82EC82B80188819981DF9181
:10EDE000CF911F910F91FF90EF900C94DFB5FC0134
:10EDF0001182108213821282158214820C94AD76D5
:10EE0000FC01118210821382128215821482611514
:10EE1000710551F0FB0101900020E9F73197AF0136
:10EE2000461B570B0C94757608950F931F93CF9341
:10EE3000DF93EC010E94B095688779878A879B876A
:10EE4000E881F9810284F385E02DCE01199597FFC1
:10EE500015C00E94B095088519852A853B85601BE1
:10EE6000710B820B930B0C811D812E813F816017EA
:10EE700071078207930720F38FEF9FEFDF91CF9108
:10EE80001F910F910895CF92DF92EF92FF920F930F
:10EE90001F93CF93DF936C017A018B01D0E0C0E028
:10EEA000C6010E94157797FD07C0F80181938F0175
:10EEB0002196EC16FD06A1F7CE01DF91CF911F91AF
:10EEC0000F91FF90EF90DF90CF900895FB0101909C
:10EED0000020E9F73197AF01461B570BDC01ED919C
:10EEE000FC910280F381E02D19948F929F92AF9252
:10EEF000BF92EF92FF920F931F93CF93DF93CDB703
:10EF0000DEB7A1970FB6F894DEBF0FBECDBF7C0170
:10EF1000FA01CB0119A2223008F42AE08E010F5D1C
:10EF20001F4F822E912CB12CA12CBF01A501940161
:10EF30000E9480BEF901CA016A300CF5605DD801FB
:10EF40006E938D01232B242B252B79F790E080E005
:10EF5000109721F0BD01C7010E946677A1960FB6F8
:10EF6000F894DEBF0FBECDBFDF91CF911F910F91FF
:10EF7000FF90EF90BF90AF909F908F900895695C45
:10EF8000DECF64EA76E00C9466770F931F93CF93FD
:10EF9000DF93EC010E9466778C01CE010E94C1775D
:10EFA000800F911FDF91CF911F910F910895DC0188
:10EFB000ED91FC910190F081E02D1994CF92DF92B8
:10EFC000EF92FF920F931F93CF93DF93211531059B
:10EFD00081F4DC01ED91FC910190F081E02D642F32
:10EFE000DF91CF911F910F91FF90EF90DF90CF9025
:10EFF00019942A30310501F52AE077FF1DC06A0116
:10F000007B01EC016DE20E94D7778C0144275527E4
:10F01000BA014C195D096E097F092AE0CE010E94F0
:10F020007577800F911FDF91CF911F910F91FF9006
:10F03000EF90DF90CF900895DF91CF911F910F91C6
:10F04000FF90EF90DF90CF900C9475778F929F9206
:10F05000AF92BF92CF92DF92EF92FF920F931F93E6
:10F06000CF93DF937C018B014C0182E0880E911CD1
:10F070005701E5E0AE0EB11CD0E0C0E0F4016191B3
:10F080004F01C8010E94118B6C016EE2C8010E9401
:10F09000D7778C0D9D1DC80FD91F8A149B0471F75B
:10F0A000F7016581C8010E94118B8C0F9D1FDF91B4
:10F0B000CF911F910F91FF90EF90DF90CF90BF9075
:10F0C000AF909F908F9008956115710511F00C9489
:10F0D000667790E080E008950F931F93CF93DF93BE
:10F0E000EC018B0167EA76E00E9464780115110556
:10F0F000C1F1F80161918F01662399F1603240F00E
:10F10000623231F06C3521F0CE010E94D777F1CF19
:10F110006CE5CE010E94D777F801319780818C3061
:10F12000D1F044F48930D9F08A30B9F0883009F749
:10F1300062E6EACF823259F024F462E78D3021F39F
:10F14000D8CF8F3231F06CE58C35F1F2D2CF62E25C
:10F15000DBCF6FE2D9CF66E6D7CF6EE6D5CF64E7D7
:10F16000D3CF62E2CE010E94D77790E080E0DF91BA
:10F17000CF911F910F910895DB0114964D915C91F1
:10F1800015976D917C91DC01ED91FC910280F381EA
:10F19000E02D1994EF92FF920F931F93CF93DF937B
:10F1A0008C017B01D0E0C0E0F701EC0FFD1F649102
:10F1B000662361F0D801ED91FC910190F081E02D82
:10F1C000C8011995892B11F02196EECFCE01DF9160
:10F1D000CF911F910F91FF90EF9008950F931F9380
:10F1E000CF93DF93EC010E94CA788C01CE010E947C
:10F1F000C177800F911FDF91CF911F910F910895DB
:10F20000DC0180E094E08D939D9384E0FB0101900C
:10F210000D928A95E1F708953F924F925F926F9217
:10F220007F928F929F92AF92BF92CF92DF92EF9296
:10F23000FF920F931F93CF93DF93CDB7DEB7EA977B
:10F240000FB6F894DEBF0FBECDBF7C012A013B0193
:10F2500069010E94B0954B015C0187010D5B1F4F56
:10F26000C8010E941D1418161906ACF00E94B09532
:10F27000681979098A099B094616570668067906AE
:10F2800008F468C10E94CD6061E070E080E090E029
:10F290000E94A894E5CF42E250E0BE016F5F7F4F2D
:10F2A000C8010E94A81389818230D1F0312C832DAE
:10F2B000EA960FB6F894DEBF0FBECDBFDF91CF91B7
:10F2C0001F910F91FF90EF90DF90CF90BF90AF9084
:10F2D0009F908F907F906F905F904F903F90089598
:10F2E000F801848995898334910501F76D817E81C8
:10F2F0008F8198850E9413BF4B015C01F6018082CB
:10F300009182A282B38246E050E0B701685F7F4FEE
:10F31000CE014D960E9413C3892B41F6F7018081DF
:10F320009181A281B38188169906AA06BB0608F4CA
:10F33000BDCF84819581A681B78188159905AA05DD
:10F34000BB0508F4B3CF89899A89AB89BC898687C4
:10F350009787A08BB18B4EEC50E070E060E0C80165
:10F360000E94A813312CC701829698AB8FA7F70192
:10F37000B696FAABE9AB08969CAB8BAB67019AE10A
:10F38000C90ED11CBD96FEABEDABC701429698AF3E
:10F390008FABFD97FAAFE9AF4701FEE18F0E911CED
:10F3A000F801818D928D181619060CF080CFC801D6
:10F3B0000E94C7138333910509F4B2C014F581305C
:10F3C000910509F464C044F4892B51F3C8010E94EB
:10F3D000C713AC01552775C08330910509F462C08D
:10F3E0000697A1F7C8010E94C713B82E44E050E069
:10F3F000B401C8010E94A813EB2DE450FF0BAF012C
:10F4000060C08A33910509F45FC084F585339105A6
:10F41000B1F1C697D9F6C8010E94C7135C01B601C5
:10F42000CE0189960E9400798BA59CA5ADA5BEA5AD
:10F43000892B8A2B8B2BB1F0EDA9FEA9408051803E
:10F4400062807380B601CE0183960E9400798DA1FF
:10F450009EA1AFA1B8A5A501481659066A067B066C
:10F4600009F0B8CF44E050E0B60118C08B339105E5
:10F4700009F440C08F3F910509F492CFA7CFC8018E
:10F480000E94C713C8010E94C713382E89CFC80134
:10F490000E94C71344E050E06FA978ADC8010E94F4
:10F4A000A8137ECFC8010E94C713B82E44E050E0D5
:10F4B00069AD7AADC8010E94A8138B2D8450990BB9
:10F4C000AC0170E060E0EACFC8010E94C71344E0DD
:10F4D00050E069A97AA9C8010E94A813F70166A1A2
:10F4E00077A180A591A50E9413BF66A377A380A7EB
:10F4F00091A756CFC8010E94C71344E050E06BA902
:10F500007CA9C8010E94A813F70162A573A584A570
:10F5100095A50E9413BF62A773A784A795A740CFA4
:10F52000C8010E94C71344E050E06FA578A9C80144
:10F530000E94A813F70162A173A184A195A10E9462
:10F5400013BF62A373A384A395A366A777A780AB19
:10F5500091AB26CF33243A94AACE2F923F924F926A
:10F560005F926F927F928F929F92AF92BF92CF9253
:10F57000DF92EF92FF920F931F93CF93DF9300D010
:10F5800000D0CDB7DEB78C010E941AB42FEC37E063
:10F5900040E050E00E94A2BEDC01CB010196A11D1B
:10F5A000B11DF80184839583A683B78380839183FB
:10F5B000A283B3835801F3E4AF0EB11CC5010E94CE
:10F5C000721364E470E0C5010E94EC14882309F40E
:10F5D00045C10E94B0952B013C01480182E4880E90
:10F5E000911C48EEC42E43E0D42EE12CF12C52E0C5
:10F5F000252E1E821D82D4018C918330B1F18111A0
:10F6000066C0F80184819581A681B7810196A11D0C
:10F61000B11D84839583A683B7830E94B095641936
:10F62000750986099709A70196010E9480BEA90164
:10F6300061E0C8010E94C67381E0D4018C938D8182
:10F640009E810197C1F20E94B095641975098609DF
:10F650009709D801D6962D913D914D915C91D997FE
:10F66000261737074807590720F6C5010E9472136D
:10F67000F80184819581A681B7810196A11DB11DF4
:10F6800084839583A683B7830E94B095F801FE9684
:10F6900060837183828393838D819E8126960FB6CA
:10F6A000F894DEBF0FBECDBFDF91CF911F910F91B8
:10F6B000FF90EF90DF90CF90BF90AF909F908F9092
:10F6C0007F906F905F904F903F902F90089584307F
:10F6D000F1F4F80184819581A681B7810196A11D7D
:10F6E000B11D84839583A683B7830E94B095641966
:10F6F000750986099709A70196010E9480BEA90194
:10F7000063E0C8010E94C673D4012C9298CF813067
:10F7100051F5F80142AD53AD64AD75AD9E012F5F5B
:10F720003F4FC8010E940C79382EF2E08F1390C031
:10F7300089819A81AB81BC81F80184839583A683FA
:10F74000B7830E94B0956419750986099709A701C6
:10F7500096010E9480BEA90163E0C8010E94C673A1
:10F76000D4013C926CCF823009F069CFF80142ADF0
:10F7700053AD64AD75AD9E012F5F3F4FC8010E9430
:10F780000C79382EF5E08F135DC0E3E0D401EC93E3
:10F79000F80182A193A1A4A1B5A1892B8A2B8B2B5F
:10F7A00041F484E893E0A0E0B0E082A393A3A4A393
:10F7B000B5A3F80186A197A1A0A5B1A5892B8A2B95
:10F7C0008B2B61F482A193A1A4A1B5A1B695A795B5
:10F7D0009795879586A397A3A0A7B1A7F80182A5BF
:10F7E00093A5A4A5B5A5892B8A2B8B2BA9F482A15F
:10F7F00093A1A4A1B5A1AC01BD0123E076956795C5
:10F80000579547952A95D1F7841B950BA60BB70BF7
:10F8100082A793A7A4A7B5A7F80186A197A1A0A541
:10F82000B1A586A797A7A0ABB1AB82A593A5A4A5C8
:10F83000B5A582AB93ABA4ABB5AB81E090E09E8362
:10F840008D83FDCE96E0891303C0D4011C92F7CEC0
:10F85000BFEF3B12F4CEF4011082F1CE1E821D8266
:10F860001BCF1F920F920FB60F9211240BB60F925F
:10F870002F933F934F935F936F937F938F939F93B8
:10F88000AF93BF93EF93FF9382E69AE00E94A46F39
:10F89000FF91EF91BF91AF919F918F917F916F9168
:10F8A0005F914F913F912F910F900BBE0F900FBE24
:10F8B0000F901F9018951F920F920FB60F92112460
:10F8C0000BB60F922F933F934F935F936F937F935A
:10F8D0008F939F93AF93BF93EF93FF9382E69AE04A
:10F8E0000E94266FFF91EF91BF91AF919F918F91F1
:10F8F0007F916F915F914F913F912F910F900BBE30
:10F900000F900FBE0F901F9018951F920F920FB679
:10F910000F9211240BB60F922F933F934F935F9347
:10F920006F937F938F939F93AF93BF93EF93FF93C7
:10F930008FEF9AE00E94A46FFF91EF91BF91AF917A
:10F940009F918F917F916F915F914F913F912F91F7
:10F950000F900BBE0F900FBE0F901F9018951F9227
:10F960000F920FB60F9211240BB60F922F933F9365
:10F970004F935F936F937F938F939F93AF93BF93B7
:10F98000EF93FF938FEF9AE00E94266FFF91EF9124
:10F99000BF91AF919F918F917F916F915F914F91A7
:10F9A0003F912F910F900BBE0F900FBE0F901F90A5
:10F9B00018951F920F920FB60F9211240BB60F924B
:10F9C0002F933F934F935F936F937F938F939F9367
:10F9D000AF93BF93EF93FF938CE99BE00E94A46FDA
:10F9E000FF91EF91BF91AF919F918F917F916F9117
:10F9F0005F914F913F912F910F900BBE0F900FBED3
:10FA00000F901F9018951F920F920FB60F9211240E
:10FA10000BB60F922F933F934F935F936F937F9308
:10FA20008F939F93AF93BF93EF93FF938CE99BE0EA
:10FA30000E94266FFF91EF91BF91AF919F918F919F
:10FA40007F916F915F914F913F912F910F900BBEDE
:10FA50000F900FBE0F901F9018951F920F920FB628
:10FA60000F9211240BB60F922F933F934F935F93F6
:10FA70006F937F938F939F93AF93BF93EF93FF9376
:10FA800088EF9CE00E94A46FFF91EF91BF91AF912E
:10FA90009F918F917F916F915F914F913F912F91A6
:10FAA0000F900BBE0F900FBE0F901F9018951F92D6
:10FAB0000F920FB60F9211240BB60F922F933F9314
:10FAC0004F935F936F937F938F939F93AF93BF9366
:10FAD000EF93FF9388EF9CE00E94266FFF91EF91D8
:10FAE000BF91AF919F918F917F916F915F914F9156
:10FAF0003F912F910F900BBE0F900FBE0F901F9054
:10FB00001895CF92DF92EF92FF921F93CF93DF93DE
:10FB1000EC016A017B01122FE889F98982E0808378
:10FB2000C11481EED806E104F104A1F060E079E0AF
:10FB30008DE390E0A70196010E9480BE215031091B
:10FB4000410951095695479537952795211580E12B
:10FB5000380798F0E889F989108260E874E88EE146
:10FB600090E0A70196010E9480BE21503109410911
:10FB700051095695479537952795EC85FD85308336
:10FB8000EE85FF852083188EEC89FD891083EA8934
:10FB9000FB89808188698083EA89FB8980818F7DE8
:10FBA0008083DF91CF911F91FF90EF90DF90CF90F6
:10FBB0000895DF92EF92FF920F931F93CF93DF93FD
:10FBC00000D000D0CDB7DEB78B017A01D22E66EA25
:10FBD00076E0CE0101960E9400779E012F5F3F4F95
:10FBE0004D2DB701C8010E94DA94CE0101960E9402
:10FBF000C47626960FB6F894DEBF0FBECDBFDF9158
:10FC0000CF911F910F91FF90EF90DF900895CF92C9
:10FC1000DF92EF92FF920F931F93CF93DF93CDB7B5
:10FC2000DEB7EC970FB6F894DEBF0FBECDBFDC0198
:10FC30002C91222309F444C06AE676E00E941CB6A7
:10FC40009A8389837E01B3E0EB0EF11C01E010E0A2
:10FC5000D02EC12E6AE676E090E080E00E941CB6CD
:10FC6000F701819391937F010E31110521F00F5F10
:10FC70001F4F892B69F70091930910919409E9802E
:10FC8000FA800115110579F1D8016D917C91C701B8
:10FC90000E9464C3892B19F5D8011296ED91FC914D
:10FCA000BE016F5F7F4F8D2D9C2D199588EF9CE0D5
:10FCB0000E94C17765E975E188EF9CE00E94CA78EF
:10FCC000EC960FB6F894DEBF0FBECDBFDF91CF919B
:10FCD0001F910F91FF90EF90DF90CF900895F80162
:10FCE00004811581CECF69E975E188EF9CE00E941F
:10FCF000EE78DCCFCF9388EF9CE00E94706F892B69
:10FD0000E9F188EF9CE00E944E6FC82F8A3089F09D
:10FD10008D3079F0883001F568E088EF9CE00E9432
:10FD2000D77780919809882331F38150809398097F
:10FD3000E2CFE0919809F0E0E95AF64F108264EAC8
:10FD400076E088EF9CE00E94647887E599E00E9465
:10FD5000077E10929809CFCF682F88EF9CE00E9411
:10FD6000D777E0919809EB3330F681E08E0F8093DE
:10FD70009809F0E0E95AF64FC083BDCFCF910895BE
:10FD80008F929F92AF92BF92CF92DF92EF92FF92AB
:10FD90000F931F93CF93DF936115710509F493C0FF
:10FDA000DB011896EC911897E295E07FE595E595D3
:10FDB000E595E595E73008F086C0EC010E2E000CC5
:10FDC000FF0B8827E951F1488F4F0C940BBFEE7E53
:10FDD000FF7E087F1F7F667F787FB17F69EA76E0CC
:10FDE000CE01DF91CF911F910F91FF90EF90DF90A7
:10FDF000CF90BF90AF909F908F900C94667719969C
:10FE00008C9163EB76E0882359F36EEA76E0E8CFD5
:10FE100019964D915D916D917C911C972AE030E08F
:10FE2000CE01DF91CF911F910F91FF90EF90DF9066
:10FE3000CF90BF90AF909F908F900C94DE771996E3
:10FE4000CD90DD90ED90FC901C9720E030E0A90172
:10FE5000C701B6010E9436BD87FF09C06DE575E098
:10FE6000CE010E946478F7FAF094F7F8F094C70195
:10FE7000B6010E940FC04B015C012AE0BC01A40145
:10FE8000CE010E94757769EB76E0CE010E9464781E
:10FE9000C501B4010E943BBD9B01AC01C701B60185
:10FEA0000E9429BF2DEC3CEC4CE45DE30E942ABF8C
:10FEB00020E030E040E251E40E949CBD0E940FC06F
:10FEC000CE010E94F78D90E080E01DC019966D91E3
:10FED0007C91CE01DF91CF911F910F91FF90EF9018
:10FEE000DF90CF90BF90AF909F908F900C946C78E4
:10FEF00016960D911C916BE5CE010E94D777019665
:10FF000079F48FEF9FEFDF91CF911F910F91FF90C9
:10FF1000EF90DF90CF90BF90AF909F908F9008951B
:10FF20000115110579F0B801CE010E94C07E01963D
:10FF300041F3D80112960D911C910115110511F094
:10FF40006CE2DACF6DE5CE010E94D77721E030E098
:10FF5000019611F030E020E088279927821B930B4F
:10FF6000D2CF16960D911C916BE7CE010E94D777E8
:10FF7000019639F20115110529F1D8016D917C9195
:10FF8000CE010E946C78019609F4BBCF6AE3CE01E2
:10FF90000E94D777019609F4B4CFB801CE010E9430
:10FFA000C07E019609F4ADCFD80112960D911C9137
:10FFB0000115110539F06CE2CE010E94D777019648
:10FFC000C9F69FCF6DE7BFCFCF93DF93EC01E881F8
:10FFD000F9810284F385E02DCE0119958F3F9807B2
:10FFE00069F0E881F981813291059CF30684F785F7
:10FFF000E02D682FCE01199590E080E0DF91CF9140
:020000021000EC
:100000000895CF92DF92EF92FF920F931F93CF93B9
:10001000DF937C016B01DC01ED91FC910284F3859F
:10002000E02D1995829761F0CFEFDFEFCE01DF91E0
:10003000CF911F910F91FF90EF90DF90CF90089597
:10004000F6018085807F8460808786E090E00E9452
:10005000A9B28C01009741F3E7E1F9E0DC01ED93EF
:10006000FC9380E4DF011D928A95E9F780E490E03B
:10007000F8019383828315821482D701ED91FC915C
:100080000284F385E02DC7011995EC010196C9F0B2
:10009000C232D10509F44DC0C032D1050CF449C0BB
:1000A000B8018C2FCC35D10549F5D701ED91FC91E4
:1000B0000284F385E02DC7011995EC018F3F980765
:1000C00021F4C8010E9445B3B1CF8236910541F1B8
:1000D0005CF48F32910509F18C359105D9F0829746
:1000E00061F6B80182E20AC08E369105E1F04CF467
:1000F000B8018CE0C636D10509F0BFCF0E945E7111
:10010000BCCF8237910591F0B80189E0C437D105A1
:10011000A9F3B3CFB8018CE5F1CFB8018FE2EECFF0
:10012000B80188E0EBCFB8018AE0E8CFB8018DE0F4
:10013000E5CFF80184819581009749F00190F08125
:10014000E02DE80FF91F31978081882321F0B80155
:1001500080E00E945E71D80114968D919C910E945E
:10016000A9B2EC01009739F067E179E00E946DC314
:10017000C8010E9445B3F601D287C187D0E0C0E034
:1001800055CF8DE090E00E94A9B2009729F02DE0B4
:10019000FC0111922A95E9F708950F931F93CF93CD
:1001A000DF930097E1F0EC010C851D850115110529
:1001B00079F0D8018D919C91009739F0DC01ED9197
:1001C000FC910488F589E02D1995C8010E9445B37A
:1001D000CE01DF91CF911F910F910C9494B6DF91D6
:1001E000CF911F910F910895AF92BF92CF92DF925E
:1001F000EF92FF920F931F93CF93DF9300D01F9244
:10020000CDB7DEB761157105B1F06B01182FDB01B9
:100210001C96AD90BC90F501E080F180D701ED9186
:10022000FC910688F789E02DC7011995811106C058
:10023000C6010E94CD808FEF9FEF13C0F501928120
:10024000911124C0D701ED91FC910190F081E02D36
:10025000612FC7011995F7018789811111C090E0BD
:1002600080E00F900F900F900F90DF91CF911F9132
:100270000F91FF90EF90DF90CF90BF90AF900895D7
:10028000612F88EF9CE00E94D777E9CF812F8F7D87
:1002900081548A31B8F280ED810F8A3098F283ED73
:1002A000810F823078F21F3569F21E3759F2113210
:1002B000B1F086EC810F823090F08AED810F8730AB
:1002C00070F01D3361F0812F8F7E8F3241F08DED04
:1002D000810F823020F01B3511F01D3511F491FF94
:1002E000B1CF19821A821B821C82812F012E000C31
:1002F000990B9F931F938BEB96E09F938F938E01A7
:100300000F5F1F4F1F930F930E94E9C36E01F4E02C
:10031000CF0ED11C0F900F900F900F900F900F9059
:10032000D8016D918D01D701ED91FC910190F08183
:10033000E02DC7011995F7018789882339F0F80165
:100340003197608188EF9CE00E94D7770C151D05DE
:1003500039F785CFCF93C82F462F61E070E00E9418
:10036000772661E070E08C2F0E94A5268111F9CFDD
:10037000CF910895AF92BF92CF92DF92EF92FF920A
:100380000F931F93CF93DF9300D01F92CDB7DEB7AB
:100390008C016B017A0180914F0A8333E9F45B0190
:1003A0006801C40ED51EC016D106A9F10E941772AD
:1003B0008FE00E942272812F0E942272802F0E9461
:1003C00022720F5F1F4F80E00E942272F50181931D
:1003D0005F010E940D72E7CF843369F50E941772A6
:1003E00019830A838F2D8F778B83EC8264E070E012
:1003F000CE0101960E94F371A70170E060E0C60192
:100400000E9479BCE114F10421F0B701C6010E94F9
:10041000F3710E940D72C7010F900F900F900F9013
:10042000DF91CF911F910F91FF90EF90DF90CF90D0
:10043000BF90AF9008950E9417720F3F110509F009
:1004400030F419820A831B8263E070E0D1CF17FD7C
:100450000BC019820A8333E0169507953A95E1F7A8
:10046000007E08600B83F0CFC80126E09695879543
:100470002A95E1F7807E19830A830115104C18F440
:1004800080618B83E1CF8861FCCFAF92BF92CF9226
:10049000DF92EF92FF920F931F93CF93DF9300D0E1
:1004A00000D01F921F92CDB7DEB78C017B016A018D
:1004B00080914F0A8333E1F45801A40EB51EA016B3
:1004C000B10609F46FC00E94177280EF0E94227279
:1004D000812F0E942272802F0E9422720F5F1F4F75
:1004E000F70181917F010E9422720E940D72E7CF75
:1004F0005B01A40EB51E8433C1F40E9417721983E8
:100500000A838D2D80688B83CC8264E070E0CE01FD
:1005100001960E94F371AE14BF0409F441C0F701C3
:1005200081917F010E942272F6CF0E9417720F3FC5
:10053000110509F028F419820A8384E08B830CC02A
:1005400017FD17C019820A8333E0169507953A956F
:10055000E1F7007E0C600B8386E0C816D104A0F59D
:10056000F701DE011496EA15FB0599F081918D9350
:10057000FACFC80126E0969587952A95E1F7807E07
:1005800019830A830115104C10F48461D7CF8C6154
:10059000D5CFB6016D5F7F4FCE0101960E94F371FA
:1005A0000E940D72C60128960FB6F894DEBF0FBEEA
:1005B000CDBFDF91CF911F910F91FF90EF90DF9012
:1005C000CF90BF90AF90089563E070E0CE010196A8
:1005D0000E94F371F70181917F010E942272AE1493
:1005E000BF04C1F7DDCFCF93DF931F92CDB7DEB746
:1005F000898341E050E0BE016F5F7F4F90E080E073
:100600000E9445820F90DF91CF9108951F93CF9361
:10061000DF931F921F92CDB7DEB78091160981112B
:1006200000C160E372E080E090E00E94A8941FB7F0
:10063000F89480911509811127C0E2EAF9E18491CB
:10064000E8EFF9E19491E82FF0E0EE0FFF1FE75C8F
:10065000F64EA591B491EC91E92321F461E085E394
:100660000E94229361E085E30E9450938CB58061E3
:100670008CBD8CB580648CBD61E084E30E94509396
:1006800061E083E30E945093809115098F5F80930E
:1006900015091FBFE7E7F9E1E491F0E0EE0FFF1F56
:1006A000ED5AF64E85919491909314098093130915
:1006B000EDECF9E1E491E093120961E08AE00E9437
:1006C00050930E940D7280E591E00E94019084E3B6
:1006D00080934F0A80E80E94F3820E94D874882396
:1006E000A1F188E00E94F3820E94D474883069F5F9
:1006F00080E10E94F3820E94D474803131F580E061
:100700000E94F3820E94D474182F81111EC08FE1C1
:1007100090E00E9494268330C1F480E4809306091F
:1007200042E06EE170E0812F0E94772642E06FE1A7
:1007300070E0812F0E9477261F5F183089F70E9492
:10074000BB2781E08093160966C087E380934F0A38
:1007500080E80E94F3820E94D8748823F9F088E030
:100760000E94F3820E94D4748830C1F480E10E9418
:10077000F3820E94D474182F803181F480E00E94AB
:10078000F3820E94D474811109C089E390E00E9431
:100790009426843019F410930609D1CF83E3809313
:1007A0004F0A80E80E94F3820E94D874882371F176
:1007B00080E10E94F3820E94D474803139F582E195
:1007C0000E94F3820E94D474823101F580E00E947D
:1007D000F3820E94D474811119C084E080930609C9
:1007E00015E51A8341E050E0BE016E5F7F4F8BE15B
:1007F00090E00E944582198341E050E0BE016F5FA6
:100800007F4F8AE190E00E94458299CF10924F0A73
:100810000E94BB2780E00F900F90DF91CF911F9136
:10082000089581E0F8CF6F927F929F92AF92BF922E
:10083000CF92DF92EF92FF920F931F93CF93DF93AC
:100840001F921F92CDB7DEB7982E8B013A01690136
:1008500022E030E0AE014F5F5F4F64E270E00E9443
:100860009527E980FA80FE24EF24FE24E00EF11E95
:100870009701377040914F0A092D10E0C8014333AA
:1008800009F04CC00896982F8827990F990F990F57
:10089000820F931F473309F446C0A9014C0D5D1D1B
:1008A0004130584008F43FC060E078E05B01A21A94
:1008B000B30AA501B3010E944582A6014A195B094A
:1008C000B3016A0D7B1D80914F0A833349F5085FA0
:1008D0001F4F000F000F000F80E0902F0E944582F5
:1008E000EC0CFD1CF982EA8222E030E0AE014F5FA1
:1008F0005F4F64E270E0892D0E9466260F900F9092
:10090000DF91CF911F910F91FF90EF90DF90CF90EB
:10091000BF90AF909F907F906F9008954096B3CF17
:10092000005F1F4FD6CFA601B301D8CFEF92FF9241
:100930001F93CF93DF931F921F92CDB7DEB7182F6F
:1009400022E030E0AE014F5F5F4F60E270E00E9456
:100950009527E980FA80FE24EF24FE2422E030E08F
:10096000AE014F5F5F4F60E270E0812F0E949527DC
:1009700089819A81982789279827E816F90689F4AA
:1009800087E0189FF0011124E95FF54FF582E482BA
:10099000C7010F900F90DF91CF911F91FF90EF90C3
:1009A00008957C01DBCF1F93CF93DF93182F80E551
:1009B00091E00E940190812F0E949684EC01812F8A
:1009C0000E94B326182F0E94BB27173121F01C313B
:1009D00011F0D0E0C0E0CE01DF91CF911F910895DA
:1009E000CF92DF92EF92FF920F931F93CF93DF93FB
:1009F000182F7B01EA014130584010F0C0E0D8E0E8
:100A000080E591E00E940190812F0E9496846C0104
:100A1000812F0E94B326082F0E94BB27073111F0B7
:100A20000C3169F5CC16DD0658F380E591E00E94A3
:100A300001909E01A70170E060E0812F0E94138465
:100A400060E270E0812F0E94AA8162E070E0812F55
:100A50000E94A52684FD1DC0812F0E94B32681110E
:100A600011C00E94BB27D0E0C0E0CE01DF91CF9142
:100A70001F910F91FF90EF90DF90CF900895D0E0FD
:100A8000C0E0D3CF0E94BB2780E591E00E94019097
:100A9000DCCF40E162E070E0812F0E9477260E9467
:100AA000BB27E3CF1F93CF93DF931F92CDB7DEB762
:100AB000182F80E591E00E940190812F0E942972F9
:100AC00027E0129FF0011124E95FF54F2281338165
:100AD000377041E050E0BE016F5F7F4F820F931F80
:100AE0000E94BA810E94BB2789810F90DF91CF912C
:100AF0001F9108950F931F93CF93DF93C82F27E083
:100B0000829F80011124095F154FF8018081918136
:100B1000009791F480E591E00E9401908C2F0E9453
:100B2000EE74EC010E94BB27F80186819E01281B10
:100B30003109C90131832083DF91CF911F910F913A
:100B400008954F925F927F928F929F92AF92BF9241
:100B5000CF92DF92EF92FF920F931F93CF93DF9389
:100B60001F921F92CDB7DEB7782E6B014A01A82ED7
:100B7000B12C27E0829FC0011124FC01E95FF54FF1
:100B80007F010081118180E591E00E9401900815AC
:100B9000190554F4872D0E94EE74F70126818C010B
:100BA000021B1109118300830115110529F5872DF9
:100BB0000E94B326843159F0882349F001E010E007
:100BC0008C3111F410E000E01195019511090E949B
:100BD000BB27C8010F900F90DF91CF911F910F910C
:100BE000FF90EF90DF90CF90BF90AF909F908F904D
:100BF0007F905F904F900895801691060CF48401C9
:100C000087E08A9DF0018B9DF00D1124E95FF54F7F
:100C1000E280F380C114D10451F12701F7E05F2293
:100C2000872D0E942972840D951D20914F0A27332C
:100C300009F453C09801240D351D2130384008F4C3
:100C40004CC020E038E0490184189508A401B601A1
:100C50000E94BA812601480C591C6801C818D9089D
:100C6000872D0E942972A601B2010E94BA81E00E6E
:100C7000F11E87E08A9DF0018B9DF00D1124E95F44
:100C8000F54FF382E28220813181201B310B3183C9
:100C900020838681800F912F911D8A3F910510F44A
:100CA000232BF1F487E08A9DF0018B9DF00D112438
:100CB000E95FF54F1682F982EA8222E030E0AE0168
:100CC0004F5F5F4F68E270E0872D0E94662660E408
:100CD00070E0872D0E94AA817ACFA801B601C5CF06
:100CE000868375CFCF93C82F80E591E00E94019055
:100CF00068E070E08C2F0E94AA81CF910C94BB27F2
:100D0000CF93C82F80E591E00E94019060E170E0F0
:100D10008C2F0E94AA81CF910C94BB27CF93C82F10
:100D200080E591E00E9401908C2F0E94B326C82F8D
:100D30000E94BB278C2FCF910895CF93DF931F92F2
:100D40001F92CDB7DEB779836A8322E030E0AE012F
:100D50004F5F5F4F60E170E00E9466260F900F903A
:100D6000DF91CF910895CF93DF931F921F92CDB75C
:100D7000DEB779836A8322E030E0AE014F5F5F4FD8
:100D800064E070E00E9466260F900F90DF91CF9193
:100D900008958F929F92AF92BF92CF92DF92EF927F
:100DA000FF920F931F93CF93DF9300D000D000D01A
:100DB0001F92CDB7DEB790914F0A992369F128E0D1
:100DC000F22E933311F494E0F92E6B01082F80E595
:100DD00091E00E9401909E012F5F3F4F5901490110
:100DE00010E0812F0E94B326F40181934F018823E4
:100DF000D9F01F5FF112F5CFF12CF50191915F0150
:100E00009D3161F0983151F09A51923038F0F3945D
:100E10001F11F3CF0E94BB2718E05EC060E170E0B5
:100E20008F2D0E94AA811F2DE12EF12CF701EE0FCC
:100E3000FF1FE15CF54F118210820E940490402F49
:100E400070E060E0812F0E9477264FEF62E070E053
:100E5000812F0E947726B601CD2891F480912C0233
:100E600090912D0201968115F0EC9F0708F448C07F
:100E700090932D0280932C0260912C0270912D0290
:100E8000812F0E94B38661E070E0812F0E94AA81C9
:100E900027E02E9DC0012F9D900D11249C01295FFC
:100EA000354F7901F9011182108222E030E0AE0164
:100EB000475F5F4F68E270E0812F0E949527898528
:100EC0009A85982789279827F7019383828316822A
:100ED000158214820E94BB27812F2A960FB6F894A0
:100EE000DEBF0FBECDBFDF91CF911F910F91FF905D
:100EF000EF90DF90CF90BF90AF909F908F9008952C
:100F000080E090ECB5CF2F923F924F925F926F921C
:100F10007F928F929F92AF92BF92CF92DF92EF9289
:100F2000FF920F931F93CF93DF9300D000D01F92B7
:100F30001F92CDB7DEB78C016B010E94E47F019652
:100F400019F48FEF9FEF1DC0D801ED91FC91028441
:100F5000F385E02DC80119957C018F3F980789F32F
:100F6000D801ED91FC910684F785E02D682FC8012A
:100F70001995B2E2EB16F104E9F4B601C8010E943A
:100F8000018028960FB6F894DEBF0FBECDBFDF916B
:100F9000CF911F910F91FF90EF90DF90CF90BF9076
:100FA000AF909F908F907F906F905F904F903F9009
:100FB0002F900895EDE2EE16F10429F0C701C097D5
:100FC0000A9708F043C1D801ED91FC910284F385A2
:100FD000E02DC80119957C018F3F980709F4B1CF26
:100FE0008D9799F5D801ED91FC910284F385E02D60
:100FF000C80119957C01019609F4A3CFEFEFFFEF2B
:10100000F887EF83C701C097812C912C54010A9770
:1010100008F5AAE0B0E0A50194010E94C1BE30E34A
:10102000E31AF1084701FF0CAA08BB08860E971EB9
:10103000A81EB91ED801ED91FC910284F385E02D24
:10104000C80119957C01C097E2CF21E030E03887D4
:101050002F83D8CFBEE2EB16F10401F1C7018F7DDB
:1010600085349105D9F0AF81B885A50194010E941E
:10107000CCBEF60161877287838794878085807FE5
:1010800082608087D801ED91FC910684F785E02D80
:101090006E2DC801199590E080E073CFC501B401B1
:1010A0000E943DBD2B013C01312C212CFEE2EF16AC
:1010B000F10499F5D801ED91FC910284F385E02DBE
:1010C000C80119957C01312C212C20E030E040E250
:1010D00051E4C301B2010E949CBD4B015C01B70108
:1010E00060537109072E000C880B990B0E943DBDBF
:1010F000A50194010E942ABF2B013C01B1E02B1AEB
:101100003108D801ED91FC910284F385E02DC801EE
:1011100019957C01C0970A97C0F2C7018F7D85346D
:10112000910509F040C0D801ED91FC910284F3854E
:10113000E02DC80119957C01D801ED91FC918B320D
:10114000910519F50284F385E02DC80119957C01FC
:10115000E1E0EE83B12CA12C8AE0982ED801ED912C
:10116000FC91C701C0978A30910508F59A9C9001BF
:101170009B9C300D11245C01A20EB31E0284F385EA
:10118000E02DC80119957C01E9CF8D9749F40284BF
:10119000F385E02DC80119957C013FEF3E83DACF3E
:1011A00081E08E83D7CFB1E0BE83B12CA12CEF813B
:1011B000F885BF01FF0F880B990B0E943DBDA3016D
:1011C00092010E949CBD2B013C01B501BB0C880B18
:1011D000990B0E943DBD4B015C01FE816F2FFF0FFB
:1011E000770B880B990B0E943DBD9B01AC01C5019B
:1011F000B4010E949CBD4B015C01B101330C880B12
:10120000990B0E943DBD9B01AC01C501B4010E9438
:101210002ABF9B01AC0160E070E080E291E40E9493
:1012200043C09B01AC01C301B2010E949CBDD60129
:1012300019966D937D938D939C931C9718968C9122
:101240001897807F836018968C931CCFBBE5EB16B4
:10125000F10409F062C0D801ED91FC910284F3859C
:10126000E02DC80119958B35910509F06ACEF6017C
:101270008085807F85608087C8010E94E47FD801D7
:10128000ED91FC910284F385E02DC80119958D350F
:10129000910509F400CFD801ED91FC910684F78502
:1012A000E02D682FC8011995BB24BA940E94C18013
:1012B0007C01009709F445CEBB2031F1F6019783FC
:1012C0008683C8010E94E47FB701C8010E9483871A
:1012D000892B09F036CEC8010E94E47FD801ED9138
:1012E000FC910284F385E02DC8011995B12C4701CA
:1012F0008C329105D9F221E030E08D35910509F06D
:101300008DC030E020E08AC0D40113969C938E9368
:101310001297FC0195828482D4CFBBE7EB16F104CF
:1013200009F08AC0D801ED91FC910284F385E02D8B
:10133000C80119958B37910509F003CEF601808518
:10134000807F86608087C8010E94E47FD801ED918C
:10135000FC910284F385E02DC80119958D37910524
:1013600009F499CED801ED91FC910684F785E02D22
:10137000682FC801199599249A940E94C1807C0114
:10138000009709F4DECD992009F44DC0F60197834A
:101390008683C8010E94E47FB701C8010E940180D2
:1013A000019609F4CECDC8010E94E47FD7011996B9
:1013B0008D919C911A9711969C938E931A961C92DC
:1013C0001E921997D801ED91FC910284F385E02DCE
:1013D000C8011995CA9709F0B4CDC8010E94E47FED
:1013E000B701C8010E948387019609F4AACDC801FC
:1013F0000E94E47FD801ED91FC910284F385E02DF9
:10140000C8011995912C57018C32910509F4B5CF7B
:1014100021E030E08D37910509F473CF88279927B3
:10142000821B930BAECDD50113969C938E9312978E
:10143000FC01B582A482ADCFBEE6EB16F10421F526
:1014400019821A821B821C82D801ED91FC910484BE
:10145000F585E02D44E050E0BE016F5F7F4FC8018D
:101460001995049709F06DCD44E050E069EA76E003
:10147000CE0101960E9484C3009709F062CDF60167
:101480002085207F20877DCDF6E6EF16F10441F51B
:101490009E012F5F3F4F790185E0D9011D928A950A
:1014A000E9F7D801ED91FC910484F585E02D45E044
:1014B00050E0B901C8011995059709F042CD45E002
:1014C00050E063EB76E0C7010E9484C3009709F007
:1014D00038CDF6012085207F21602087118651CDEF
:1014E000F4E7EF16F10409F02CCD19821A821B8261
:1014F0001C82D801ED91FC910484F585E02D44E037
:1015000050E0BE016F5F7F4FC8011995049709F045
:1015100018CD44E050E06EEA76E0CE0101960E94DC
:1015200084C3009709F00DCDF6012085207F21604E
:10153000208721E0218725CD0F931F93CF93DF9341
:101540008B01FC01C681D781209759F0B8018881B1
:1015500099810E943BC3892B21F00A80DB81C02D39
:10156000F3CFCE01DF91CF911F910F91089580911C
:101570006C0C90916D0C009711F480E02FC0DC0191
:10158000ED91FC910688F789E02D199520918F0C3B
:101590003091900C81111FC0232B79F78DEF9FEFB5
:1015A0009093900C80938F0C80916C0C90916D0CAB
:1015B000DC01ED91FC910680F781E02D1995809179
:1015C0006C0C90916D0CDC01ED91FC910488F58917
:1015D000E02D1995D2CF81E0232B79F60895CF9392
:1015E000DF93EC01FA013296E60FF71FDC019D0153
:1015F0002C1B3D0BCF01861B970B4D91442311F003
:101600004193F5CFAC01421B530B640F751FFB01D7
:101610003297308361507109FB012083DF91CF91B4
:101620000895462F50E070E060E02AE00C94757752
:10163000FC0186819781009739F0662329F061507B
:10164000FC0182819381F7CF0895AB01770F660B80
:10165000770B2AE030E00C94DE77DC011696ED91F2
:10166000FC9180E0309729F08F5F0280F381E02DBC
:10167000F9CF0895E091C70CF091C80C128A118A35
:10168000148A138A84E690E095878487168680E022
:1016900090E3908B87870895CF93DF9387E70E942D
:1016A0003A8B8091C70C9091C80CDC01ED91FC91B4
:1016B0000684F785E02D70E060E01995D0E0C0E089
:1016C0008091C70C9091C80CDC01ED91FC911197B1
:1016D0001C962D913C91C217D30738F40190F081EC
:1016E000E02D60E019952196EBCF0684F785E02D7B
:1016F00070E060E01995CDE2D3E08091C70C909145
:10170000C80C6991DC01ED91FC910190F081E02D14
:101710001995B3E0C133DB0781F78091C70C909135
:10172000C80CDC01ED91FC910288F389E02D19953C
:1017300081E0DF91CF910895CF93DF938091C70C23
:101740009091C80C892B99F182E70E943A8B809185
:10175000C70C9091C80CDC01ED91FC910684F785D3
:10176000E02D70E060E01995CDE2D3E0B3E0C13345
:10177000DB0709F18091C70C9091C80CDC01ED9159
:10178000FC910284F385E02D19952991022E000C1D
:10179000330B8217930751F38091C70C9091C80CBB
:1017A000DC01ED91FC910288F389E02D199580E030
:1017B000DF91CF91089581E0FBCFAF92BF92CF929E
:1017C000DF92EF92FF920F931F93CF93DF935C0111
:1017D0007B018B01040F151FEB016E01CE18DF0892
:1017E000C017D10741F0C5010E94157718161906D8
:1017F00014F48993F2CFC601DF91CF911F910F911D
:10180000FF90EF90DF90CF90BF90AF900895CF936F
:10181000DF932091C70C3091C80C232B11F480E08A
:1018200041C0EC010E949C8B8823C9F3FE0101900A
:101830000020E9F73197EC1BFD0B709780F782E7EA
:101840000E943A8B8091C70C9091C80CDC01ED91FD
:10185000FC910684F785E02D6CE370E01995BE01DC
:101860008091C70C9091C80C0E9464788091C70C3D
:101870009091C80CDC01ED91FC910190F081E02D7C
:1018800060E01995EC018091C70C9091C80CDC01C7
:10189000ED91FC910288F389E02D199581E0CD2B23
:1018A00009F4BDCFDF91CF910895CF93DF932091BD
:1018B000C70C3091C80C232B11F480E041C0EC011F
:1018C0000E949C8B8823C9F3FE0101900020E9F758
:1018D0003197EC1BFD0B709780F782E70E943A8BE3
:1018E0008091C70C9091C80CDC01ED91FC910684AD
:1018F000F785E02D6CE470E01995BE018091C70C6E
:101900009091C80C0E9464788091C70C9091C80C8B
:10191000DC01ED91FC910190F081E02D60E01995E2
:10192000EC018091C70C9091C80CDC01ED91FC9109
:101930000288F389E02D199581E0CD2B09F4BDCF04
:10194000DF91CF9108950F931F93CF93DF9300D032
:101950001F92CDB7DEB7FC0182819381A481B5814E
:1019600089839A83AB83BC838091C70C9091C80C08
:10197000892B11F480E033C00E949C8B8823D1F323
:1019800082E70E943A8B8091C70C9091C80CDC01D1
:10199000ED91FC910684F785E02D6CE070E01995DF
:1019A0008091C70C9091C80CDC01ED91FC910280F4
:1019B000F381E02D44E050E0BE016F5F7F4F199549
:1019C0008C018091C70C9091C80CDC01ED91FC91C9
:1019D0000288F389E02D199581E0012B59F20F90CF
:1019E0000F900F900F90DF91CF911F910F9108955D
:1019F0000F931F93CF93DF9300D01F92CDB7DEB725
:101A0000FC0182819381A481B58189839A83AB8310
:101A1000BC838091C70C9091C80C892B11F480E095
:101A200033C00E949C8B8823D1F382E70E943A8BBB
:101A30008091C70C9091C80CDC01ED91FC9106845B
:101A4000F785E02D68E170E019958091C70C9091C1
:101A5000C80CDC01ED91FC910280F381E02D44E0A3
:101A600050E0BE016F5F7F4F19958C018091C70CCC
:101A70009091C80CDC01ED91FC910288F389E02D76
:101A8000199581E0012B59F20F900F900F900F9054
:101A9000DF91CF911F910F9108950F931F93CF93D3
:101AA000DF9300D01F92CDB7DEB7FC018281938116
:101AB000A481B58189839A83AB83BC838091C70C51
:101AC0009091C80C892B11F480E033C00E949C8B4C
:101AD0008823D1F382E70E943A8B8091C70C9091C2
:101AE000C80CDC01ED91FC910684F785E02D60E1E6
:101AF00070E019958091C70C9091C80CDC01ED91B4
:101B0000FC910280F381E02D44E050E0BE016F5F64
:101B10007F4F19958C018091C70C9091C80CDC0106
:101B2000ED91FC910288F389E02D199581E0012B5C
:101B300059F20F900F900F900F90DF91CF911F915E
:101B40000F9108950F931F93CF93DF9300D01F92AF
:101B5000CDB7DEB7FC0182819381A481B5818983F1
:101B60009A83AB83BC838091C70C9091C80C892B5E
:101B700011F480E033C00E949C8B8823D1F382E76C
:101B80000E943A8B8091C70C9091C80CDC01ED91BA
:101B9000FC910684F785E02D64E170E01995809151
:101BA000C70C9091C80CDC01ED91FC910280F3818F
:101BB000E02D44E050E0BE016F5F7F4F19958C012E
:101BC0008091C70C9091C80CDC01ED91FC910288CA
:101BD000F389E02D199581E0012B59F20F900F90B8
:101BE0000F900F90DF91CF911F910F910895AB014E
:101BF00070E060E02AE00C94757761157105C1F022
:101C0000DC011696ED91FC911797309731F41796F9
